:100000000C9443510C9474510C9474510C9474518D
:100010000C9474510C9474510C9474510C9474514C
:100020000C9474510C9474510C9474510C9474513C
:100030000C944E750C9474510D94A3140D94E71107
:100040000C9474510D943C220C9474510C94745182
:100050000C9474510C9474510C9474510C94CE6D96
:100060000C9474510D94E6990C9474510C94745141
:100070000C9474510C94F57D0C9474510C9474513F
:100080000D94ED160C9474510C9474510C9474519D
:100090000D94A2990C9474510C9474510C94745155
:1000A0000C9474510C9474510D94420D0C94745131
:1000B0000C9474510D94370D0C9474510C9474512C
:1000C0000C9474510C9474510C9474510D94F70C5D
:1000D0000C9474510C9474510C9474510C9474518C
:1000E0000C947451000000000000000000000000AB
:1000F0000000000000000000000000000000000000
:100100005F5345435F4C414E470000000000000034
:1001100000000000000000000000000000000000DF
:1001200000000000000000000000000000000000CF
:1001300000000000000000000000000000000000BF
:1001400000000000000000000000000000000000AF
:103600000000536F6D652070726F626C656D206590
:103610006E636F756E74657265642C205A2D6C65CF
:1036200076656C696E6720656E666F72636564208F
:103630002E2E2E0001004D65736820626564206C9B
:103640006576656C696E67206661696C65642E20BD
:103650005072696E742063616E63656C65642E00E0
:10366000020048656174696E672064697361626C09
:103670006564206279207361666574792074696D70
:1036800065722E000300472D636F646520736C69BB
:1036900063656420666F7220612064696666657286
:1036A000656E74206C6576656C2E20436F6E746950
:1036B0006E75653F000400472D636F646520736C71
:1036C0006963656420666F7220612064696666655F
:1036D00072656E74206C6576656C2E20506C656129
:1036E00073652072652D736C69636520746865204D
:1036F0006D6F64656C20616761696E2E2050726920
:103700006E742063616E63656C6C65642E000500E9
:10371000472D636F646520736C6963656420666F11
:10372000722061206E65776572206669726D7761BF
:1037300072652E20436F6E74696E75653F000600DA
:10374000472D636F646520736C6963656420666FE1
:10375000722061206E65776572206669726D77618F
:1037600072652E20506C656173652075706461749C
:103770006520746865206669726D776172652E20B8
:103780005072696E742063616E63656C6C65642E43
:10379000000700472D636F646520736C696365647F
:1037A00020666F72206120646966666572656E745A
:1037B000207072696E74657220747970652E204372
:1037C0006F6E74696E75653F000800472D636F6406
:1037D0006520736C6963656420666F722061206484
:1037E0006966666572656E74207072696E74657262
:1037F00020747970652E20506C6561736520726548
:103800002D736C69636520746865206D6F64656CE9
:1038100020616761696E2E205072696E7420636149
:103820006E63656C6C65642E00090050726573737D
:1038300020746865206B6E6F6220746F20707265F3
:1038400068656174206E6F7A7A6C6520616E6420A1
:10385000636F6E74696E75652E000A00506C656149
:10386000736520707265737320746865206B6E6F6A
:103870006220746F20756E6C6F61642066696C6184
:103880006D656E74000B00616E64207072657373F9
:1038900020746865206B6E6F62000C00496E736562
:1038A00072742066696C616D656E74000D00436F03
:1038B0006C6F72206E6F7420636F72726563740038
:1038C0000E0046696C616D656E74206E6F74206CBD
:1038D0006F61646564000F004368616E6765642012
:1038E000636F72726563746C790010004C6F616471
:1038F000696E6720636F6C6F720011004368616EC0
:103900006765207375636365737321001200506CE3
:1039100065617365206F70656E2069646C657220E7
:10392000616E642072656D6F76652066696C616D8D
:10393000656E74206D616E75616C6C792E0013007C
:103940005761732066696C616D656E7420756E6C6D
:103950006F6164207375636365737366756C3F0094
:103960001400506C656173652075706772616465E1
:103970002E0015004E6577206669726D776172655D
:103980002076657273696F6E20617661696C616221
:103990006C653A00160057616974696E6720666F3E
:1039A000722050494E44412070726F626520636FEF
:1039B0006F6C696E67001700506C656173652077E6
:1039C0006169740018004E6F206D6F76652E0019C6
:1039D000005761697420666F7220757365722E2EB0
:1039E0002E001A00537461626C6520616D62696516
:1039F0006E742074656D70657261747572652032C5
:103A0000312D323643206973206E6565646564200C
:103A100061207269676964207374616E64206973E0
:103A20002072657175697265642E001B00506C65AB
:103A30006173652072756E2058595A2063616C69F4
:103A400062726174696F6E2066697273742E001CF5
:103A500000506C6561736520756E6C6F61642074D5
:103A600068652066696C616D656E74206669727345
:103A7000742C207468656E207265706561742074A2
:103A800068697320616374696F6E2E001D0043685E
:103A900065636B73001E004E6F7A7A6C6520642E2E
:103AA000001F00416C706861626574002000536FF4
:103AB000727400210054696D650022004E6F726DB2
:103AC000616C00230053442063617264002400533E
:103AD000656C656374206C616E6775616765002550
:103AE000004E6F7A7A6C65206368616E67650026A8
:103AF0000048572053657475700027004C6F61644F
:103B0000696E6720546573740028004469736162AC
:103B10006C652073746570706572730029004D6F59
:103B200076652061786973002A0054656D7065724E
:103B30006174757265002B0050494E4441206361E9
:103B40006C2E002C0052657365742058595A2063FE
:103B5000616C6962722E002D0053686F7720656E6C
:103B6000642073746F7073002E00504944206361A9
:103B70006C6962726174696F6E002F004265642027
:103B80006C6576656C20636F7272656374003000DB
:103B90004D65736820426564204C6576656C696E7E
:103BA0006700310043616C696272617465205A007C
:103BB000320043616C6962726174652058595A0021
:103BC000330053656C667465737400340057697A0A
:103BD00061726400350054657374696E67206669AC
:103BE0006C616D656E740036004C6F616420416CD1
:103BF0006C003700506C656173652070756C6C20CB
:103C00006F75742066696C616D656E7420696D6D89
:103C10006564696174656C79003800526573657418
:103C200000390052656E616D65003A004669727335
:103C300074206C617965722063616C2E003B0053C7
:103C4000656C656374003C00537465656C20736833
:103C500065657473003D00537570706F7274003E3B
:103C6000004661696C207374617473204D4D55007A
:103C70003F004661696C20737461747300400053A7
:103C800074617469737469637300410043616C69A2
:103C900062726174696F6E0042004175746F4C6F9F
:103CA00061642066696C616D656E740043004C6FE1
:103CB00061642066696C616D656E74004400556EC8
:103CC0006C6F61642066696C616D656E740045009F
:103CD0004C6F616420746F206E6F7A7A6C65004659
:103CE000005072656C6F616420746F204D4D5500FB
:103CF00047004E6F205344206361726400480050B7
:103D000072696E742066726F6D20534400490052D0
:103D10006573756D65207072696E74004A0050613C
:103D2000757365207072696E74004B005365742062
:103D30005265616479004C00536574206E6F742085
:103D40005265616479004D00507265686561740068
:103D50004E0054756E65004F004C697665206164B5
:103D60006A757374205A00500052657072696E74DF
:103D7000005100496E666F2073637265656E005274
:103D8000004173736973740053004F6E6365005490
:103D900000536F756E640055004C6F7564005600DB
:103DA00046696C2E2073656E736F7200570043680E
:103DB000616E67652066696C616D656E74005800A0
:103DC000466C6F770059005370656564005A004D6A
:103DD00061676E65747320636F6D702E005B004EBB
:103DE0002F41005C005A2D70726F6265206E722E3A
:103DF000005D004D657368005E0053657474696E04
:103E00006773005F005965730060004E6F006100CA
:103E100053746F70207072696E740062004368653D
:103E2000636B696E672066696C6500630046696C48
:103E30006520696E636F6D706C6574652E20436FCD
:103E40006E74696E756520616E797761793F006483
:103E50000084526566726573680065004D61696E25
:103E600000660057616974696E6720666F72206E24
:103E70006F7A7A6C6520616E642062656420636F7E
:103E80006F6C696E6700670053656C6563742066CC
:103E9000696C616D656E743A00680053656C667498
:103EA000657374204F4B00690053656C66746573CD
:103EB00074207374617274006A0053776170706566
:103EC00064006B0046726F6E742F6C6566742066BA
:103ED000616E73006C0041786973006D0041786910
:103EE00073206C656E677468006E004C6F6F73654D
:103EF0002070756C6C6579006F00456E6473746F2B
:103F000070206E6F7420686974007000456E647371
:103F1000746F700071004D6F746F72007200456EA7
:103F20006473746F7073007300576972696E6720F1
:103F30006572726F720074004265642F4865617427
:103F400065720075004E6F7420636F6E6E656374EA
:103F500065640076004865617465722F5468657207
:103F60006D6973746F72007700506C6561736520C2
:103F7000636865636B3A00780053656C66746573BB
:103F800074206572726F722100790046696C616DF0
:103F9000656E742073656E736F72007A005072697B
:103FA0006E742066616E3A007B00486F74656E64C3
:103FB0002066616E3A007C0043616C6962726174D4
:103FC000696E6720686F6D65007D0053656C66746F
:103FD000657374206661696C6564007E00416C6C79
:103FE00020636F7272656374007F00436865636B62
:103FF000696E672073656E736F727300800043682B
:1040000065636B696E6720686F74656E640081001C
:10401000436865636B696E67206265640082004374
:104020006865636B696E67205A20617869730083E5
:1040300000436865636B696E672059206178697316
:10404000008400436865636B696E6720582061785F
:104050006973008500436865636B696E6720656EF0
:104060006473746F707300860043617264207265BC
:104070006D6F7665640087004261636B0088004164
:1040800075746F20706F77657200890053696C6575
:104090006E74008A004D6F6465008B004869676824
:1040A00020706F776572008C0053747269637400BE
:1040B0008D005761726E008E004E6F6E65008F002E
:1040C000486F74656E64206174203238304321205B
:1040D0004E6F7A7A6C65206368616E6765642061F3
:1040E0006E64207469676874656E656420746F20FF
:1040F00073706563733F009000466F722061204EBD
:104100006F7A7A6C65206368616E676520706C6594
:1041100061736520726561640A70727573612E69DE
:104120006F2F6E6F7A7A6C652D6D6B337300910013
:104130005049442063616C2E2066696E697368651E
:10414000640092005049442063616C2E009300503B
:1041500072696E74207061757365640094005072AA
:10416000696E742061626F72746564009500436FBC
:1041700070792073656C6563746564206C616E672B
:10418000756167653F0096004E6F7A7A6C652064B2
:1041900069616D6574657220646966666572732015
:1041A00066726F6D2074686520472D636F64652E9D
:1041B00020436F6E74696E75653F0097004E6F7A8D
:1041C0007A6C65206469616D6574657220646966E6
:1041D000666572732066726F6D2074686520472D66
:1041E000636F64652E20506C65617365206368653C
:1041F000636B207468652076616C756520696E203C
:1042000073657474696E67732E205072696E7420C2
:1042100063616E63656C6C65642E0098005468651C
:104220007265206973206E6F2066696C616D656EC2
:1042300074206C6F616465642E20436F6E74696EC8
:1042400075653F0099005468657265206973206E3A
:104250006F2066696C616D656E74206C6F6164655A
:10426000642E205072696E742063616E63656C6C9D
:1042700065642E009A005468657265206973207326
:1042800074696C6C2061206E65656420746F206DAC
:10429000616B65205A2063616C6962726174696F39
:1042A0006E2E20506C6561736520666F6C6C6F7745
:1042B00020746865206D616E75616C2C2063686187
:1042C00070746572204669727374207374657073BC
:1042D0002C2073656374696F6E2043616C69627230
:1042E0006174696F6E20666C6F772E009B00507250
:1042F000696E74657220686173206E6F74206265E8
:10430000656E2063616C69627261746564207965B1
:10431000742E20506C6561736520666F6C6C6F77CE
:1043200020746865206D616E75616C2C2063686116
:10433000707465722046697273742073746570734B
:104340002C2073656374696F6E2043616C696272BF
:104350006174696F6E20666C6F772E009C005365E8
:104360006C66746573742077696C6C20626520726A
:10437000756E20746F2063616C6962726174652070
:1043800061636375726174652073656E736F726CBF
:10439000657373207265686F6D696E672E009D008E
:1043A0004F6C642073657474696E677320666F75F3
:1043B0006E642E2044656661756C74205049442CEF
:1043C00020457374657073206574632E2077696C63
:1043D0006C206265207365742E009E005761726EBA
:1043E000696E673A20626F7468207072696E7465D6
:1043F00072207479706520616E64206D6F746865D9
:1044000072626F6172642074797065206368616E96
:104410006765642E009F005761726E696E673A206F
:104420007072696E7465722074797065206368615A
:104430006E6765642E00A0005761726E696E673A00
:10444000206D6F74686572626F6172642074797038
:1044500065206368616E6765642E00A1005368651E
:10446000657400A2004E6F74207370696E6E696E81
:104470006700A3005370696E6E696E6700A4004CFC
:1044800065667420686F74656E642066616E3F00B7
:10449000A50046726F6E74207072696E742066613A
:1044A0006E3F00A60046616E207465737400A7001D
:1044B00058595A2063616C6962726174696F6E2029
:1044C000616C6C2072696768742E20536B6577206D
:1044D00077696C6C20626520636F727265637465C6
:1044E00064206175746F6D61746963616C6C792EA1
:1044F00000A80058595A2063616C6962726174693E
:104500006F6E20616C6C2072696768742E20582F62
:104510005920617865732061726520736C696768E2
:10452000746C7920736B657765642E20476F6F64B8
:10453000206A6F622100A90058595A2063616C6992
:1045400062726174696F6E206F6B2E20582F592034
:1045500061786573206172652070657270656E6444
:104560006963756C61722E20436F6E67726174753A
:104570006C6174696F6E732100AA0058595A2063E8
:10458000616C6962726174696F6E20636F6D7072C5
:104590006F6D697365642E20526967687420667256
:1045A0006F6E742063616C6962726174696F6E20F2
:1045B000706F696E74206E6F7420726561636861DC
:1045C000626C652E00AB0058595A2063616C6962B9
:1045D000726174696F6E20636F6D70726F6D697355
:1045E00065642E2046726F6E742063616C6962721E
:1045F0006174696F6E20706F696E7473206E6F7472
:1046000020726561636861626C652E00AC00585968
:104610005A2063616C6962726174696F6E206661B1
:10462000696C65642E2052696768742066726F6ECB
:10463000742063616C6962726174696F6E20706F5F
:10464000696E74206E6F7420726561636861626C5C
:10465000652E00AD0058595A2063616C6962726121
:1046600074696F6E206661696C65642E2046726F96
:104670006E742063616C6962726174696F6E207020
:104680006F696E7473206E6F742072656163686108
:10469000626C652E00AE0058595A2063616C6962E5
:1046A000726174696F6E206661696C65642E20505A
:1046B0006C6561736520636F6E73756C74207468CC
:1046C00065206D616E75616C2E00AF0058595A20DF
:1046D00063616C6962726174696F6E206661696C96
:1046E00065642E204265642063616C696272617446
:1046F000696F6E20706F696E7420776173206E6FC2
:104700007420666F756E642E00B000506C65617326
:104710006520706C61636520737465656C207368D7
:10472000656574206F6E20686561746265642E0033
:10473000B10044697374616E636520626574776566
:10474000656E20746970206F6620746865206E6FD6
:104750007A7A6C6520616E64207468652062656495
:10476000207375726661636520686173206E6F7473
:10477000206265656E20736574207965742E205003
:104780006C6561736520666F6C6C6F77207468650B
:10479000206D616E75616C2C206368617074657248
:1047A0002046697273742073746570732C2073656E
:1047B0006374696F6E204669727374206C617965E9
:1047C000722063616C6962726174696F6E2E00B2EF
:1047D00000506C6163652061207368656574206FAB
:1047E0006620706170657220756E646572207468F1
:1047F00065206E6F7A7A6C6520647572696E6720C9
:104800007468652063616C6962726174696F6E209F
:104810006F66206669727374203420706F696E74DD
:10482000732E20496620746865206E6F7A7A6C65F5
:1048300020636174636865732074686520706170BB
:1048400065722C20706F776572206F6666207468C1
:1048500065207072696E74657220696D6D6564693A
:104860006174656C792E00B3005365617263686989
:104870006E67206265642063616C6962726174694D
:104880006F6E20706F696E7400B4004D6561737552
:1048900072696E67207265666572656E6365206811
:1048A0006569676874206F662063616C6962726114
:1048B00074696F6E20706F696E7400B500506C651E
:1048C00061736520636C65616E20746865206E6F2E
:1048D0007A7A6C6520666F722063616C69627261BE
:1048E00074696F6E2E20436C69636B207768656E08
:1048F00020646F6E652E00B6004175746F20686F7E
:104900006D6500B700526573756D696E67207072D2
:10491000696E7400B80050494E4441204865617486
:10492000696E6700B90043616C6962726174696F96
:104930006E20646F6E6500BA0043616C69627261DB
:1049400074696E67205A00BB0042656420646F6E14
:104950006500BC004265642048656174696E67004B
:10496000BD0048656174696E6720646F6E652E00D6
:10497000BE0048656174696E6700BF00546F746162
:104980006C00C0004C617374207072696E7400C159
:10499000004D4D55206661696C7300C2004D4D5548
:1049A000206C6F6164206661696C7300C3004D4DBB
:1049B0005520706F776572206661696C7300C40062
:1049C0004D6174657269616C206368616E676573BF
:1049D00000C5004C617374207072696E742066614A
:1049E000696C7572657300C600546F74616C2066E3
:1049F00061696C7572657300C70046696C2E207220
:104A0000756E6F75747300C80054656D7065726162
:104A1000747572657300C90053656E736F72206997
:104A20006E666F00CA00457874727564657220699D
:104A30006E666F00CB0058595A2063616C2E20645B
:104A4000657461696C7300CC005072696E74657234
:104A500020495020416464723A00CD00756E6B6E3F
:104A60006F776E00CE004D4D5520636F6E6E65639F
:104A700074656400CF00446174653A00D000746FBF
:104A800020756E6C6F61642066696C616D656E7413
:104A900000D100746F206C6F61642066696C616D79
:104AA000656E7400D200507265737320746865205F
:104AB0006B6E6F6200D30050726568656174696ED9
:104AC0006720746F2063757400D400507265686548
:104AD0006174696E6720746F20656A65637400D5C0
:104AE0000050726568656174696E6720746F207527
:104AF0006E6C6F616400D6005072656865617469A0
:104B00006E6720746F206C6F616400D700436F6F15
:104B10006C646F776E00D80046696C616D656E7469
:104B200020657874727564696E67202620776974D1
:104B30006820636F727265637420636F6C6F723F7D
:104B400000D900456A65637400DA004175746F6CC2
:104B50006F6164696E672066696C616D656E742053
:104B60006973206163746976652C206A757374209B
:104B7000707265737320746865206B6E6F6220615C
:104B80006E6420696E736572742066696C616D6510
:104B90006E742E2E2E00DB00546F74616C206669DB
:104BA0006C616D656E7400DC00546F74616C207014
:104BB00072696E742074696D6500DD0046696C6110
:104BC0006D656E74207573656400DE005072696EE9
:104BD000742074696D6500DF0050726568656174EA
:104BE00020746865206E6F7A7A6C652100E000455C
:104BF00052524F523A00E100592064697374616E59
:104C000063652066726F6D206D696E00E2004C6511
:104C1000667400E300526967687400E4004D6561E2
:104C2000737572656420736B657700E500536C697A
:104C300067687420736B657700E60053657665726C
:104C40006520736B657700E7005B303B305D20705B
:104C50006F696E74206F666673657400E800416466
:104C60006A757374696E67205A00E9005265617253
:104C70002073696465205BE46D5D00EA0046726F35
:104C80006E7420736964655BE46D5D00EB005269CE
:104C900067687420736964655BE46D5D00EC004CCB
:104CA0006566742073696465205BE46D5D00ED00EA
:104CB0005365742074656D70657261747572653AC0
:104CC00000EE00417265206C65667420616E6420A0
:104CD0007269676874205A2D6361727269616765D1
:104CE0007320616C6C2075703F00EF0043616C694C
:104CF00062726174696E672058595A2E20526F741F
:104D000061746520746865206B6E6F6220746F201B
:104D10006D6F766520746865205A206361727269D0
:104D200061676520757020746F2074686520656EFA
:104D3000642073746F70706572732E20436C6963A6
:104D40006B207768656E20646F6E652E00F00043FF
:104D5000616C6962726174696E67205A2E20526FAD
:104D60007461746520746865206B6E6F6220746F67
:104D7000206D6F766520746865205A2063617272B9
:104D80006961676520757020746F2074686520659F
:104D90006E642073746F70706572732E20436C693B
:104DA000636B207768656E20646F6E652E00F1007E
:104DB00050494E44412063616C6962726174696F4D
:104DC0006E206661696C656400F20050494E444192
:104DD0002063616C6962726174696F6E206973200F
:104DE00066696E697368656420616E6420616374CE
:104DF0006976652E2049742063616E2062652064A7
:104E0000697361626C656420696E206D656E7520E2
:104E100053657474696E67732D3E50494E4441204A
:104E200063616C2E00F300457874727564657200DE
:104E3000F4004D6F7665205A00F5004D6F766520C1
:104E40005900F6004D6F7665205800F700536865ED
:104E5000657420252E37730A5A206F666673657451
:104E60003A20252B312E33666D6D0A2563436F6E14
:104E700074696E75650A2563526573657400F80080
:104E8000506C65617365206C6F61642066696C614C
:104E90006D656E742066697273742E00F9003E436E
:104EA000616E63656C00FA0052756E6E696E672004
:104EB00057697A6172642077696C6C2064656C65EF
:104EC00074652063757272656E742063616C6962CB
:104ED000726174696F6E20726573756C7473206192
:104EE0006E642073746172742066726F6D207468D2
:104EF0006520626567696E6E696E672E20436F6E0E
:104F000074696E75653F00FB005072656865617479
:104F1000696E67206E6F7A7A6C652E20506C6561C1
:104F2000736520776169742E00FC00506C656173B5
:104F30006520696E736572742066696C616D656E5B
:104F40007420696E746F207468652065787472755A
:104F50006465722C207468656E20707265737320AE
:104F6000746865206B6E6F6220746F206C6F616473
:104F70002069742E00FD00506C6561736520696EB8
:104F8000736572742066696C616D656E7420696EFC
:104F9000746F20746865206669727374207475621A
:104FA00065206F6620746865204D4D552C2074680F
:104FB000656E20707265737320746865206B6E6F08
:104FC0006220746F206C6F61642069742E00FE0093
:104FD000546865207072696E7465722077696C6CB4
:104FE000207374617274207072696E74696E6720C8
:104FF00061207A69672D7A6167206C696E652E2061
:10500000526F7461746520746865206B6E6F6220E6
:10501000756E74696C20796F7520726561636820A4
:10502000746865206F7074696D616C20686569676C
:1050300068742E20436865636B207468652070690E
:1050400063747572657320696E2074686520686189
:105050006E64626F6F6B202843616C696272617469
:10506000696F6E2063686170746572292E00FF009D
:1050700053656C6563742074656D706572617475D9
:105080007265207768696368206D61746368657311
:1050900020796F7572206D6174657269616C2E0084
:1050A000000153656C65637420612066696C616DF5
:1050B000656E7420666F722074686520466972732D
:1050C00074204C617965722043616C69627261740D
:1050D000696F6E20616E642073656C65637420690E
:1050E0007420696E20746865206F6E2D736372651D
:1050F000656E206D656E752E0001014E6F7720493B
:105100002077696C6C2063616C69627261746520E0
:1051100064697374616E6365206265747765656E3A
:1051200020746970206F6620746865206E6F7A7ACB
:105130006C6520616E6420686561746265642073CB
:105140007572666163652E0002015A2063616C69A5
:1051500062726174696F6E207265636F6D6D656EEA
:105160006465642E2052756E206974206E6F773FDF
:10517000000301506C656173652072656D6F766523
:1051800020737465656C2073686565742066726F42
:105190006D20686561746265642E000401497320A6
:1051A000737465656C207368656574206F6E206824
:1051B0006561746265643F000501506C65617365EB
:1051C00020636865636B206F75722068616E64622E
:1051D0006F6F6B20616E642066697820746865204B
:1051E00070726F626C656D2E205468656E207265FA
:1051F00073756D65207468652057697A61726420E3
:105200006279207265626F6F74696E672074686579
:10521000207072696E7465722E000601416C6C20FC
:10522000697320646F6E652E2048617070792070FC
:1052300072696E74696E6721000701596F7520638A
:10524000616E20616C7761797320726573756D652D
:10525000207468652057697A6172642066726F6D88
:105260002043616C6962726174696F6E202D3E200B
:1052700057697A6172642E000801496620796F755A
:105280002068617665206164646974696F6E616C21
:1052900020737465656C207368656574732C206376
:1052A000616C6962726174652074686569722070EE
:1052B00072657365747320696E2053657474696ECA
:1052C0006773202D204857205365747570202D205A
:1052D000537465656C207368656574732E000901ED
:1052E000506C6561736520636C65616E20686561F3
:1052F0007462656420616E64207468656E207072EB
:1053000065737320746865206B6E6F622E000A01EE
:10531000446F20796F752077616E7420746F2072EE
:105320006570656174206C6173742073746570209E
:10533000746F20726561646A757374206469737434
:10534000616E6365206265747765656E206E6F7A45
:105350007A6C6520616E6420686561746265643F83
:10536000000B0153656C656374206E6F7A7A6C650F
:1053700020707265686561742074656D7065726116
:1053800074757265207768696368206D61746368FD
:10539000657320796F7572206D6174657269616CD7
:1053A0002E000C0149732066696C616D656E742076
:1053B0006C6F616465643F000D014E6F772049207A
:1053C00077696C6C2070726568656174206E6F7AA5
:1053D0007A6C6520666F7220504C412E000E014998
:1053E0002077696C6C2072756E207A2063616C691D
:1053F00062726174696F6E206E6F772E000F014EBE
:105400006F772072656D6F766520746865207465AE
:105410007374207072696E742066726F6D2073747D
:1054200065656C2073686565742E001001506C65AD
:105430006173652072656D6F766520736869707041
:10544000696E672068656C70657273206669727337
:10545000742E001101492077696C6C2072756E20E2
:1054600078797A2063616C6962726174696F6E2009
:105470006E6F772E2049742077696C6C2074616B95
:105480006520757020746F203234206D696E732E24
:1054900000120146697273742C20492077696C6C84
:1054A0002072756E207468652073656C6674657310
:1054B0007420746F20636865636B206D6F73742054
:1054C000636F6D6D6F6E20617373656D626C7920B3
:1054D00070726F626C656D732E00130148692C2029
:1054E0004920616D20796F7572204F726967696E0E
:1054F000616C205072757361206933207072696E1F
:105500007465722E20576F756C6420796F75206CEE
:10551000696B65206D6520746F206775696465200F
:10552000796F75207468726F75676820746865207C
:1055300073657475702070726F636573733F0014C8
:105540000148692C204920616D20796F7572204FC8
:10555000726967696E616C2050727573612069337E
:10556000207072696E7465722E20492077696C6CA8
:1055700020677569646520796F75207468726F752E
:10558000676820612073686F72742073657475702A
:105590002070726F636573732C20696E2077686961
:1055A000636820746865205A2D6178697320776973
:1055B0006C6C2062652063616C6962726174656401
:1055C0002E205468656E2C20796F752077696C6C7D
:1055D00020626520726561647920746F2070726941
:1055E0006E742E00150150617573650016014653E7
:1055F00020416374696F6E001701436F6E742E0053
:105600001801462E206175746F6C6F61640019017A
:10561000462E2072756E6F7574001A01437574748E
:105620006572001B0146616E207370656564001C25
:1056300001426564001D0146616E73206368656305
:105640006B001E014D6F64656C001F014E6F7A7A0E
:105650006C6500200146656564696E6720746F2083
:105660004653656E736F720021014D6F76696E67E8
:105670002073656C6563746F72002201486F6D69F9
:105680006E67002301526574726163742066726FE5
:105690006D2046494E4441002401456A65637469A2
:1056A0006E672066696C616D656E740025015061DE
:1056B000726B696E672073656C6563746F72002628
:1056C0000152657475726E696E672073656C6563EF
:1056D000746F72002701506572666F726D696E6734
:1056E0002063757400280150757368696E672066C1
:1056F000696C616D656E740029015072657061722C
:10570000696E6720626C616465002A0153656C658F
:105710006374696E672066696C2E20736C6F740009
:105720002B01556E6C6F6164696E672066696C61F0
:105730006D656E74002C0145525220544D43206615
:1057400061696C6564002D014552522048656C709A
:105750002066696C616D656E74002E0145525220A1
:10576000496E7465726E616C002F0145525220576C
:1057700061697420666F722055736572003001464E
:10578000696E697368696E67206D6F76656D656EA9
:10579000747300310141766F6964696E67206772C6
:1057A000696E6400320146656564696E6720746FD6
:1057B000206E6F7A7A6C6500330146656564696EA8
:1057C0006720746F206578747275646572003401A7
:1057D00046656564696E6720746F2046494E444192
:1057E000003501556E6C6F6164696E6720746F20BF
:1057F00070756C6C6579003601556E6C6F6164690B
:105800006E6720746F2046494E4441003701446959
:1058100073656E676167696E672069646C657200A5
:105820003801456E676167696E672069646C6572EF
:105830000039014F4B003A01554E4B4E4F574E2009
:105840004552524F52003B0146494C414D454E5442
:10585000204348414E4745003C0146494C414D4597
:105860004E5420454A4543544544003D01554E4C55
:105870004F4144204D414E55414C4C59003E01464C
:10588000572052554E54494D45204552524F5200D3
:105890003F014D4D55204657205550444154452019
:1058A0004E45454445440040015155455545204627
:1058B000554C4C004101494E56414C494420544FEF
:1058C0004F4C00420146494C2E20414C5245414428
:1058D00059204C4F41444544004301434F4D4D55E1
:1058E0004E49434154494F4E204552524F52004475
:1058F000014D4D55204E4F5420524553504F4E446C
:10590000494E470045014D4D55204D4355204552C8
:10591000524F520046014D4D552053454C4654457B
:105920005354204641494C4544004701544D4320BF
:105930004452495645522053484F5254454400481A
:1059400001544D4320554E444552564F4C54414707
:105950004520455252004901544D43204452495676
:105960004552205245534554004A01544D4320446A
:105970005249564552204552524F52004B01544D08
:1059800043204F56455248454154204552524F52AC
:10599000004C015741524E494E4720544D4320542C
:1059A0004F4F20484F54004D0149444C455220432D
:1059B000414E4E4F54204D4F5645004E0149444CE8
:1059C00045522043414E4E4F5420484F4D45004FC5
:1059D0000153454C4543544F522043414E4E4F5482
:1059E000204D4F564500500153454C4543544F52AE
:1059F0002043414E4E4F5420484F4D450051014CDD
:105A00004F414420544F20455854522E204641497E
:105A10004C4544005201494E535045435420464999
:105A20004E44410053014653454E534F5220544F6C
:105A30004F204541524C5900540150554C4C45594A
:105A40002043414E4E4F54204D4F56450055014680
:105A500053454E534F522046494C2E2053545543E4
:105A60004B0056014653454E534F52204449444E35
:105A7000542054524947472E00570146494E44414D
:105A80002046494C414D2E20535455434B0058015C
:105A900046494E4441204449444E542054524947BB
:105AA0004745520059014375742066696C616D6504
:105AB0006E74005A01456A6563742066726F6D20CA
:105AC0004D4D55005B014C6F6164696E67206669DE
:105AD0006C616D656E74005C014D4D5520526574AE
:105AE00072793A20526573746F72696E67207465BB
:105AF0006D70657261747572652E2E2E005D015396
:105B00006F7274696E672066696C6573005E01531D
:105B10006F6D652066696C65732077696C6C206EAB
:105B20006F7420626520736F727465642E204D61FE
:105B3000782E204E6F2E206F662066696C6573206C
:105B4000696E203120666F6C64657220666F72200A
:105B5000736F7274696E67206973203130302E0064
:105B60005F0153544F505045442E0060014F66660C
:105B70000061014F6E006201556E65787065637457
:105B80006564206572726F72206F636375727265EF
:105B9000642E0063014D3630302046696C616D65BE
:105BA0006E74204368616E67652E204C6F616420BF
:105BB00061206E65772066696C616D656E74206F1B
:105BC0007220656A65637420746865206F6C642058
:105BD0006F6E652E00640152656D6F766520746886
:105BE0006520656A65637465642066696C616D65CE
:105BF0006E742066726F6D207468652066726F6EB9
:105C000074206F6620746865204D4D552E00650127
:105C100046696C616D656E74206465746563746556
:105C20006420756E65787065637465646C792E2088
:105C3000456E73757265206E6F2066696C616D6567
:105C40006E74206973206C6F616465642E204368F4
:105C500065636B207468652073656E736F72732063
:105C6000616E6420776972696E672E006601496E05
:105C70007465726E616C2072756E74696D652065F5
:105C800072726F722E20547279207265736574740B
:105C9000696E6720746865204D4D55206F722075C0
:105CA00070646174696E6720746865206669726DDE
:105CB000776172652E0067014D4D5520465720765D
:105CC000657273696F6E20697320696E636F6D70A2
:105CD000617469626C652077697468207072696E9E
:105CE0007465722046572E55706461746520746F18
:105CF0002076657273696F6E20332E302E332E003E
:105D000068014D4D55204669726D77617265206955
:105D10006E7465726E616C206572726F722C207089
:105D20006C656173652072657365742074686520A5
:105D30004D4D552E0069015265717565737465642A
:105D40002066696C616D656E7420746F6F6C20697C
:105D500073206E6F7420617661696C61626C65207E
:105D60006F6E207468697320686172647761726510
:105D70002E20436865636B2074686520472D636F30
:105D8000646520666F7220746F6F6C20696E646545
:105D900078206F7574206F662072616E67652028A9
:105DA00054302D5434292E006A0143616E6E6F7495
:105DB00020706572666F726D20746865206163740F
:105DC000696F6E2C2066696C616D656E74206973F5
:105DD00020616C7265616479206C6F616465642E0A
:105DE00020556E6C6F6164206974206669727374EB
:105DF0002E006B014D4D55206E6F742072657370CF
:105E00006F6E64696E6720636F72726563746C791C
:105E10002E20436865636B2074686520776972691A
:105E20006E6720616E6420636F6E6E6563746F725F
:105E3000732E006C014D4D55206E6F74207265738A
:105E4000706F6E64696E672E20436865636B2074A3
:105E5000686520776972696E6720616E6420636F80
:105E60006E6E6563746F72732E006D014D6F726597
:105E70002064657461696C73206F6E6C696E652E49
:105E8000006E015468652049646C65722063616E20
:105E90006E6F7420686F6D652070726F7065726CC4
:105EA000792E20436865636B20666F7220616E797E
:105EB0007468696E6720626C6F636B696E672069D6
:105EC0007473206D6F76656D656E742E006F01437F
:105ED000616E2774206D6F76652053656C65637401
:105EE0006F72206F722049646C65722E00700154CD
:105EF00068652053656C6563746F722063616E6EB4
:105F00006F7420686F6D652070726F7065726C7948
:105F10002E20436865636B20666F7220616E797412
:105F200068696E6720626C6F636B696E6720697465
:105F300073206D6F76656D656E742E0071014C6F08
:105F40006164696E6720746F20657874727564652A
:105F500072206661696C65642E20496E737065639A
:105F600074207468652066696C616D656E74207458
:105F700069702073686170652E20526566696E6570
:105F8000207468652073656E736F722063616C693D
:105F900062726174696F6E2C206966206E6565643B
:105FA00065642E00720153656C6563746F722063C3
:105FB000616E2774206D6F76652064756520746F3F
:105FC0002046494E444120646574656374696E6778
:105FD00020612066696C616D656E742E204D616B69
:105FE000652073757265206E6F2066696C616D65E2
:105FF0006E7420697320696E2053656C6563746FDD
:106000007220616E642046494E444120776F726B66
:10601000732070726F7065726C792E00730146691F
:106020006C616D656E742073656E736F722074722F
:106030006967676572656420746F6F206561726C53
:1060400079207768696C65206C6F6164696E672080
:10605000746F2065787472756465722E204368656C
:10606000636B2074686572652069736E27742061A4
:106070006E797468696E6720737475636B20696EDE
:10608000205054464520747562652E204368656330
:106090006B20746861742073656E736F7220726513
:1060A0006164732070726F7065726C792E00740178
:1060B00050756C6C6579206D6F746F7220737461AC
:1060C0006C6C65642E20456E73757265207468650E
:1060D0002070756C6C65792063616E206D6F7665DC
:1060E00020616E6420636865636B20746865207747
:1060F0006972696E672E00750146696C616D656E27
:10610000742073656E736F72206469646E277420E7
:10611000737769746368206F6666207768696C6559
:1061200020756E6C6F6164696E672066696C616D65
:10613000656E742E20456E737572652066696C619C
:106140006D656E742063616E206D6F766520616E83
:1061500064207468652073656E736F7220776F7248
:106160006B732E00760146696C616D656E742073E9
:10617000656E736F72206469646E2774207472692F
:1061800067676572207768696C65206C6F61646908
:106190006E67207468652066696C616D656E742E2B
:1061A00020456E73757265207468652073656E7323
:1061B0006F722069732063616C69627261746564D7
:1061C00020616E64207468652066696C616D656E1F
:1061D0007420726561636865642069742E007701BC
:1061E00046494E4441206469646E27742073776980
:1061F000746368206F6666207768696C6520756EC9
:106200006C6F6164696E672066696C616D656E7440
:106210002E2054727920756E6C6F6164696E6720F0
:106220006D616E75616C6C792E20456E737572654B
:106230002066696C616D656E742063616E206D6FA0
:10624000766520616E642046494E444120776F7226
:106250006B732E00780146494E4441206469646E98
:1062600027742074726967676572207768696C6546
:10627000206C6F6164696E67207468652066696C64
:10628000616D656E742E20456E737572652074683D
:10629000652066696C616D656E742063616E206D4A
:1062A0006F766520616E642046494E444120776FC9
:1062B000726B732E00790144697361626C65007AB8
:1062C0000153746F70007B014C6F6164007C015559
:1062D0006E6C6F6164007D0152657365744D4D5540
:1062E000007E015265747279007F01426564206C02
:1062F0006576656C696E67206661696C65642E20E1
:1063000053656E736F72206469646E2774207472B3
:1063100069676765722E20446562726973206F6ECB
:10632000206E6F7A7A6C653F2057616974696E6779
:1063300020666F722072657365742E00800153654C
:106340006E7369746976697479008101446F6E6552
:1063500000656E717565696E67202200446F6E6519
:10636000207072696E74696E672066696C65004E94
:106370006F204C696E65204E756D6265722077697D
:10638000746820636865636B73756D2C204C617352
:1063900074204C696E653A20004E6F204368656337
:1063A0006B73756D2077697468206C696E65206EFB
:1063B000756D6265722C204C617374204C696E653A
:1063C0003A2000636865636B73756D206D69736D4A
:1063D000617463682C204C617374204C696E653A5B
:1063E00020004C696E65204E756D62657220697380
:1063F000206E6F74204C617374204C696E65204E62
:10640000756D6265722B312C204C617374204C6960
:106410006E653A2000257520627974657320777265
:10642000697474656E20746F202553206174206137
:10643000646472657373203078253038780A0044BC
:106440002564202D20526561642F57726974652080
:1064500025530A003F3F00526F6D616E6100487224
:10646000766174736B69004D616779617200536C7A
:106470006F76656E63696E61004E6F72736B005369
:1064800076656E736B61004E656465726C616E64F7
:106490007300506F6C736B69004974616C69616E55
:1064A0006F004672616E6361697300457370616E5F
:1064B0006F6C004465757473636800436573746939
:1064C0006E6100456E676C6973680020436F756E7E
:1064D0007420583A200045303A25642052504D200F
:1064E00050524E313A25642052504D204530403AAA
:1064F00025752050524E31403A25750A0052657379
:10650000656E640025533A20256C640A25530A0001
:106510002F2F616374696F6E3A6E6F746966696379
:106520006174696F6E2025530A0046696C616D6560
:106530006E742072756E6F75742064657465637413
:106540006564210064697361626C656400656E61F5
:10655000626C656400454550524F4D005352414DA9
:1065600000442D31202D20456E646C657373206CC2
:106570006F6F700A004163746976652045787472A4
:10658000756465723A203000496E76616C696420EA
:106590006578747275646572004D3232302053250F
:1065A00064005344207072696E74696E672062796A
:1065B00074652000257500556E6B6E6F776E2063D5
:1065C0006F6D6D616E643A2022004D32303020498B
:1065D0006E76616C6964206578747275646572208A
:1065E000007A5F6D61783A20007A5F6D696E3A20BB
:1065F00000795F6D696E3A20005452494747455211
:106600004544006F70656E00785F6D696E3A2000DA
:106610005265706F7274696E6720656E6473746F13
:106620007020737461747573004D31313220636171
:106630006C6C65642E20456D657267656E637920AC
:1066400053746F702E002F2F616374696F6E3A75EB
:10665000766C6F5F7265636F766572795F72656184
:1066600064790053494C454E54004E4F524D414CB5
:10667000002553204D4F44453A2050657263656EA6
:106680007420646F6E653A20256868643B207072E0
:10669000696E742074696D652072656D61696E69DB
:1066A0006E6720696E206D696E733A2025643B2009
:1066B0004368616E676520696E206D696E733A206C
:1066C00025640A005072696E746572537461746552
:1066D0003A2025640A00456E642066696C65206C6A
:1066E00069737400426567696E2066696C65206C29
:1066F00069737400556E6B6E6F776E20256320632F
:106700006F64653A2025730A000A50494E444120BF
:1067100074656D70657261747572653A20252E31ED
:1067200066205A20736869667420286D6D293A20A6
:10673000252E3366000A537465703A2025642F367F
:106740000A000A537465703A2025642F3620287396
:106750006B6970706564290A50494E444120746524
:106760006D70657261747572653A202564205A20D7
:10677000736869667420286D6D293A300A000A5AD8
:1067800045524F3A20252E33660A007374617274A5
:106790002074656D70657261747572653A20252E7E
:1067A00031660A0025642020252E326600255320FC
:1067B000583A20252E356620593A20252E35662058
:1067C0005A3A20252E35660A00536C6565702E2EC8
:1067D0002E0045303A25642052504D0A50524E301A
:1067E0003A25642052504D0A004D31303700537520
:1067F00070657250494E44410048426564206F6E96
:10680000206C6F616400466C617368416972004579
:1068100072723A484F54454E442046414E204552EC
:10682000524F52002F2F616374696F6E3A72657315
:10683000756D6564002F2F616374696F6E3A7265C0
:1068400073756D65002F2F616374696F6E3A7265A1
:10685000616479002F2F616374696F6E3A6E6F7493
:106860005F7265616479002F2F616374696F6E3A9E
:1068700063616E63656C004F4B004C43442073743E
:1068800061747573206368616E67656400534420AA
:10689000636172642072656C6561736564002F2F9B
:1068A000616374696F6E3A7374617274004D383449
:1068B000004D373032004732382057004D353030E8
:1068C0000042616420696E7465727275707400575D
:1068D00061746368646F672074696D656F757400B7
:1068E000537461746963206D656D6F72792068619E
:1068F000730A6265656E206F76657277726974746B
:10690000656E004649524D5741524520435241530E
:1069100048210A437261736820726561736F6E3A31
:106920000A002020506C616E6E6572427566666565
:106930007242797465733A20002046726565204D75
:10694000656D6F72793A2000207C20417574686F04
:10695000723A2000204C6173742055706461746534
:10696000643A200020536F66747761726520526527
:1069700073657400205761746368646F67205265A3
:10698000736574002042726F776E206F75742052A9
:1069900065736574002045787465726E616C205271
:1069A0006573657400506F7765725570006572721B
:1069B0006F722077726974696E6720746F206669E0
:1069C0006C6500446F6E6520736176696E67206642
:1069D000696C652E006F6B0046696C616D656E7445
:1069E000004D6561737572656420736B6577733AEA
:1069F0002025662025660A0046697474696E672042
:106A00006661696C6564203D3E2063616C696272F9
:106A10006174696F6E206661696C65642E0A00435B
:106A2000616C6962726174696F6E2073756363650E
:106A300073732E0A00416C6C20342063616C6962B0
:106A4000726174696F6E20706F696E747320666F07
:106A5000756E642E0A00312F3400312F3400312F2F
:106A600039004572723A5052494E542046414E20E8
:106A70004552524F520025632533642F256481000F
:106A80005A25362E32662563005A2020202D2D2DC2
:106A90002000862533642525002D2D2D2525002554
:106AA0003364252500205344002020200020484F37
:106AB000002046524D2000872D2D3A2D2D202000FC
:106AC0008725337568202563256300872530327557
:106AD0003A2530327525632563002F2F6163746971
:106AE0006F6E3A706175736564002F2F616374690E
:106AF0006F6E3A70617573650044756D7020746FC8
:106B00002073657269616C0068656C702E707275B7
:106B1000736133642E636F6D00666F72756D2E70D6
:106B20007275736133642E636F6D0070727573617B
:106B300033642E636F6D004D3730310025533A0AB0
:106B40002531382E32666D200A25533A0A25313018
:106B50006C646420253032646820253032646D0016
:106B600025533A0A2531382E32666D200A25533ACC
:106B70000A2531306C646820253032646D20253060
:106B80003264730025362E32666D6D0025530A255A
:106B9000530A25533A0A25533A0025332E3266818B
:106BA00000252D31342E3134533A0A25530A252D30
:106BB00031342E3134533A25332E3266810A252D55
:106BC00031342E3134533A25332E32668100202061
:106BD00030002020310046494E44410050494E4487
:106BE000410057697A61726420656E642073746134
:106BF00074653A2025640A0053706F6F6C4A6F69A0
:106C00006E004669726D77617265005072757361CE
:106C1000206933204D4B322E3553204F4B2E004DE3
:106C20003630300053442063617264206F6B006F14
:106C300070656E526F6F74206661696C6564007672
:106C40006F6C756D652E696E6974206661696C651F
:106C50006400534420696E6974206661696C006F3A
:106C600070656E206661696C65642C2046696C6590
:106C70003A200043616E6E6F7420656E74657220F9
:106C80007375626469723A20004D3234004D3233BC
:106C9000202573005072696E7465722073746F7072
:106CA0007065642064756520746F206572726F7200
:106CB000732E205375706572766973696F6E2072DA
:106CC000657175697265642E0047312045252D2E4A
:106CD0003366204632373030004D383300312F399B
:106CE00000880020746F6F206C6F6E672065787469
:106CF000727573696F6E2070726576656E74656407
:106D00000020636F6C6420657874727573696F6EB0
:106D10002070726576656E746564004D6F766520CF
:106D200061626F7274656400084AD73B3BCE016EA6
:106D300084BCBFFDC12F3D6C74319ABD56833DDAD2
:106D40003D00C77F11BED9E4BB4C3E916BAAAABEE1
:106D5000000000803F05A84CCDB2D44EB93836A90A
:106D6000020C50B9918688083CA6AAAA2ABE000047
:106D700000803F07634236B79BD8A71A3968561878
:106D8000AEBAAB558C1D3CB7CC5763BD6DEDFD75F0
:106D90003EF6177231BF000000803F08000000BEC1
:106DA000922449123EABAAAA2ABECDCCCC4C3E00BE
:106DB000000080BEABAAAAAA3E00000000BF0000EF
:106DC00000803F0000000000084178D3BB4387D11A
:106DD000133D190E3CC3BD4282AD2B3E68EC82765A
:106DE000BED98FE1A93E4C80EFFFBE01C4FF7F3FBB
:106DF0000000000000000C942BFE0C949CF60D94F7
:106E0000DE640D94B10E0C94ECB00D940F2F0C9425
:106E1000366E0D943E070D94E02E0C947DE90C9493
:106E200002EA0C9419B50C940FB30D94B6000D94AE
:106E3000CA300D94C1640D94F22E0C94B4FE0D94DE
:106E400066010C9456E60C9463BC0C9482BC0D94C1
:106E5000B4100D94FB030C941BB30C946DFF0C94B5
:106E60008EBB0D94A6010C9405B50D946B2E0C945D
:106E70000CC10D94CC390C9467FC0C9495B10D9415
:106E800041310C9447FC0C94E8B00D94040C0D9423
:106E900011310C94EFFB0D9431310C94E0700C9493
:106EA000B0B30D946F390C94AEE20D94DC040C94E5
:106EB000ACB80D9498300D947F640C947BFC0C94CA
:106EC00085FC0D9439310C9417C60C94E25E0C9439
:106ED000D2BA0D94E8060C9477EA0C945CB40C9446
:106EE000E9FD0C9433FC0C94FAFD0D94C4300D9420
:106EF000520F0C9497FD0D9451310D9410110C9478
:106F000014B50C9424EF0D9420010D94C92E0C940B
:106F1000FDEA0C94BBC00D9449310C940AB50C9455
:106F2000FAB00C948FB10C94C8BB0C942AB30C9497
:106F3000FDC30C94ADFC0D94800D0C949FEA0D9450
:106F400071060C943DFC0D94F56A0C94A2E20C942D
:106F50003EC10C94A3F70C941EB50D9461020D94E0
:106F600021310D94EF080C947FFD0C947EFE0D945E
:106F7000E36A0C94ACC00C9423B50C94B3F60D9456
:106F800097040D944A1D0C94A2FD0C945BBC0C94C8
:106F900081EA0C9477BC0D943D0A0D9492040D94F3
:106FA000C7300D94E06A0C94CFC00C94E0FD0D94B2
:106FB000C7100C94C6E70D94FE300C94F6E20D94C5
:106FC000AF2E0C94E7E20D945E2F0C94C3B00C949A
:106FD000F9E20C94D4BB0D945B300D9419310C94F0
:106FE00050B70C9439C60C94DAB00C94C6B00C941B
:106FF00016C10C94C6E20C94126E0C943F6E0C9465
:10700000206E0D9446120C94FCE20C949EF60C94A7
:10701000746E0C94B1C00C9408E30D9466640C94E7
:10702000196C0C948BFD0C9424FE0C9453BC0D94A1
:107030006A1C0C9493BC0D944D960C94F2B00C9475
:1070400040FE0C94F3C00D9429310C94C56F0C9440
:1070500042BA0C94CCE70C94CEBB0C9472B60D944F
:1070600083060D94B9020D94FB300C9471FC0C94C2
:1070700010EF0C9412E90D94F06A0C9432FE0C940B
:10708000B7B00D94F8300C9451FC0C9485EA0C9434
:107090009CFC0C94F9FF0D9459310C9441B30D9460
:1070A000C10C0C94CBBB0C9467B50D941B300C94A5
:1070B000D1BB0C94076E0C94CAB50C94BBB00C9465
:1070C000BBF70D943F2E0C9489EA0C942AC10D94C1
:1070D00043110D94E76A0D9458300D94C46A0C94D2
:1070E000F6B00C94C5C00D945F2E0C94FDC00D94A9
:1070F00054110C940FB50D9433300D948A040D94F3
:1071000046940C9439FE0C9496BC0C94D6B00C9416
:10711000C4FD0C94DFC00C945DB00C94DDBB0C94EA
:107120007DEA0D94FB2E0D9401310D9462300D9487
:10713000FA010D94E42E0D947A060C946BBC0C9419
:107140005BFC0C94ADEF0C94D0B00C9491BC0C94FF
:1071500036B30D9465300C94C8BA0C9479E90C944C
:1071600020C10C94C5BB0C94D7C00C94F3E20C94D2
:1071700092B60D947E6A0C94E3B50C94A4C00D9461
:10718000E5640C9451B50C94CCB00D94752E0D940F
:10719000DA2E0D94E1640D9409310C94FEEB0C94FD
:1071A000DEB00C94BFB00D9470110C94ED6D0C9486
:1071B000F1B00C943DF70C94E7FD0C94B1B00C9435
:1071C000E4B00C94626E0C9400B50D943B070D94E2
:1071D000DC210C947AB40C9434C10C94FEB00C9461
:1071E000E9C00C94DBFC0D94B53F0C94FDBA6E61C4
:1071F0006E00696E660000407A10F35A00A0724E6D
:1072000018090010A5D4E80000E87648170000E44B
:107210000B54020000CA9A3B000000E1F505000093
:1072200080969800000040420F000000A0860100F8
:107230000000102700000000E803000000006400C8
:10724000000000000A000000000001000000000033
:107250002C76D888DC674F0823DFC1DFAE59E1B157
:10726000B796E5E3E453C63AE651997696E8E6C266
:107270008426EB898C9B62ED407C6FFCEFBC9C9F6D
:1072800040F2BAA56FA5F490055A2AF75C936B6C8F
:10729000F9676DC11BFCE0E40D47FEF520E6B50083
:1072A000D0ED902E0300943577050080841E0800F1
:1072B00000204E0A000000C80C333333330F986EA1
:1072C00012831141EF8D2114893BE65516CFFEE65E
:1072D000DB18D1844B381BF77C1D901DA4BBE42424
:1072E000203284725E228100C9F124ECA1E53D27A1
:1072F0002200002045535000204E535000204F469E
:107300004600204F4E005056303100205B4D505DFE
:107310002000256920686F757273202569206D69CA
:107320006E757465730052582074696D656F75745D
:10733000004D333130004D313132004D31313000AC
:1073400046756C6C20525820427566666572005313
:10735000657474696E67732053746F72656400534B
:10736000746F7265642073657474696E67732072DC
:1073700065747269657665640048617264636F6400
:1073800065642044656661756C7420536574746926
:107390006E6773204C6F61646564005632000000B4
:1073A00000C8420000C8420000C843000005430076
:1073B00000484300004843000040410000F042E81C
:1073C000030000E8030000C800000088130000006C
:1073D000409C4400409C440000000000000000204D
:1073E0004E00000000204100002041CDCCCC3E00EA
:1073F000009040000000000000000000000000CDF0
:10740000CCCC3E3D0A8141FF08433EB099AB438F4F
:1074100042FC42E65A343F4C62B045000000000096
:107420004040000034420000000000000000000066
:107430000041000000E03F00002C4300002C43000E
:107440000040410000F042C0030000C0030000C83B
:10745000000000881300001010101000409C440031
:1074600000803F0000003F19140000002030780029
:10747000203078006572726F723A200044323320F7
:107480002D20656D657267656E637920736572691D
:10749000616C2064756D7000437573746F6D004E80
:1074A000796C6F6E504100536174696E20200054F6
:1074B000657874757200536D6F6F746800312E308B
:1074C00000312E3500554E4B4E4F574E004C41313A
:1074D00030433A204C696E65617220416476616E7A
:1074E0006365206D6F64653A20004C413130433A4A
:1074F0002041646A757374656420452D4A65726B1A
:107500003A2000CE80CEDE3E0FA8AF00480069963C
:107510000000DF6025555887680427F2E0005E34DC
:1075200003CC1960F33C0EF88F00DB080294920044
:107530003E1C079A8700E524008528527E06001B22
:10754000E4007E781270787061F812788F88417844
:107550004270787061782570787061F850788F8803
:10756000D1F02527078761F025278F88412C0D272B
:10757000AA50D1BC0707871161BE788F8811417866
:107580005270787061F852788F8841201278887034
:1075900063205278887063485278888743031117B4
:1075A000997064181278F870654412F8F8F045186C
:1075B0004278F87065182578F87065185278F87078
:1075C00065185078F870650C078F872365A20F8FB8
:1075D0008F11450012062270690012072227490008
:1075E0002506227069002507222749001206222756
:1075F0006C026236A2706C40456C44704C0362228F
:1076000022706C43888888F04C7812BC88806E7831
:1076100052BC88806E38127888706F7812788887AC
:107620004F38427888706F38257888706F3A0079C3
:10763000AC786F3D079AAC786F7850788887EF39CF
:10764000497888706F0852BC8880729852F88F9879
:107650005220127870F07348127863875320527862
:1076600070F0734852786387531007870F247312A2
:10767000786387245360699A988BE22304E444304A
:1076800074104E444324747C12888960753C508881
:107690008870557825288960757949088960753C16
:1076A00012887070790C12885222594412F124F019
:1076B0007A4452F124F07A8C52F0368F5A4420F1F9
:1076C00024F07A00401454CDCCCC3D0AD7233C178B
:1076D000B7D13877CC2B329595E6241FB14F0A00ED
:1076E0000020410000C84200401C4620BCBE4CCADD
:1076F0001B0E5AAEC59D744E414E494E4600007A4F
:10770000430000524300005243000000000000808C
:10771000C09A99193E00000000000080C09A991993
:107720003E20503A002042403A0020403A00202FAC
:10773000002054303A00202F0020423A00202F0031
:10774000543A002553457863657373697665206202
:107750006564206C6576656C696E6720636F727214
:10776000656374696F6E3A202569206D6963726F75
:107770006E730A00426564206C6576656C696E679D
:10778000206661696C65642E20546F6F206D75638F
:107790006820766172696174696F6E2066726F6DC0
:1077A00020656570726F6D206D6573680042656459
:1077B000206C6576656C696E67206661696C6564CE
:1077C0002E2053656E736F722074726967676572DD
:1077D000656420746F6F20736F6F6E002020004D02
:1077E0006561737572656420706F696E74733A00B9
:1077F0005A20736561726368206865696768743AC6
:1078000020352E3066004E756D20582C593A2037A1
:107810002C37004D65736820626564206C65766561
:107820006C696E67206E6F74206163746976652E73
:107830000020453A00205A3A0020593A0020453AA3
:1078400000205A3A0020593A00583A00202D3E2094
:107850000053706F6F6C4A6F696E3A20002C2000E5
:10786000496E6163746976697479205368757464CC
:107870006F776E004B494C4C45442E005072696E38
:107880007465722068616C7465642E206B696C6C21
:1078900028292063616C6C656421005A206C69762C
:1078A000652061646A757374206F7574206F66203B
:1078B00072616E67652E2053657474696E672074FB
:1078C0006F20302E20436C69636B20746F20636FD0
:1078D0006E74696E75652E005A206C69766520613C
:1078E000646A757374206F7574206F662072616EA0
:1078F00067652E2053657474696E6720746F20303D
:107900000020453A3020423A00543A0062757379BB
:107910003A2070617573656420666F7220696E70BD
:10792000757400627573793A2070617573656420AF
:10793000666F72207573657200627573793A207094
:10794000726F63657373696E670073657269616CEA
:107950002064756D702000496E76616C69642054F6
:1079600020636F64652E004475706C696361746593
:1079700020542D636F64652069676E6F7265642E95
:1079800000416476616E6365204B3D004B206F754E
:1079900074206F6620616C6C6F7765642072616E15
:1079A000676521004D4B322E3553004D4B322E353D
:1079B000534D4D553253001C4FFC002533642F2589
:1079C00033640025336400200A200A200A200025A1
:1079D000534172632053657474696E67733A205023
:1079E0003A4D6178206C656E677468286D6D29204A
:1079F000533A4D696E206C656E67746820286D6D12
:107A000029204E3A436F7272656374696F6E7320FA
:107A1000523A4D696E207365676D656E74732046CA
:107A20003A5365676D656E74732F7365632E0A250F
:107A30005320204D3231342050252E3266205325DC
:107A40002E3266204E256420522564204625640A85
:107A500000255346696C616D656E7420736574749E
:107A6000696E67733A2044697361626C65640A00E9
:107A7000255346696C616D656E7420736574746915
:107A80006E67733A0A25532020204D32303020444F
:107A9000252E32660A002553526574726163743A6A
:107AA00020533D4C656E67746820286D6D29204613
:107AB0003A537065656420286D6D2F6D29205A3A00
:107AC000205A4C69667420286D6D290A25532020A0
:107AD000204D3230372053252E32662046252E3257
:107AE00066205A252E32660A25535265636F7665E5
:107AF000723A20533D4578747261206C656E6774EC
:107B00006820286D6D2920463A53706565642028E9
:107B10006D6D2F6D290A25532020204D32303820DD
:107B200053252E32662046252E32660A255341758E
:107B3000746F2D526574726163743A20533D302026
:107B4000746F2064697361626C652C203120746FDE
:107B500020696E74657270726574206578747275D0
:107B600064652D6F6E6C79206D6F7665732061731F
:107B7000207265747261637473206F722072656322
:107B80006F7665726965730A25532020204D323067
:107B900039205325640A0025535049442068656103
:107BA000746265642073657474696E67733A0A253C
:107BB000532020204D3330342050252E326620496A
:107BC000252E32662044252E32660A002553504960
:107BD000442073657474696E67733A0A25532020D4
:107BE000204D3330312050252E32662049252E324B
:107BF000662044252E32660A00255353746570733F
:107C00002070657220756E69743A0A255320204DE4
:107C100039322058252E32662059252E3266205AB8
:107C2000252E32662045252E32660A25534D617871
:107C3000696D756D20666565647261746573202871
:107C40006D6D2F73293A0A255320204D3230332091
:107C500058252E32662059252E3266205A252E327E
:107C6000662045252E32660A25534D6178696D756B
:107C70006D20616363656C65726174696F6E202845
:107C80006D6D2F7332293A0A255320204D32303141
:107C90002058256C752059256C75205A256C752047
:107CA00045256C750A2553416363656C6572617483
:107CB000696F6E3A20503D7072696E742C20523D8F
:107CC000726574726163742C20543D7472617665C0
:107CD0006C0A255320204D3230342050252E326638
:107CE0002052252E32662054252E32660A25534115
:107CF0006476616E636564207661726961626C6549
:107D0000733A20533D4D696E2066656564726174F7
:107D10006520286D6D2F73292C20543D4D696E20F0
:107D200074726176656C2066656564726174652045
:107D3000286D6D2F73292C20423D6D696E696D751C
:107D40006D207365676D656E742074696D6520289C
:107D50007573292C20583D6D6178696D756D2058BB
:107D600059206A65726B20286D6D2F73292C202095
:107D70005A3D6D6178696D756D205A206A65726B28
:107D800020286D6D2F73292C2020453D6D61786969
:107D90006D756D2045206A65726B20286D6D2F739F
:107DA000290A255320204D3230352053252E3266A6
:107DB0002054252E32662042256C752058252E32FF
:107DC000662059252E3266205A252E3266204525FA
:107DD0002E32660A2553486F6D65206F666673659F
:107DE0007420286D6D293A0A255320204D323036F3
:107DF0002058252E32662059252E3266205A252EEF
:107E000032660A004361703A25533A25630A0050EE
:107E1000525553415F4D4D553200455854454E44DF
:107E200045445F4D3230004155544F5245504F52FA
:107E3000545F504F534954494F4E004155544F528F
:107E400045504F52545F46414E53004155544F5296
:107E500045504F52545F54454D50000044656C6589
:107E600074696F6E206661696C65642C2046696C6C
:107E7000653A200046696C652064656C65746564CC
:107E80003A004E6F74205344207072696E74696EAC
:107E900067005072696E74207361766564005344A4
:107EA000207072696E74207061757365640025338B
:107EB000642F253364006676007468780050524E53
:107EC0000022283229006E6F2076616C696420637D
:107ED0006F6D6D616E64007A65726F72697A656448
:107EE00000666163746F727920726573746F726576
:107EF0006400696E6465782C2074656D702C207543
:107F0000737465702C20756D0050494E4441206398
:107F1000616C207374617475733A2000503A005795
:107F200061697420666F722050494E44412074612B
:107F3000726765742074656D7065726174757265C1
:107F40003A00204100205000204200204C002052E6
:107F500000205A00204E4F5420494E495449414C6C
:107F6000495A45440053686565742000205A2056DC
:107F7000414C5545204F5554204F462052414E47C5
:107F80004500496E76616C6964207368656574208C
:107F900049442E20416C6C6F7765643A20302E2E58
:107FA000004155544F004C414E472053454C20460C
:107FB0004F524345440020643A0020693A00207043
:107FC0003A0020643A0020693A0020703A0025699E
:107FD00025250A00256925250A0022283129002F98
:107FE0002F00002045585452554445525F434F5589
:107FF0004E543A3100204D414348494E455F545953
:1080000050453A00312E3000206261736564206F64
:108010006E204D61726C696E204649524D57415237
:10802000455F55524C3A68747470733A2F2F6769E4
:10803000746875622E636F6D2F707275736133642F
:108040002F50727573612D4669726D77617265206C
:1080500050524F544F434F4C5F56455253494F4E29
:108060003A00303030303030303030005F0038325D
:108070003337002B004649524D574152455F4E4120
:108080004D453A50727573612D4669726D77617214
:108090006520004D3131332053006F6B2000206389
:1080A0006D2E00206D696E20005354415453200002
:1080B0006E2F61003F546F736869626120466C6186
:1080C0007368416972204765744950206661696C24
:1080D00065640A00000125301D0CFF24311C0BFFD4
:1080E000232F1B0A17FF0406222B1A0336353538B7
:1080F0002569206D696E2C20256920736563004910
:108100006E76616C6964204D20636F64653A20254A
:10811000730A0050494E44412070726F62652063BB
:10812000616C6962726174696F6E207374617274DC
:10813000004E6F2050494E444120746865726D694D
:1081400073746F7200736574006E6F7A7A6C650079
:108150004D424C004652004C7A004C616E67003133
:108160005F37356D6D5F4D4B3235532D52414D426A
:108170006F3130612D453344763666756C6C005234
:10818000657600332E31342E312D383233370046A8
:10819000697200534E20696E76616C696400534EBB
:1081A000005245534554004D4D5552455300757688
:1081B0006C6F0046414E0046414E50494E54535458
:1081C0000050525553410047312058313020593129
:1081D0003830204634303030004731205A3130209A
:1081E0004631333030004D313430205330004D3182
:1081F000303420533000473120452D302E30373574
:1082000020463231303000473120463430303000A3
:108210004D323034205331303030004731205A3520
:1082200020463732303000473120452D312E352061
:108230004632313030004739300047312058352040
:108240004534204631303030004731205A302E320C
:108250002046313030300047312058353520453206
:108260003520463134303000473120592D322046F8
:1082700031303030004731205832343020453235EB
:1082800020204632323030004731205A302E332001
:1082900046313030300047312058353520453820C0
:1082A00046323030300047312058352045323920B1
:1082B0004631383030004731205835352045323985
:1082C00020463130373300473932204530004732BD
:1082D00038004D313039004D313930001000C902BD
:1082E00010012C014001220170011801B0010E01A2
:1082F000F00104015002FA00B002F0003003E60081
:10830000D003DC009004D2007005C800A006BE00B7
:108310000008B400B009AA00D00BA000600E9600BF
:1083200060118C000015820020197800C01D6E00BD
:10833000A0226400B0275A00902C50000031460063
:10834000E0343C0010383200903A2800603C1E00B7
:10835000A03D1400803E0A00203F00004578706573
:1083600072696D656E74616C00302E383000302E8D
:10837000363000302E343000302E323500446973F0
:1083800061626C65206661726D206D6F646500527C
:1083900065736574204D4D55004D4D55004D343479
:1083A000004739390044697361626C652066617207
:1083B0006D206D6F64653F00473238205859004D7D
:1083C00020383400852E2E002533642F30002533CD
:1083D000642F30006C63645F73656C66636865630B
:1083E0006B5F617869732025642C2025640A00483E
:1083F0006F74656E6400426564005A00590058004D
:108400002D2D2D2D2D2D2D2D2D2D2D2D2D2D2D2D9C
:108410002D2D2D2D00537570657250494E44413AF3
:1084200000E967F681EE81E681D981C78147312075
:10843000582564205925642045252D2E3566004792
:1084400031204631303830004731205A252D2E3327
:1084500066204637323030004731205835302059B9
:1084600031353500C7823682D96C27821B82108253
:1084700007824731205825642045252D2E3366205C
:10848000463130303000B682A68296828882C7821A
:1084900075826882578249823A8254256400473146
:1084A000205A302E342046313030300047312059A8
:1084B0002D3320463130303000E967D782D282CE6A
:1084C00082C7824D3834205859004D3130392053FD
:1084D0003238300047312058313235205A3230306E
:1084E00020463130303000496E76616C696420502E
:1084F00049442063616C2E20726573756C74732E11
:10850000204E6F742073746F72656420746F204501
:108510004550524F4D2E004D3330312050252E32D4
:10852000662049252E32662044252E3266004D33C2
:1085300030332045302053253375005243004445E5
:1085400056004245544100414C5048410000002132
:1085500000240027002A002D003000330001010014
:1085600000040107010A0100002200250028002B59
:10857000002E003100340002010000050108010B4B
:1085800001000020002300260029002C002F0032CB
:1085900000000100000301060109010505050507AA
:1085A0000508080808020202020A0A08080404046E
:1085B000040101010101010101030303030303039A
:1085C00003040707070C0C0C0C0C0C0C0C02020229
:1085D0000206060606060606060B0B0B0B0B0B0B1C
:1085E0000B07070A0A0A0A0A0A0505050404040813
:1085F00008010210202008081020401020408002AE
:1086000001020108040201010204081020408080D8
:10861000402010080402018004020180402010085C
:108620000402010804020101020408102040800134
:108630000204081020408010080408801020400424
:108640004080102040048000000A0B02090C0D0E2F
:108650000807030401000000000000000000000003
:10866000000000000000000000000000000000000A
:1086700000000012111000000000000000000000C7
:1086800000000000000000000000000000000000EA
:1086900000000000000000000000000000332E3148
:1086A000342E31000A204F726967696E616C205068
:1086B000727573612069330A2020205072757361CE
:1086C0002052657365617263680A2532302E32303C
:1086D000530053706F6F6C4A6F696E20697320008E
:1086E0006164635F696E697400200A200A200A20B1
:1086F00000416C6C2044617461005365727669635B
:10870000652070726570005368697070696E6720CB
:108710007072657000537461746973746963730077
:108720004C616E67756167650045524153494E471C
:1087300020616C6C206461746100466163746F72C7
:1087400079205245534554005052555341334446C5
:10875000570003000E00010040000300020000006B
:108760000400556E6B6E6F776E00313937302D30E7
:10877000312D30312030313A30303A303000203332
:108780002E31342E312D383233375F3030303030A7
:1087900030303030007374617274004D323900250E
:1087A0002D392E39535B0033332942000058419A4A
:1087B000998D4133335340200A200A20004D4D55F6
:1087C000323A004D6561737572652063656E74653C
:1087D0007220200078797A63616C5F6D65617375D2
:1087E00072655F656E7465720A0078797A63616C90
:1087F0005F73706972616C382063783D2564206313
:10880000793D2564207A303D256420647A3D2564D5
:10881000207261646975733D25642061643D25643F
:108820000A0078797A63616C5F7365617263685A74
:10883000206E6F207369676E616C0A20783D256C2D
:108840006420793D256C64207A3D256C640A002003
:108850004F4E2D5349474E414C20617420783D25A1
:108860006420793D2564207A3D25642061643D259E
:10887000640A0078797A63616C5F7365617263681A
:108880005A20783D256C6420793D256C64207A3D22
:10889000256C640A002530327800205B256620258F
:1088A000665D206D6D207061747465726E20636505
:1088B0006E7465720A00205B25662025665D5B2567
:1088C000665D206D6D20646976657267656E6365AF
:1088D0000A000000F000F801FC03FE07FE07FE0797
:1088E000FE07FC03F801F000000000000000F000AB
:1088F000F801FC03FC03FC03FC03F801F00000009A
:10890000000078797A63616C5F6D6561737572657B
:108910005F6C656176650A00203C20005741524E2D
:10892000494E473A2046726F6E7420706F696E74BC
:10893000206E6F7420726561636861626C652E20C1
:108940005920636F6F7264696E6174653A0000004C
:108950000040410000804000005C43000080400077
:10896000005C4300004443000040410000444325B4
:10897000642F3400497465726174696F6E3A200027
:1089800043616C6962726174696F6E206661696CC3
:1089900065642120436865636B2074686520617895
:1089A000657320616E642072756E20616761696E07
:1089B0002E004D494E54454D502042454420666995
:1089C000786564004D494E54454D5020484F5445FC
:1089D0004E442066697865640024F4D43050C38E18
:1089E00020C2A24017828B7011127A910D816CD92E
:1089F0000AA861E108C7586607615143061E4B5D2E
:108A000005C145A7041A411104093D980371393184
:108A1000034036DB0265339102D4305402802E1DB0
:108A200002632CEE01752AC501B028A00110278130
:108A3000018F2564012B244B01E0223401AC211F5E
:108A4000018D200D01801FFC00841EED00971DDFAD
:108A500000B81CD200E61BC600201BBC00641AB282
:108A600000B219A8000A19A0006A189900D117913C
:108A70000040178B00B516840031167E00B31579BF
:108A8000003A157300C7146F0058146A00EE13669D
:108A9000008813630025135E00C7125B006C125739
:108AA0000015125400C111510070114F0021114BDB
:108AB00000D61049008D10470046104400021042B5
:108AC00000C00F4000800F3E00420F3C00060F3BED
:108AD00000CB0E3800930E37005C0E3500270E34A5
:108AE00000F30D3200C10D3100900D3000600D2EED
:108AF00000320D2D00050D2C00D90C2B00AE0C29D9
:108B000000850C29005C0C2700350C27000E0C2674
:108B100000E80B2400C40B2400A00B23007D0B23D2
:108B2000005A0B2100390B2100180B2000F80A1FF6
:108B300000D90A1E00BB0A1E009D0A1D00800A1DE6
:108B400000630A1C00470A1B002C0A1B00110A1AAA
:108B500000F7091A00DD091900C4091900AB091949
:108B600000920917007B091800630917004C0916C9
:108B70000036091600200916000A091500F5081527
:108B800000E0081400CC081400B8081400A408146D
:108B900000900813007D0812006B0813005808129B
:108BA00000460812003408110023081100120811B1
:108BB0000001081100F0071000E0071000D00710B6
:108BC00000C0071000B0070F00A107100091070EAA
:108BD0000083070F0074070F0065070E0057070E8C
:108BE0000049070E003B070D002E070E0020070D61
:108BF0000013070D0006070D00F9060C00ED060D29
:108C000000E0060C00D4060C00C8060C00BC060CE4
:108C100000B0060C00A4060B0099060C008D060B94
:108C20000082060B0077060B006C060B0061060A3B
:108C30000057060B004C060A0042060A0038060AD6
:108C4000002E060A0024060A001A060A0010060969
:108C50000007060A00FD050900F4050900EB0509F7
:108C600000E2050900D9050900D0050900C705097A
:108C700000BE050900B5050800AD050800A50509F9
:108C8000009C050800940508008C05080084050870
:108C9000007C050800740508006C050700650508E0
:108CA000005D050700560508004E0507004705074B
:108CB000004005080038050700310507002A0507B0
:108CC00000230507001C050600160507000F050711
:108CD000000805060002050700FB040600F504076E
:108CE00000EE040600E8040600E2040700DB0406C8
:108CF00000D5040600CF040600C9040600C304061C
:108D000000BD040600B7040600B1040500AC04066B
:108D100000A6040600A00405009B040600950405B7
:108D200000900406008A04050085040500800406FE
:108D3000007A04050075040500700405006B040545
:108D40000066040500610405005C04050057040585
:108D500000520405004D04050048040500430405C5
:108D6000003E0404003A0405003504050030040404
:108D7000002C04050027040400230405001E04043D
:108D8000001A04040016040500110404000D040474
:108D900000090405000404040000040400FC0304AA
:108DA00000F8030400F4030400F0030400EC0304DF
:108DB00000E8030400E4030400E0030400DC03040F
:108DC00000D8030400D4030400D0030400CC03043F
:108DD00000C8030300C503030024F404D9201BC406
:108DE0000C5C0E9804C4095F0265077101F405F973
:108DF00000FB04B30048048700C103690058035511
:108E00000003034500BE023A008402310053022AE7
:108E1000002902250004022000E4011C00C80119F9
:108E200000AF0117009801140084011300710110B4
:108E3000006101100051010E0043010D0036010BCD
:108E4000002B010B0020010B00150109000C01098A
:108E50000003010800FB000800F3000800EB000716
:108E600000E4000600DE000600D8000600D200067E
:108E700000CC000500C7000500C2000500BD0004CD
:108E800000B9000400B5000400B1000400AD000406
:108E900000A9000400A5000300A20003009F000435
:108EA000009B00030098000300950002009300035C
:108EB00000900003008D0002008B00030088000278
:108EC000008600020084000300810002007F00028F
:108ED000007D0002007B00020079000200770001A3
:108EE00000760002007400020072000100710002AE
:108EF000006F0002006D0001006C0002006A0001BA
:108F000000690002006700010066000100650001C1
:108F100000640002006200010061000100600001C5
:108F2000005F0002005D0001005C0001005B0001C9
:108F3000005A0001005900010058000100570001CB
:108F400000560001005500010054000100530000CC
:108F500000530001005200010051000100500001C7
:108F6000004F0001004E0000004E0001004D0001C6
:108F7000004C0001004B0000004B0001004A0001C2
:108F800000490001004800000048000100470001BE
:108F900000460000004600010045000000450001B9
:108FA00000440001004300000043000100420000B3
:108FB00000420001004100000041000100400001AA
:108FC000003F0000003F0001003E0000003E0001A5
:108FD000003D0000003D0001003C0000003C00009E
:108FE000003C0001003B0000003B0001003A000093
:108FF000003A00010039000000390001003800008B
:109000000038000000380001003700000037000180
:109010000036000000360000003600010035000078
:10902000003500000035000100340000003400006D
:109030000034000100330000003300000033000161
:109040000032000000320000003200010031000058
:10905000003100000031000100300000003000004D
:1090600000300001002F0000002F0000002F000042
:10907000002F0001002E0000002E0000002E000135
:10908000002D0000002D0000002D0000002D00012B
:10909000002C0000002C0000002C0000002C00011F
:1090A000002B0000002B0000002B0000002B000113
:1090B000002A0000002A0000002A0000002A000107
:1090C00000290000002900000029000000290000FC
:1090D00000290001002800000028000000280000EE
:1090E00000280000002800010027000000270000E1
:1090F00000270000002700000027000100260000D4
:1091000000260000002600000026000000260001C6
:1091100000250000002500000025000000250000BB
:1091200000250000002500010024000000240000AC
:10913000002400000024000000240001002300009F
:109140000023000000230000002300000023000093
:109150000023000000230001002200000022000084
:109160000022000000220000002200000022000176
:10917000002100000021000000210000002100006B
:10918000002100000021000000210001002000005B
:10919000002000000020000000200000002000004F
:1091A000002000000020000000200001001F00003F
:1091B000001F0000001F0000001F0000001F000033
:1091C000001F0000001F0001001E0000001E000024
:1091D000001E0000001E00000045303A20005A3AF0
:1091E0002000593A2000583A20004D53312C4D535D
:1091F000322050696E7300504944204175746F7479
:10920000756E652066696E697368656421205075A6
:109210007420746865206C617374204B702C204B33
:109220006920616E64204B6420636F6E7374616E9D
:1092300074732066726F6D2061626F766520696E4F
:10924000746F20436F6E66696775726174696F6EC3
:109250002E6800504944204175746F74756E652006
:109260006661696C6564212074696D656F75740051
:1092700020403A00543A00423A0050494420417597
:10928000746F74756E65206661696C656421205425
:10929000656D706572617475726520746F6F20689A
:1092A00069676800204B643A2000204B693A20002F
:1092B000204B703A200020436C6173736963205027
:1092C000494420002054753A2000204B753A200074
:1092D000206D61783A2000206D696E3A200020648C
:1092E0003A200020626961733A20005049442041CD
:1092F00075746F74756E6520737461727400504973
:1093000044204175746F74756E65206661696C6583
:10931000642E2042616420657874727564657220E1
:109320006E756D6265722E00486F74656E6420669E
:10933000616E207370656564206973206C6F77655A
:1093400072207468616E206578706563746564006E
:109350005072696E742066616E207370656564205A
:109360006973206C6F776572207468616E20657810
:10937000706563746564004D494E54454D502042FC
:109380004544004D494E54454D50004D41585445BB
:109390004D50004D415854454D50204245440070B9
:1093A000012C0190012701B0012201C0011D01F033
:1093B0000118011002130130020E01600209019030
:1093C000020401C002FF000003FA004003F5008020
:1093D00003F000D003EB002004E6007004E100E09D
:1093E00004DC004005D700C005D2004006CD00D007
:1093F00006C8008007C3003008BE00F008B900C0EE
:1094000009B400B00AAF00B00BAA00D00CA5000050
:109410000EA000500F9B00C010960050129100004B
:10942000148C00C0158700B0178200B0197D00D0E1
:109430001B7800001E730040206E0090226900F02F
:1094400024640040275F0090295A00E02B5500104B
:109450002E500020304B0010324600E03341009087
:10946000353C001037370070383200A0392D00B07D
:109470003A2800A03B2300603C1E00103D190090DC
:109480003D1400103E0F00703E0A00C03E05000073
:109490003F000020484F54454E4420544845524D0B
:1094A000414C2052554E41574159002048454154A6
:1094B00042454420544845524D414C2052554E415E
:1094C00057415900544845524D414C2052554E4148
:1094D0005741590042454420544845524D414C2083
:1094E00052554E415741590020544845524D414C28
:1094F0002052554E41574159202850524548454128
:109500005420484F54454E44290020544845524D5C
:10951000414C2052554E4157415920285052454800
:109520004541542048454154424544290050524544
:1095300048454154204552524F5200424544205024
:10954000524548454154204552524F5200207472B2
:109550006967676572656421004865617465727347
:10956000207377697463686564206F66662E2000D7
:109570003A20004572723A200000FF010201000209
:10958000FFFFFE0001FE01FF00506C656173652066
:109590007265737461727400555341525432207273
:1095A000782046756C6C212121003A2000252D3150
:1095B000322E313253252D642F36002533642F256A
:1095C0002D336400203A200025335300252D3773B6
:1095D00000252D31352E313553252D35640A252DA5
:1095E00031352E313553252D35640A0025530A2097
:1095F000252D31362E313653252D33640A20252D65
:1096000031362E313653252D33640025530A20255B
:109610002D31362E313653252D33640A20252D3138
:10962000362E313653252D33640A20252D31362E22
:10963000313653252D33640025530A20252D31362C
:109640002E313653252D33640A25530A20252D311A
:10965000362E313653252D33640A002025732533E9
:109660006481200A0025752E25752E25752E2575F9
:109670000020002000466C617368416972204950E7
:1096800020416464723A004D4D5520202020202056
:1096900020204E2F410025642E25642E25640020B5
:1096A00046573A00313937302D30312D30310045B1
:1096B0003344763666756C6C0052414D426F3130E2
:1096C0006100315F37356D6D5F4D4B323553002092
:1096D000486173683A3030303030303030300020FC
:1096E0005265706F3A556E6B6E6F776E0020332E39
:1096F00031342E312D38323337004669726D77613F
:1097000072653A00464C4558202D20203234302FC7
:10971000353000464C4558202D2020323430005042
:10972000502020202D20203235342F313030005071
:10973000502020202D20203235340048495053201D
:109740002D20203232302F31303000484950532004
:109750002D20203232300041425320202D20203253
:1097600035352F3130300041425320202D2020321A
:1097700035350050412020202D20203237352F391B
:10978000300050412020202D202032373500505607
:109790004220202D20203231352F373500505642BF
:1097A00020202D20203231350050432020202D2034
:1097B000203237352F3130350050432020202D20E6
:1097C000203237350041534120202D2020323630C1
:1097D0002F3130350041534120202D2020323630AA
:1097E0000050455420202D20203233302F383500B2
:1097F00050455420202D202032333000504C412041
:10980000202D20203231352F363000504C41202081
:109810002D2020323135006E6F7A7A6C65202D2034
:10982000203235302F30006661726D2020202D20CF
:10983000203235302F383000252D31322E31325341
:10984000252B382E31660045787472756465723A3E
:109850000025632531372E32666D6D00583A005968
:109860003A005A3A002563252D31332E31335325E2
:109870002B352E3366002533750050494E44412068
:1098800063616C6962726174696F6E206661696C94
:1098900065642E20436F6E74696E756520776974F8
:1098A00068207072657373696E6720746865206BD9
:1098B0006E6F622E0050494E44412063616C6962B4
:1098C000726174696F6E20646F6E652E20436F6ED7
:1098D00074696E756520776974682070726573733A
:1098E000696E6720746865206B6E6F622E005A3057
:1098F000005A3100593000593100583000583100B9
:10990000456E642073746F707320646961670047EB
:109910003830004D3435004D3435205A0047373645
:10992000004D3730312050300057697A6172642021
:1099300073746174653A2025640A0078797A6361EA
:109940006C5F73706972616C322063783D256420AE
:1099500063793D2564207A303D256420647A3D2575
:1099600064207261646975733D25642061643D25DE
:10997000640A000A00436F756E74646F776E3A2054
:109980002564200025640A005363616E20636F75AF
:109990006E74646F776E3A20005061747465726EF5
:1099A0002063656E746572205B25662025665D2CDC
:1099B000206D6174636820256625250A00205B25DB
:1099C000662C2025665D5B25665D2066696E616C90
:1099D00020636972636C650A000000A0400000A06B
:1099E000400000004000007A43000056439AD951DD
:1099F00043FFFFFFE02D903E8988B24111369C3E27
:109A00007777C14129CBB03EEFEEDA41BA49CC3E7F
:109A1000EFEEFC4161C3F33EEFEE16429CA2133F12
:109A2000CDCC36428AB0113FABAA56428863DD3DA9
:109A3000ABAA5642B8AF433F555572421826533F22
:109A400033B38242302A593FEF6E8642000070C124
:109A50000000C8420000C4C10000A0410000E0C0F6
:109A600000002041000060C00000C0400000A04194
:109A70002222F2400000A0C19A99A14000000CC22D
:109A800055550542436F6F6C696E672074696D654B
:109A9000722073746F7070656400486561746572DC
:109AA00020636F6F6C646F776E00436F6F6C696ECD
:109AB000672054696D656F75742073746172746585
:109AC0006400536176696E6720616E642070617214
:109AD0006B696E670048656174657220636F6F6CB7
:109AE000646F776E2070656E64696E67005265738F
:109AF000756D696E672058595A00473120582564A2
:109B00002059252D2E32662045252D2E33660057EF
:109B1000726974696E6720746F2066696C653A209B
:109B20000046696C6520616C7265616479206F70B4
:109B3000656E656400315820580C58F757E157CED0
:109B400057B857A45793577D570C58205869575A00
:109B500057465735572057C45A0A57F856E556D432
:109B600056BF56AC56985683567A56685653564D3D
:109B7000363030204155544F0046494E444120660E
:109B8000696C616D656E742072756E6F75742100FD
:109B9000436F6D6D756E69636174696F6E20746972
:109BA0006D656F75740050726F746F636F6C2045D4
:109BB00072726F720003000356657273696F6E20D4
:109BC0006D69736D6174636800436F6D6D616E6480
:109BD000204572726F7200436F6D6D616E6420720A
:109BE000656A6563746564004D4D552042757474F3
:109BF0006F6E207075736865640052657472794287
:109C00007574746F6E50726573736564008E5A79E3
:109C10005A625A4D5A385A245A145AFD59E659CFA5
:109C200059BB59A7599159915991597C597C597CE3
:109C3000596959695969595659565956593F593FA1
:109C4000593F592A592A592A59145914591459044F
:109C500059EF58D958C358B458A75890587D586BE5
:109C600058585846583658427574746F6E00436899
:109C700065636B55736572496E7075742D62746E91
:109C80004C4D52200052657365745265747279416F
:109C90007474656D7074730046493A202046533AD7
:109CA000202020203E2020822020208100486F7428
:109CB000656E642074656D7065726174757265207F
:109CC0007265616368656400526573756D696E677E
:109CD0002054656D7000436F6F6C646F776E206603
:109CE0006C616720636C65617265640020573A009F
:109CF00020453A00543A004E6F2030784646207294
:109D0000656365697665640053656E64696E672096
:109D1000307846460046696C652073656C656374EF
:109D20006564002053697A653A200046696C6520B5
:109D30006F70656E65643A20004E6F7720667265BD
:109D400073682066696C653A20004E6F7720646FF7
:109D5000696E672066696C653A20002220706F7317
:109D6000002220706172656E743A2200535542528F
:109D70004F5554494E452043414C4C207461726705
:109D800065743A2200747279696E6720746F20637B
:109D9000616C6C207375622D67636F646520666902
:109DA0006C6573207769746820746F6F206D616EC5
:109DB00079206C6576656C732E0020222573220055
:109DC0002025236C78004449525F4558495400448B
:109DD00049525F454E5445523A202573202225733F
:109DE000220A006175746F25692E6700041A4465A4
:109DF0006372656D656E74526574727941747465D1
:109E00006D70747300081B1C0B14525354436F6D18
:109E10006D54696D656F7574002C206C61737420CE
:109E200062797465733A200022206661696C65640A
:109E30003A204275666665722066756C6C21002258
:109E400000456E717565696E6720746F2074686572
:109E50002066726F6E743A2022004572726F723AF9
:109E6000004D4D5532746F6F6C3D004D4D55323A7B
:109E7000004D4D55323A006563686F3A003E5330ED
:109E80002A63362E004D4D552069732000252E3152
:109E90003053200025346400457872656D65207369
:109EA00070616E206F6620746865205A2076616C40
:109EB000756573210025642F39004D4D55323A00E8
:109EC0002533640018010419020A5462DE616461DA
:109ED000F760AE601C60A45F3C5FED5ECD5E815EAE
:109EE000CD5E6A5E6A5E6A5E6A5E6A5E6A5E6A5ECF
:109EF0006A5E6A5E6A5E6A5E6A5E6A5E6A5E6A5E22
:109F00006A5E6A5E6A5E6A5E6A5E6A5E6A5E335E48
:109F1000F25DA85D355D005DB65C6C5C0E5CD55B8A
:109F2000935B765B01010101010101027101710185
:109F30003232320303030303030303030303030364
:109F4000030303030303939324380393030102568B
:109F500003650066006700680069006A006B006CBA
:109F600000730074007D007E00C900D300DD00CACC
:109F700000D400DE002D01370141012E01380142DD
:109F8000012F013901430130013A01440131013B04
:109F9000014501320191019201F501F601F701F845
:109FA00001F901FA01FB01FC018403E1624A63D675
:109FB00062CD62C662414B503DBF62B562252E3212
:109FC00030530A70727573612E696F2F30342568B3
:109FD00075007B5B4552523A00332E31342E3100EE
:109FE0005D5B4657523A005D5B54494D3A005D5BFC
:109FF000464E4D3A005D5B46454D3A005D5B504331
:10A00000443A005B5446553A005B50524E3A005B6E
:10A0100050464E3A305D005B4449413A005D5B4139
:10A0200054423A005D5B4154303A005D5B53544208
:10A030003A005B5354303A007B5B50524E3A355DE8
:10A04000007B5B50524E3A305D007B5B50524E3A83
:10A05000395D007B5B50524E3A385D007B5B524568
:10A06000533A305D5B46494C3A007B5B5245533A6C
:10A07000315D5B46494C3A000000211042206330BC
:10A080008440A550C660E770088129914AA16BB150
:10A090008CC1ADD1CEE1EFF13112100273325222F8
:10A0A000B5529442F772D662399318837BB35AA3A0
:10A0B000BDD39CC3FFF3DEE36224433420040114C8
:10A0C000E664C774A44485546AA54BB528850995F0
:10A0D000EEE5CFF5ACC58DD5533672261116300698
:10A0E000D776F6669556B4465BB77AA71997388740
:10A0F000DFF7FEE79DD7BCC7C448E5588668A77858
:10A100004008611802282338CCC9EDD98EE9AFF98F
:10A11000488969990AA92BB9F55AD44AB77A966A37
:10A12000711A500A333A122AFDDBDCCBBFFB9EEBDF
:10A13000799B588B3BBB1AABA66C877CE44CC55C07
:10A14000222C033C600C411CAEED8FFDECCDCDDD2F
:10A150002AAD0BBD688D499D977EB66ED55EF44ED7
:10A16000133E322E511E700E9FFFBEEFDDDFFCCF7F
:10A170001BBF3AAF599F788F8891A981CAB1EBA1D3
:10A180000CD12DC14EF16FE18010A100C230E3204F
:10A190000450254046706760B9839893FBA3DAB3F7
:10A1A0003DC31CD37FE35EF3B1029012F322D2329F
:10A1B0003542145277625672EAB5CBA5A8958985C7
:10A1C0006EF54FE52CD50DC5E234C324A0148104EF
:10A1D0006674476424540544DBA7FAB79987B89797
:10A1E0005FE77EF71DC73CD7D326F2369106B0163F
:10A1F00057667676154634564CD96DC90EF92FE957
:10A20000C899E9898AB9ABA944586548067827688E
:10A21000C018E1088238A3287DCB5CDB3FEB1EFB36
:10A22000F98BD89BBBAB9ABB754A545A376A167ADE
:10A23000F10AD01AB32A923A2EFD0FED6CDD4DCD06
:10A24000AABD8BADE89DC98D267C076C645C454C2E
:10A25000A23C832CE01CC10C1FEF3EFF5DCF7CDFD6
:10A260009BAFBABFD98FF89F176E367E554E745E7E
:10A27000932EB23ED10EF01E7C3C3E3F2F2A225C34
:10A280000000F338E25E11241FBECFEFD1E2DEBF43
:10A29000CDBF00E00CBF13E0A0E0B2E0E2E9FEE4D5
:10A2A00003E00BBF02C007900D92A430B107D9F7AD
:10A2B00027E1A4E0B3E001C01D92A430B207E1F7AA
:10A2C00011E5C2E4D1E500E006C021970109802F25
:10A2D000FE010F948DA1C134D10780E00807A9F7D2
:10A2E0000E9499D80D9437A70C9446752F923F92EF
:10A2F0004F925F926F927F928F929F92AF92BF9296
:10A30000CF92DF92EF92FF920F931F93CF93DF9341
:10A31000CDB7DEB72F970FB6F894DEBF0FBECDBF17
:10A320006C011B015A01FC011782168283819E0178
:10A330002F5F3F4F490181FDD2C08FEF9FEFEEC2EB
:10A34000F12C512C00E0003238F48B3209F190F4FA
:10A350008032F9F0833209F107FD34C020ED280F77
:10A360002A3020F506FF1BC0FAE0FF9E200D1124C5
:10A37000F22E05C08D3279F0803371F70160F10162
:10A3800093FD859193FF81911F018111DCCF1AC04C
:10A3900002600460F4CF0860F2CF0061F0CF3AE0D1
:10A3A000539E200D1124522E0062E9CF8E3221F4EB
:10A3B00006FDB1C20064E3CF8C3611F40068DFCF34
:10A3C0008836E9F29BEB980F933008F05FC000618C
:10A3D000805E06FD02C046E0F42E102F1F73853606
:10A3E00009F05BC0106417FF61C08F2D9BE39F15C0
:10A3F00008F48BE344244394480E27E03501F4E04D
:10A400006F0E711CF5016081718182819381042D31
:10A41000A4010F94369D5C01F981FC87F0FF03C015
:10A420000DE2F3FF07C00BE211FD04C0012F047021
:10A4300012FD00E22C852C70E22E09F46BC0011194
:10A44000D8C2F3E0E12CF515A0F483E0E52CE81A7E
:10A4500013FD08C0B60180E290E00F94E59EEA94F7
:10A46000E110F8CF002329F0B601802F90E00F947F
:10A47000E59E3C852EEEA22E21E7B22E33FD04C0D0
:10A4800092EFA92E91E7B92E107122C09BE9980F87
:10A49000933008F047C10F7E9CCF863611F41068C8
:10A4A000A2CFFF2009F49FCFFA949DCFE7E02F2D94
:10A4B000EF1518F427E037E0F32E412C9FCF111150
:10A4C0008052B60190E00F94E59E8FEFA81AB80A6B
:10A4D000F50184918111F3CFE11084C25301F6019B
:10A4E0009381F10193FD859193FF81911F01882351
:10A4F00009F411C2853241F493FD859193FF819156
:10A500001F01853209F01CCFB60190E00F94E59E43
:10A510003501E4CF17FF6FC04A0CFC85F4FF04C07F
:10A520008A81813309F44A9414140CF086C028E01F
:10A53000241510F488E0482E85E090E017FF06C04F
:10A54000C501B7FE02C090E080E0019601110196BE
:10A55000FF2031F02F2D30E02F5F3F4F820F931FF0
:10A560005816190619F014F0E52CE81A812F897095
:10A5700011F4E11067C0002329F0B601802F90E0AC
:10A580000F94E59E13FD02C0E11063C017FF7CC06D
:10A590008501B7FE02C010E000E0C50184199109F1
:10A5A0002C016F2D70E0EE27FF27E61BF70BFF87CE
:10A5B000EE870F3F100729F4B6018EE290E00F946A
:10A5C000E59EA016B1060CF44BC0401651060CF0E7
:10A5D00047C0F501E01BF10BE80DF91D8181015029
:10A5E00011092E853F8502171307E4F1B60190E0AB
:10A5F0000F94E59EDECF16FD9FCFEF2DF0E0EA151C
:10A60000FB0534F03CEFA3163FEFB3060CF01068E7
:10A610003296E80DF91D01C0FA94FF2019F08291DD
:10A620008033D1F317FF88CF442443944F0CFA149E
:10A630001B0431F02CF0FA187FCF442443947CCFD4
:10A64000F12C7ACFB60180E290E00F94E59EEA9477
:10A6500090CFB60180E390E00F94E59EEA9494CF0A
:10A6600080E3BDCFA016B10641F49A81963350F431
:10A67000953319F43C8534FF05C0B60190E00F9482
:10A68000E59E2ACF81E3F9CF8A81813319F09C8539
:10A690009F7E9C87B60190E00F94E59EFF20A9F075
:10A6A000B6018EE290E00F94E59EF394F394E2E01D
:10A6B00001E00E0FE80DF92DF11D8081B60190E04B
:10A6C0000F94E59EE02F0F11F3CF85E690E014FF85
:10A6D00002C085E490E0B6010F94E59EB7FC06C089
:10A6E000A114B104C1F4EC85E4FF15C0B194A194A8
:10A6F000B1088DE2B60190E00F94E59E80E32AE078
:10A70000A216B10454F4B60190E00F94E59EB60190
:10A71000C501C096B4CF8BE2EDCF8F5FFAE0AF1AE0
:10A72000B108EDCF8336C9F0833771F1833509F075
:10A730005BC03501F2E06F0E711CF501A080B180A5
:10A740006F2D70E006FD02C06FEF7FEFC5010F9423
:10A75000799E9D878C8700680DC0350132E0630EBD
:10A76000711CF5018081898321E030E03D872C87D1
:10A7700054010F7703FD06C02C853D855216130644
:10A7800009F0A8F4E52C2BC0350132E0630E711CF2
:10A79000F501A080B1806F2D70E006FD02C06FEF63
:10A7A0007FEFC5010F949E9E9D878C87E2CFB601F7
:10A7B00080E290E00F94E59E5A94DECFF50107FD0C
:10A7C000859107FF81915F01B60190E00F94E59EAE
:10A7D000E110EA948C859D8501979D878C87EC8597
:10A7E000FD85EF2B59F778CE843619F0893609F0BC
:10A7F00074C0350107FF66C0F4E06F0E711CF501EF
:10A800006081718182819381102F1F7697FF08C02C
:10A8100090958095709561957F4F8F4F9F4F1068F1
:10A820002AE030E0A4010F940CA0A82EA818BA2C9E
:10A83000012F16FF0AC00E7FAF1438F414FF04C0B6
:10A8400012FD02C0012F0E7EBF2C04FFA3C0FE012B
:10A85000EA0DF11D8081803309F095C0097EF02F4B
:10A86000F870EF2E03FDA5C000FF9FC0FA2CB514B1
:10A8700010F4F50CFB1804FFA2C0B60180E390E0D1
:10A880000F94E59E02FF09C088E790E001FF02C037
:10A8900088E590E0B6010F94E59EAF1408F49BC0E4
:10A8A000AA940A2D10E00F5F1F4F080D191DF80123
:10A8B00082918F01B60190E00F94E59E801691067B
:10A8C000B1F70ACEF2E06F0E711CF5016081718163
:10A8D000072E000C880B990B97CF102F8537A9F402
:10A8E0001F7E2AE030E0350117FF44C0F4E06F0E10
:10A8F000711CF5016081718182819381A4010F94A3
:10A900000CA0A82EA8181F7792CF197F8F3679F147
:10A91000F0F4883539F1F601868197812F960FB6CC
:10A92000F894DEBF0FBECDBFDF91CF911F910F9185
:10A93000FF90EF90DF90CF90BF90AF909F908F905F
:10A940007F906F905F904F903F902F900895803749
:10A9500039F0883701F714FD146020E130E0C3CFEF
:10A960001061F9CF04FD166020E132E0BCCF28E091
:10A9700030E0B9CFF2E06F0E711CF501608171819A
:10A9800090E080E0BBCF02FD02C0B39468CFB394E7
:10A99000B39465CF802F867809F461CFF6CFB601E6
:10A9A00080E290E00F94E59EB394B514C0F3E12CDF
:10A9B00062CFE52CEB18B51408F45DCFF8CF802FEB
:10A9C000867809F46ACF8BE201FF80E207FD8DE211
:10A9D000B60190E060CFB60180E390E00F94E59E71
:10A9E000FA945BCFB60180E290E00F94E59EEA9482
:10A9F00073CD24E0E12C251508F036CD84E026CD7A
:10AA000020E030E040E85FEB60917E0270917F02D1
:10AA100080918002909181020F949AA2882321F163
:10AA2000E091CB11F091CC11E252F04F80818B7FFD
:10AA30008230D1F480E1EEE7F2E0A5EFB1E10190E0
:10AA40000D928A95E1F780E090E0A0E8BFEB80935B
:10AA50007E0290937F02A0938002B0938102809146
:10AA6000E0119091E111089581E090E0089580E176
:10AA7000E3E9F6E0A5EFB1E101900D928A95E1F7E7
:10AA80000895E6ECF6E7833021F0E82FF0E0ED538F
:10AA9000F948849108958091AF059091B005209177
:10AAA000B1053091B205821B930B8F7799270895DA
:10AAB000982F9F7083FF0DC080917B0088608093EA
:10AAC0007B0080917C00887F9770892B80937C002D
:10AAD000089580917B00877FF2CF8091B10590919E
:10AAE000B2059093B0058093AF0585ED99E69F93ED
:10AAF0008F938091D1119091D211A091D311B091E7
:10AB0000D4110196A11DB11DBF93AF939F938F9355
:10AB10008DEF94E69F938F9384E095E69F938F93B8
:10AB20000F943F9F8DB79EB70A960FB6F8949EBFBD
:10AB30000FBE8DBF08950F931F93CF93DF93EC014A
:10AB4000C60FD71F8C179D0779F08C010F5F1F4F21
:10AB50000F947DA08F3F31F081E0DF91CF911F9165
:10AB60000F910895C801EECF80E0F7CF682F880FCE
:10AB7000770B8091CB119091CC118F51904F0F9406
:10AB8000D4A69C019093F6168093F51681E0232BB2
:10AB900009F480E008958091F5169091F6164AE048
:10ABA00050E070E060E001960F94089C862F0895B5
:10ABB0008091F5169091F6164AE050E070E060E062
:10ABC00001960F94089CCB0108950F931F93CF9388
:10ABD000DF938C01862FEA010E94B655882319F174
:10ABE0000E94D8559C0197FF03C0319521953109EA
:10ABF000253631059CF09F938F938AE59EE99F93BC
:10AC00008F9383E497E79F938F930F943F9F0F90C9
:10AC10000F900F900F900F900F9080E0DF91CF91E9
:10AC20001F910F910895F80180818823B1F3CE011F
:10AC3000DF91CF911F910F910D947DA08091F5161A
:10AC40009091F6164AE050E070E060E001960D94B5
:10AC5000089C60E086E69FE00F94A1A060E088E693
:10AC60009FE00F94A1A060E085E69FE00F94A1A073
:10AC700060E084E69FE00F94A1A060E082ED9EE09A
:10AC80000F94A1A060E08FEC9EE00D94A1A080360F
:10AC90009105F8F44091CB115091CC112091DC0F2B
:10ACA0003091DD0F4217530739F46091CF11709145
:10ACB000D011161617066CF0B901680F791FFB0149
:10ACC000E359FF4F2417350730F481E04E175F0733
:10ACD00008F480E00895EE3EF140F8F06C5F7F4F9D
:10ACE0006E3E714018F449365105B8F483599F4FB0
:10ACF0004817590770F34DEE51E0421B530B70E0BB
:10AD000060E0C9018252904F0F94AFA68FB7F894BC
:10AD10001092DD0F1092DC0F8FBF81E008952F920B
:10AD20003F924F925F926F927F928F929F92AF92DB
:10AD3000BF92CF92DF92EF92FF920F931F93CF9328
:10AD4000DF93CDB7DEB7CC58D2400FB6F894DEBF54
:10AD50000FBECDBFCB58DD4F688379838A839B8339
:10AD6000C557D240FE01E754FE4F88E2DF011D9235
:10AD70008A95E9F7E85BF1401F0180E991E0DF0186
:10AD8000FC011D923197E9F7C75ADD4F19821882ED
:10AD9000C955D2409E012F513E4FC159DD4F3983D5
:10ADA0002883CF56D2408E01075A1D4FCE018F5CAB
:10ADB0009D4FC359DD4F99838883CD56D2403C01C6
:10ADC000490140EBA42E4FE0B42E53E2C52ED12C06
:10ADD000F12CE12CB6010D2C000C880B990B0F9473
:10ADE0000B9BD4016D937D938D939D934D01F80141
:10ADF000619171918F01072E000C880B990B0F94B4
:10AE00000B9BD3016D937D938D939D933D01BFEF7C
:10AE1000EB1AFB0AE6E0EE16F10409F038C3CB5852
:10AE2000DD4F288139814A815B81C557D240C159A4
:10AE3000DD4FA881B981CF56D2406D917D918D9122
:10AE40009C910F942EA4412C512C320118160CF415
:10AE500002C3C359DD4F08811981CD56D2400C5E23
:10AE60001F4FC159DD4FE880F980CF56D240B4E181
:10AE7000EB0EF11C6E01EFEDCE1AEDEFDE0A9E0136
:10AE80002B553E4FCF58DD4F39832883C157D240D1
:10AE9000D8014D905D906D907C90F701608171813B
:10AEA00082819381D7015E914E913E912E917D01D9
:10AEB0000F94A4A14B015C01F8015291429132918F
:10AEC00022918F01C301B2010F94A4A1A5019401A5
:10AED0000F94A4A2D6019E938E937E936E936D01E0
:10AEE000CF58DD4FE881F981C157D240B292A2928A
:10AEF00092928292CF58DD4FF983E883C157D240B6
:10AF0000C359DD4F28813981CD56D240021713072E
:10AF100009F0BECF4E013FE6831A3EEF930A5E0171
:10AF200083EFA81A8DEFB80A61018101EE24E39442
:10AF3000F12CD4014D905D906D907D904D012D913F
:10AF40003D914D915C91C301B2010F94A5A19B016C
:10AF5000AC010F94A5A1F80164A775A786A797A7D0
:10AF6000F1E0EF16F10461F0D80198964D925D92F0
:10AF70006D927C929B97F80144825582668277821B
:10AF8000FFEFEF1AFF0AF5012081318142815381E1
:10AF900084E0A80EB11C64817581868197810F942D
:10AFA000A4A120E030E040EC50E40F944A9BD6018D
:10AFB000DC966D937D938D939C93DF97045D1F4F7B
:10AFC000B8E2CB0ED11CE5E0EE16F10409F0B1CFEA
:10AFD0007E01FDE2EF0EF11C28E2A22EB12C00EB67
:10AFE0001FEF24E0220E311CD7012D913D914D9190
:10AFF0005C91139798966D917D918D919C919B9703
:10B000000F94A4A22B013C016101C01AD10A88242B
:10B010008394912CF601E00FF11FEA0DFB1D2081B6
:10B02000318142815381C301B2010F944A9B9B013C
:10B03000AC01F60160817181828193810F94A4A19A
:10B04000D6016D937D938D939D936D01BFEF8B1A08
:10B050009B0AE6E08E169104E9F63CE2E30EF11C51
:10B060000852110988E2A80EB11C08339FEF190796
:10B0700009F0BACF1E01F5EB2F0E311C6E0121EB4A
:10B08000C20ED11C7E0137E3E31A3EEFF30A04E05F
:10B0900010E04801B12CA12C412C512C3201F601B9
:10B0A000EA0DFB1DD701AA0DBB1D2D913D914D91C0
:10B0B0005C9160817181828193810F944A9B9B0195
:10B0C000AC01C301B2010F94A5A12B013C018FEF8C
:10B0D000881A980A94E0A90EB11CA5E08A1691047A
:10B0E000F1F6A3019201F101608171818281938166
:10B0F0000F94A4A1D6012D913D914D915C910F9497
:10B10000A4A2F701608371838283938301501109A4
:10B11000F8E22F1A31082CE2C21AD10834E0E31AFF
:10B12000F1080115110509F0B4CFCB50DE4F88812D
:10B130009981AA81BB81C55FD140CF57DD4F8883FC
:10B140009983AA83BB83C158D2401E0197E4291A70
:10B150009EEF390A10E000E0C159DD4FA881B981A6
:10B16000CF56D240CD90DD90ED90FD90C159DD4F8E
:10B17000B983A883CF56D240CB58DD4F288139817F
:10B180004A815B81C557D240C701B6010F949AA28C
:10B190001816B4F0CB58DD4F288139814A815B8184
:10B1A000C557D240C159DD4FE881F981CF56D24011
:10B1B00060817181828193810F942EA487FF18C0D2
:10B1C0000430110509F030C1CB58DD4F2881398199
:10B1D0004A815B81C557D240CF57DD4F6881798165
:10B1E0008A819B81C158D2400F949AA287FF1CC1CB
:10B1F000D10114968D909D90AD90BC9017978D9134
:10B200009D910D90BC91A02DCF58DD4F88839983DF
:10B21000AA83BB83C157D240F801EE0FFF1FEE0F88
:10B22000FF1F21E931E02C0F3D1FE20FF31F40808B
:10B23000518062807380C359DD4FA881B981CD569A
:10B24000D2408D919D910D90BC91A02DC358DD4FA2
:10B2500088839983AA83BB83CD57D240A7019601E7
:10B26000CB58DD4F688179818A819B81C557D24057
:10B270000F94A4A16B017C0120E030E040E450E495
:10B280000F9415A5CB57DD4F688379838A839B8301
:10B29000C558D240C358DD4F288139814A815B812E
:10B2A000CD57D240C359DD4FE881F981CD56D24008
:10B2B00064817581868197810F94A4A1A301920175
:10B2C0000F94A4A2C758DD4F688379838A839B8338
:10B2D000C957D240A3019201C301B2010F94A5A1A5
:10B2E000CF58DD4F288139814A815B81C157D240D7
:10B2F0000F944A9BC757DD4F688379838A839B836A
:10B30000C958D240A3019201C501B4010F944A9BD0
:10B310009B01AC01C757DD4F688179818A819B8190
:10B32000C958D2400F94A5A120E030E040EC50E491
:10B330000F94A4A29B01AC01C758DD4F68817981AD
:10B340008A819B81C957D2400F94A4A1A70196017D
:10B350000F944A9BC758DD4F688379838A839B8308
:10B36000C957D240CF58DD4F288139814A815B814E
:10B37000C157D240C501B4010F94A4A14B015C0197
:10B3800020E030E040EC50E4C301B2010F944A9B4E
:10B390009B01AC01C501B4010F94A4A2CB57DD4FB2
:10B3A000288139814A815B81C558D2400F944A9BDC
:10B3B0004B015C0120E030E040E05FE3CF58DD4F1F
:10B3C000688179818A819B81C157D2400F944A9BC1
:10B3D0002B013C01A7019601C701B6010F944A9BBE
:10B3E0009B01AC01C301B2010F944A9B9B01AC01CC
:10B3F000C501B4010F94A5A19B01AC01C758DD4F55
:10B40000688179818A819B81C957D2400F94A5A117
:10B41000C358DD4F288139814A815B81CD57D240A5
:10B420000F94A5A12B013C010F5F1F4FF4E02F0EDD
:10B43000311CC359DD4F28813981CD56D2402C5F54
:10B440003F4FC359DD4F39832883CD56D240053055
:10B45000110509F081CEC301B201C457DD4F0FB60B
:10B46000F894DEBF0FBECDBFDF91CF911F910F913A
:10B47000FF90EF90DF90CF90BF90AF909F908F9014
:10B480007F906F905F904F903F902F900895C501EF
:10B490000F948BA0D8018D939C93B5E0CB0ED11C5B
:10B4A000E2E0AE0EB11C96CC0F931F93CF93209188
:10B4B0009412213079F58C0180E50E94B6558823DD
:10B4C00049F10E94CB55C82F853020F5013C82E020
:10B4D000180749F0023C124069F08C2FCF911F9160
:10B4E0000F910D944C6B60E08C2FCF911F910F91B9
:10B4F0000D948F6B8EEC9EE00F947DA0882351F00D
:10B500000F945554882331F08C2FCF911F910F91B8
:10B510000D940C6CCF911F910F9108958F929F9273
:10B52000AF92BF92CF92DF92EF92FF920F931F9351
:10B53000CF93DF930091F5161091F6160F5F1F4F12
:10B5400068018FEFC81AD80AD801DC918D2F90E0DE
:10B550000F940E9E7C01892B01F5DD3201F5680107
:10B56000B2E0CB0ED11CF801D181C1E086010150BF
:10B57000110943E050E06AEF76E7C8010F94449E5A
:10B58000892BC1F460E070E080E89FEFC111DBC05F
:10B5900060E070E080E89FE7D6C08601D1CFDB3263
:10B5A00039F46801F2E0CF0ED11CD8011196DC917C
:10B5B000C0E0DCCF43E050E067EF76E7C8010F94CE
:10B5C000449E892B09F4CCC0F60110E000E020E095
:10B5D00030E0A9016F01D053DA3060F5BC2E6894D9
:10B5E000B1F88C2F8870C2FF09C0811102C00F5FB3
:10B5F0001F4F3196D601DC91CB2DECCF882311F073
:10B6000001501109A5E0B0E00F9412A19B01AC011B
:10B61000220F331F441F551F2D0F311D411D511D7A
:10B620002839B9E93B074B07B9E15B0710F3C6605E
:10B63000BC2EDFCFDE3F31F4C3FD33C0BC2E689497
:10B64000B3F8D7CFD53369F580818D3231F4C0613D
:10B65000BF016E5F7F4F818105C0BF018B32C9F38F
:10B660006F5F7F4F80538A30E0F4FB01B0E8EB1648
:10B67000BCE0FB065CF4B701660F771F660F771F0F
:10B68000E60EF71EEE0CFF1CE80EF11C81918053B4
:10B690008A3060F3C4FF03C0F194E194F1080E0D09
:10B6A0001F1DCA01B9010F94099BC370C33009F46F
:10B6B00090584B015C0120E030E0A9010F949AA260
:10B6C000882309F43EC0C3EFD6E717FF05C01195E4
:10B6D00001951109CBEDD6E76E01E8E1CE1AD1084C
:10B6E00080E2E82EF12C0DC0FE01259135914591A7
:10B6F00054910E191F09C501B4010F944A9B4B01C7
:10B700005C01D501C4010E151F0574F72497F5944B
:10B71000E794CC16DD06A9F78A2F880F8B2F881F98
:10B720008F3F49F020E030E0A901C501B4010F943A
:10B730009AA2811106C082E290E09093F91680935C
:10B74000F816C501B401DF91CF911F910F91FF90C1
:10B75000EF90DF90CF90BF90AF909F908F90089523
:10B7600060E070E080EC9FE7EECF2F923F924F9227
:10B770005F926F927F928F929F92AF92BF92CF9281
:10B78000DF92EF92FF920F931F93CF93DF93CDB78A
:10B79000DEB7A1970FB6F894DEBF0FBECDBF84EC25
:10B7A00092E09D8F8C8F85EF282E81E1382E03E962
:10B7B00016E091E09A8F198EEC8DFD8D8191FD8FB1
:10B7C000EC8F0E94B655E82E882309F454C1F090FE
:10B7D000EB11FA8DFF220E948E5A2B013C01F801D9
:10B7E0004082518262827382F98DF33009F045C044
:10B7F000DD24D394F11001C0D12C809010029090E0
:10B800001102A0901202B090130220E030E040E854
:10B810005FE3C501B4010F949AA2882359F1F11096
:10B8200015C02091011230910212409103125091E3
:10B830000412C301B2010F94A4A160939F067093F8
:10B84000A0068093A1069093A206DE2CA501940188
:10B8500060919F067091A0068091A1069091A2062A
:10B860000F944A9B60939F067093A0068093A10655
:10B870009093A206D11003C05FC0FF2089F0F101B0
:10B880002081318142815381F801608171818281FF
:10B8900093810F94A5A1F8016083718382839383C0
:10B8A000F98DF230D9F580918903823009F0EEC02C
:10B8B0008CE0E0EAF2E0DE011D9601900D928A959F
:10B8C000E1F78CE0ECEAF2E0DE01119601900D92D6
:10B8D0008A95E1F7C0909B06D0909C06E0909D066B
:10B8E000F0909E0620E030E0A901C701B6010F9458
:10B8F0009AA287FF52C0CE0101967C01D12CF7019C
:10B9000061917191819191917F010F9416A38D2D79
:10B910000F946121D394F3E0DF12F1CFF98DFF5F33
:10B92000F98F8A8D880F8A8F94E0290E311C0C5F65
:10B930001F4FF43009F040CF86E40E94B6558823AB
:10B9400099F00E948E5A6B017C0120E030E0A90141
:10B950000F942EA4181644F4C0927A02D0927B025F
:10B96000E0927C02F0927D02A1960FB6F894DEBFC1
:10B970000FBECDBFDF91CF911F910F91FF90EF9040
:10B98000DF90CF90BF90AF909F908F907F906F90FF
:10B990005F904F903F902F90089520E030E048E472
:10B9A00053E4C701B6010F942EA41816A4F4CE01D7
:10B9B0000D967C01D12CF70161917191819191914A
:10B9C0007F010F9416A38D2D0F946121D394F3E082
:10B9D000DF12F1CFA3CFCE01019699A388A3FE0178
:10B9E0003D96FF8FEE8F1B8EE8A1F9A1C190D190FB
:10B9F000E190F190F9A3E8A3EE8DFF8D6191719133
:10BA000081919191FF8FEE8FA70196010F94A4A1D0
:10BA100020E030E048E453E40F94A4A24B015C0121
:10BA200020919B0630919C0640919D0650919E0668
:10BA30000F944A9B2B013C0120E030E0A901C50195
:10BA4000B4010F944A9B9B01AC01C701B6010F944E
:10BA5000A4A19B01AC01C301B2010F94A5A10F9455
:10BA600016A38B8D0F946121FB8DFF5FFB8FF3304D
:10BA700009F0BACF53CFF10180819181A281B381C6
:10BA8000F80180839183A283B38348CFEA8DEE0FC0
:10BA9000EA8FF4E02F0E311C0C5F1F4F83E0898F7B
:10BAA0008BCE609100177091011790E08A3020F0E2
:10BAB000895A9F4F0D94E59EC096FCCF2FB784FF07
:10BAC0001EC0F894909105019260909305012FBFDC
:10BAD0002FB785FF19C0F89490910501916090935C
:10BAE00005012FBF86FF15C0459A87FF14C0469AEF
:10BAF000739A85E08A95F1F7000073980895F89499
:10BB0000909105019D7FE1CFF894909105019E7F72
:10BB1000E6CF4598EACF4698EBCF0F931F93CF938C
:10BB2000DF93C82FD62F8A0160FF15C05F9A8AE184
:10BB30008A95F1F700C08C2F0E945E5DD1FD04C094
:10BB40008C2F82950E945E5DC801DF91CF911F917D
:10BB50000F910C94D9BF5F98EACFCF92DF92EF920A
:10BB6000FF92CF93DF93EC016A017B010F9485A0D4
:10BB70006F3F7F4F8F4F9F4F59F4B701A601CE0102
:10BB8000DF91CF91FF90EF90DF90CF900D94D3A0F5
:10BB9000DF91CF91FF90EF90DF90CF9008957F924B
:10BBA0008F929F92AF92BF92CF92DF92EF92FF92CD
:10BBB0000F931F93CF93DF93CDB7DEB760970FB688
:10BBC000F894DEBF0FBECDBF5C016B01742E81E027
:10BBD000809378021F930F931F922F938FE394E625
:10BBE0009F938F930F943F9F81E40E94B6550F90CF
:10BBF0000F900F900F900F900F90882389F08091F5
:10BC0000F5169091F616FC012181283709F056C0EF
:10BC100040E150E070E060E002960F94089C5B0108
:10BC200083E40E94B655882309F44DC00E941E5635
:10BC30004B017501CA14DB0408F47601C4018E0DB2
:10BC40009F1DC816D90618F08E159F0518F44601D9
:10BC50008E189F0888E50E94B655882309F471C0A4
:10BC60002091F5163091F6162F5F3F4FCE010196C9
:10BC70005C01DC01D12CC12CF90180812F5F3F4F89
:10BC80008823B9F190E1C916D10499F18032A1F36A
:10BC90008A3079F190ED980F9A30C8F48295807FC0
:10BCA0009F012E5F3F4F918140ED490F4A30B8F41C
:10BCB000842B8D93EFEFCE1ADE0ADECF0E948E5AD0
:10BCC0000F9416A3ACCF88248A94982CB2CF9FE906
:10BCD000980F963058F48295807F8057E1CF4FE9D6
:10BCE000490F463018F49755892BE3CFD194C1946E
:10BCF000D108912C812CC814D90491F0F5016191DF
:10BD00005F01C4018E0D9F1DF1E07F1631F0FC0133
:10BD10006083FFEF8F1A9F0AEECF0F94C5A0F9CF73
:10BD2000FF92EF921F930F939F928F9285E194E67B
:10BD30009F938F930F943F9F0FB6F894DEBF0FBE73
:10BD4000CDBF472DB401C70160960FB6F894DEBF92
:10BD50000FBECDBFDF91CF911F910F91FF90EF905C
:10BD6000DF90CF90BF90AF909F908F907F900D9479
:10BD7000835280E1E5EFF1E1A0E9B2E001900D929C
:10BD80008A95E1F780918E0290918F029093F41141
:10BD90008093F3118091F1119091F2119093F01131
:10BDA0008093EF118091ED118093EC118091EB1154
:10BDB00083FB882780F98093EA118091E9118093B1
:10BDC000E8110895CF93DF938AEF95E10E94C67042
:10BDD00088E394E1892B51F0CAE0D5E1A397CE0125
:10BDE0000E94C67084E1C833D807C1F785E194E1A9
:10BDF0000E94C67080EF93E1DF91CF910C94C670E2
:10BE0000CF93DF93C5EFD1E120E030E048EC51E47F
:10BE10006C857D858E859F850F94A5A16C877D8718
:10BE20008E879F8763E373E383E590E4DF91CF918F
:10BE30000D94118560E085EA9FE00F94A1A060E079
:10BE40008FE79CE00F94A1A080E090E0A0E8BFEB1A
:10BE500080937E0290937F02A0938002B093810230
:10BE600082E0809379021092E71108958091EF119A
:10BE70009091F0112091F1113091F21128173907AA
:10BE800071F09093F2118093F11181E08093990306
:10BE90000F94460F0F94364E82E0809399030895D5
:10BEA0008091E711882341F080918E0290918F025A
:10BEB0009093F4118093F3110895CF92DF92EF9253
:10BEC000FF92C090CA04D090CB04E090CC04F090D4
:10BED000CD048091C904882309F44EC020E030E0ED
:10BEE000A901C701B6010F942EA418160CF044C086
:10BEF0002BED3FE049E450E4C701B6010F944A9BA3
:10BF0000A70196010F944A9B20E030E040E85EE3F1
:10BF10000F944A9B9B01AC0160E070E080E89FE3D6
:10BF20000F94A4A26B017C016091590270915A0296
:10BF300064367105A1F0072E000C880B990B0F9445
:10BF40000B9B2AE037ED43E25CE30F944A9B9B0195
:10BF5000AC01C701B6010F944A9B6B017C01C092F2
:10BF60001002D0921102E0921202F0921302FF909E
:10BF7000EF90DF90CF900895C12CD12C80E8E82E6F
:10BF80008FE3F82ED1CF8F929F92AF92BF92CF9234
:10BF9000DF92EF92FF9281EF9FE00F9455486B0183
:10BFA0007C018DEE9FE00F9455484B015C010F948E
:10BFB000381C2CE330E040E050E00F94F0A0BA01D0
:10BFC000A901480D591D6A1D7B1D8DEE9FE00F9440
:10BFD000B3A0609184067091850680918606909149
:10BFE000870628EE33E040E050E00F94F0A0BA015D
:10BFF000A9014C0D5D1D6E1D7F1D81EF9FE00F940B
:10C00000B3A00F940D201092840610928506109212
:10C0100086061092870680919412813081F4609197
:10C0200098127091991290E080E00F943D48109220
:10C0300099121092981210929B1210929A12FF90DD
:10C04000EF90DF90CF90BF90AF909F908F9008952A
:10C050008091E9111F928F93809140031F928F93DB
:10C06000E5E8F3E0428153812CE3249FC001259F42
:10C07000900D11249F938F9340815181249FC00183
:10C08000259F900D11249F938F9386ED94E69F93A7
:10C090008F930F943F9F8DB79EB70A960FB6F89473
:10C0A0009EBF0FBE8DBF08958AE493E00D94731177
:10C0B00020E030E040E752E40F94A4A208951092EB
:10C0C000770240913B0350913C0360913D03709196
:10C0D0003E0340937A0250937B0260937C027093FC
:10C0E0007D0290938F0280938E028AE493E00D94F8
:10C0F00073111F93CF93DF93182F80917A02909141
:10C100007B02A0917C02B0917D0280933B039093CF
:10C110003C03A0933D03B0933E03C0918E02D091A7
:10C120008F0284E690E090938F0280938E028AE4DF
:10C1300093E00F94731110937702CE01DF91CF91AA
:10C140001F910895CF92DF92EF92FF920F931F936A
:10C15000CF93DF9390E0EC01CC0FDD1FCC0FDD1F00
:10C16000FE01EB5EF8482591359145915491FE0111
:10C17000E657FB4FC080D180E280F3808E010B50E8
:10C180001E4EC701B6010F94A5A1F801608371830B
:10C1900082839383FE01E75FF848259135914591AD
:10C1A00054918E010C5D1D4FC701B6010F94A5A1DE
:10C1B000F8016083718382839383FE01E350F94821
:10C1C0002591359145915491C85EDD4FC701B60167
:10C1D0000F94A5A1688379838A839B83DF91CF9194
:10C1E0001F910F91FF90EF90DF90CF90089540E066
:10C1F00050E0BA018DEE9FE00F94B3A040E050E014
:10C20000BA0181EF9FE00F94B3A00E94295670E01D
:10C2100060E085E09FE00F94BFA070E060E083E005
:10C220009FE00F94BFA070E060E081E09FE00F947A
:10C23000BFA070E060E08FEF9EE00F94BFA070E0C1
:10C2400060E083ED9EE00F94BFA070E060E080EDC1
:10C250009EE00F94BFA040E050E0BA0188EA9CE065
:10C260000D94B3A0F89488E19FE00FB6F894A895D8
:10C27000809360000FBE90936000FFCF85EA9FE03F
:10C280000F947DA091E0811101C090E0892F089565
:10C2900080919B03811106C081E0909159039230F7
:10C2A00009F080E0089580916A1381110AC080919D
:10C2B000D511811106C081E090915903913009F0A8
:10C2C00080E00895CF93DF93C0910512C1111FC084
:10C2D0008091061281111CC00E944861811118C012
:10C2E000D091C80DD43061F48091F1119091F21188
:10C2F000892B91F48091ED119091EE11892B61F4CD
:10C300000E945361C82F811103C0C1E0D111C0E068
:10C310008C2FDF91CF910895C1E0FACF0E94626126
:10C32000882389F020E030E040E050E46091FD1186
:10C330007091FE118091FF11909100120F949AA2BA
:10C34000881F8827881F08950E945361811118C093
:10C350000E944861811114C08091E711811110C0C1
:10C360008091C80D81110BC080919512811107C079
:10C3700080910512811104C080910612089581E018
:10C38000089580E1E5EFF1E1A3E9B6E001900D92B7
:10C390008A95E1F708954F925F926F927F928F9204
:10C3A0009F92AF92BF92CF92DF92EF92FF920F9344
:10C3B0001F93CF93DF9300D000D01F921F92CDB771
:10C3C000DEB72091E711222309F473C120919C0369
:10C3D000223009F46EC120919C03213011F4109297
:10C3E0009C032B013C011092E9111091EC1160911A
:10C3F0008A0370918B0380918C0390918D030F942D
:10C400001DA3611731F0812F90E09093EE1180937E
:10C41000ED110E94365F8091E8118093E9119091AF
:10C42000EB118091EA118195892788708927809383
:10C43000EB11A301920160919C0270919D02809189
:10C440009E0290919F020F94A4A16D837E838F839F
:10C450009887CE0105960F9469751092400220E0EE
:10C4600030E040E85FEB6091900270919102809122
:10C470009202909193020F949AA2811120C0809110
:10C48000F5119091F611A091F711B091F8118093E8
:10C49000900290939102A0939202B09393028091A4
:10C4A000F9119091FA11A091FB11B091FC118093B8
:10C4B000940290939502A0939602B0939702A301E1
:10C4C000920160919C0270919D0280919E029091D8
:10C4D0009F020F94A4A169837A838B839C83E0904D
:10C4E000FD11F090FE110091FF11109100122091AA
:10C4F000940230919502409196025091970260917A
:10C5000090027091910280919202909193021F92F9
:10C510001F921F921F92E2E68E2EE7E29E2EE6E722
:10C52000AE2EE2E4BE2EFE0131966F010F94C3756C
:10C53000A301920160919C0270919D0280919E02E4
:10C5400090919F020F94A4A169837A838B839C832B
:10C55000E0909802F090990200919A0210919B024B
:10C560002091940230919502409196025091970249
:10C570006091900270919102809192029091930249
:10C580001F921F921F921F920F94C375E090980202
:10C59000F090990200919A0210919B0220919402CE
:10C5A00030919502409196025091970260919002CD
:10C5B0007091910280919202909193021F921F922A
:10C5C0001F921F92812C912CF8EEAF2EF2E4BF2E19
:10C5D000ACE9CA2EA2E0DA2E0F94C3750F94142290
:10C5E00011E0109340026091E2117091E31190E02C
:10C5F00080E00F94099B60937A0270937B02809392
:10C600007C0290937D028091F3119091F4119093AC
:10C610008F0280938E0280E1E0E9F2E0A5EFB1E1C4
:10C6200001900D928A95E1F70E94C1618091790293
:10C630000FB6F894DEBF0FBECDBF811151C060911F
:10C64000D8117091D9118091DA119091DB1160931A
:10C650007E1670937F1680938016909381160F94A8
:10C6600094438091D8119091D911A091DA11B09191
:10C67000DB118093DC119093DD11A093DE11B09358
:10C68000DF1110936A1360E085EA9FE00F94A1A088
:10C6900060E08FE79CE00F94A1A08BE09CE60E94F5
:10C6A0005FE682E0809379021092E71181E0809347
:10C6B000AC0D28960FB6F894DEBF0FBECDBFDF914C
:10C6C000CF911F910F91FF90EF90DF90CF90BF908F
:10C6D000AF909F908F907F906F905F904F90089554
:10C6E000813089F68091D8119091D911A091DA11F9
:10C6F000B091DB118093D1119093D211A093D311FB
:10C70000B093D4111092DB0F1092DA0F0E946D5586
:10C71000BACF3F924F925F926F927F928F929F9289
:10C72000AF92BF92CF92DF92EF92FF920F931F933F
:10C73000CF93DF933090DC16332009F480C08B0157
:10C74000EC0131FE54C088809980AA80BB80FB0137
:10C75000C080D180E280F3802091B1163091B21672
:10C760004091B3165091B416C501B4010F944A9B81
:10C770002B013C012091B5163091B6164091B716A9
:10C780005091B816C701B6010F944A9B9B01AC01AA
:10C79000C301B2010F94A5A12B013C012091A91660
:10C7A0003091AA164091AB165091AC16C501B40158
:10C7B0000F944A9B4B015C012091AD163091AE164F
:10C7C0004091AF165091B016C701B6010F944A9B25
:10C7D0009B01AC01C501B4010F94A5A168837983C5
:10C7E0008A839B83F801408251826282738230FE89
:10C7F00026C02091D4163091D5164091D61650916E
:10C80000D716688179818A819B810F94A5A168835D
:10C8100079838A839B832091D8163091D9164091D1
:10C82000DA165091DB16F801608171818281938163
:10C830000F94A5A1F8016083718382839383DF91B4
:10C84000CF911F910F91FF90EF90DF90CF90BF900D
:10C85000AF909F908F907F906F905F904F903F90A0
:10C8600008952F923F924F925F926F927F928F9294
:10C870009F92AF92BF92CF92DF92EF92FF920F936F
:10C880001F93CF93DF9300D000D01F921F92CDB79C
:10C89000DEB78C011B01FC0180819181A281B381F3
:10C8A00089839A83AB83BC83FB0180819181A281C0
:10C8B000B3818D839E83AF83B887BE016B5F7F4F4B
:10C8C000CE0101960E948963C980DA80EB80FC80EA
:10C8D00020E030E0A901C701B6010F949AA287FFBA
:10C8E00035C019821A821B821C82FF24F3948D802A
:10C8F0009E80AF80B88420E030E040E850ECC50175
:10C90000B4010F949AA287FF35C080E090E0A0E8C0
:10C91000B0EC8D839E83AF83B887CD80DE80EF80BF
:10C92000F88489809A80AB80BC807090DC1671108E
:10C930004CC0F80180829182A282B382F101C08250
:10C94000D182E282F382FF24F39425C020E030E01C
:10C950004AE753E4C701B6010F942EA4F12C181630
:10C9600034F680E090E0AAE7B3E489839A83AB834E
:10C97000BC83BBCF20E030E042E553E4C501B40105
:10C980000F942EA418162CF480E090E0A2E5B3E4F6
:10C99000C0CFF110C2CF8F2D28960FB6F894DEBF0E
:10C9A0000FBECDBFDF91CF911F910F91FF90EF9000
:10C9B000DF90CF90BF90AF909F908F907F906F90BF
:10C9C0005F904F903F902F90089570FE1CC0209173
:10C9D000D4163091D5164091D6165091D716C50170
:10C9E000B4010F94A4A14B015C012091D8163091A1
:10C9F000D9164091DA165091DB16C701B6010F9493
:10CA0000A4A16B017C0171FE9ECF2091C4163091D0
:10CA1000C5164091C6165091C716C501B4010F94B2
:10CA20004A9B2B013C012091C8163091C9164091B8
:10CA3000CA165091CB16C701B6010F944A9B9B01B1
:10CA4000AC01C301B2010F94A5A1F8016083718309
:10CA5000828393832091CC163091CD164091CE16CF
:10CA60005091CF16C501B4010F944A9B4B015C0154
:10CA70002091D0163091D1164091D2165091D316F4
:10CA8000C701B6010F944A9B9B01AC01C501B401DB
:10CA90000F94A5A1F101608371838283938353CFA7
:10CAA000CF92DF92EF92FF92CF93DF93EC01BC0124
:10CAB0006C5F7F4F0E943164C0902C02D0902D0299
:10CAC000E0902E02F0902F02A701960168857985EB
:10CAD0008A859B850F949AA287FF04C0C886D98651
:10CAE000EA86FB86C0902002D0902102E0902202CC
:10CAF000F0902302A7019601688579858A859B8538
:10CB00000F942EA4181624F4C886D986EA86FB86CC
:10CB1000DF91CF91FF90EF90DF90CF9008952F920B
:10CB20003F924F925F926F927F928F929F92AF92BD
:10CB3000BF92CF92DF92EF92FF920F931F93CF930A
:10CB4000DF93CDB7DEB7A2970FB6F894DEBF0FBE66
:10CB5000CDBF1C0183E996E00E9450658AE493E012
:10CB60000F9473114090F5115090F6116090F711E9
:10CB70007090F811C0909306D0909406E0909506BE
:10CB8000F0909606A7019601C301B2010F949AA2F4
:10CB900081113FC0209197063091980640919906E7
:10CBA00050919A066091F9117091FA118091FB11E0
:10CBB0009091FC110F949AA281112BC020E030E0DB
:10CBC00040E752E460917A0270917B0280917C028E
:10CBD00090917D020F94A4A20F94DE840E94375599
:10CBE000A2960FB6F894DEBF0FBECDBFDF91CF91F6
:10CBF0001F910F91FF90EF90DF90CF90BF90AF907B
:10CC00009F908F907F906F905F904F903F902F906C
:10CC1000089560918E0270918F02072E000C880B90
:10CC2000990B0F940B9B20917A0230917B024091DB
:10CC30007C0250917D020F944A9B2EE333EC4EE22E
:10CC400059E30F944A9B6F83788789879A878091ED
:10CC50009C12882309F40FC1A3019201C701B601F8
:10CC60000F94A4A12B013C012091F9113091FA11EC
:10CC70004091FB115091FC116091970670919806BC
:10CC80008091990690919A060F94A4A16B877C8756
:10CC90008D879E87C301B2019F772B853C854D858B
:10CCA0005E855F770F94A5A16B017C0120E030E0E9
:10CCB000A9010F942EA418160CF0DDC020E030E07E
:10CCC00040EF51E4C701B6010F94A4A20F9483A2D0
:10CCD0000F941DA37E836D836230710508F4CBC071
:10CCE0002114310409F4C7C02091FD113091FE11C7
:10CCF0004091FF115091001260919B0670919C062B
:10CD000080919D0690919E060F94A4A16F87788BC9
:10CD1000898B9A8B2091011230910212409103125B
:10CD20005091041260919F067091A0068091A10617
:10CD30009091A2060F94A4A16B8B7C8B8D8B9E8B04
:10CD4000AD81BE81CD01B0E0A0E08F8F98A3A9A3F3
:10CD5000BAA32D813E812216330608F08CC0B101A2
:10CD600090E080E00F94099B6B017C016F8D78A1AE
:10CD700089A19AA10F94099B9B01AC01C701B6013F
:10CD80000F94A4A26B017C01AC019B016B897C898F
:10CD90008D899E890F944A9B9B01AC016091011281
:10CDA0007091021280910312909104120F94A5A128
:10CDB00069837A838B839C83A70196016F85788929
:10CDC00089899A890F944A9B2091FD113091FE1117
:10CDD0004091FF11509100120F94A5A16F8B788F95
:10CDE000898F9A8FA70196016B857C858D859E859D
:10CDF0000F944A9B2091F9113091FA114091FB1147
:10CE00005091FC110F94A5A16B8F7C8F8D8F9E8FFD
:10CE1000A7019601C301B2010F944A9B2091F5111D
:10CE20003091F6114091F7115091F8110F94A5A18E
:10CE30003F922F92A5EFB1E1BF93AF938F8098847B
:10CE4000A984BA84DE0111966D01EF88F88C098DF2
:10CE50001A8D2B8D3C8D4D8D5E8D0F94C3750F906B
:10CE60000F900F900F908091AC0D8111B7CEBFEF56
:10CE70002B1A3B0A6ECFE0909B06F0909C06009127
:10CE80009D0610919E06209197063091980640913C
:10CE9000990650919A06609193067091940680913C
:10CEA0009506909196061F921F92E5EFF1E1FF9390
:10CEB000EF938F809884A984BA84EFE9CE2EE6E0C0
:10CEC000DE2E0F94C3750F900F900F900F9086CEAB
:10CED000CF92DF92EF92FF92CF93C090FD11D0904E
:10CEE000FE11E090FF11F0900012A70196010F943F
:10CEF000A5A16093FD117093FE118093FF11909393
:10CF0000001283B19091A506911102C084FF26C042
:10CF100085EF91E10E94506560914E0470914F043D
:10CF200080915004909151040F9411850F94142214
:10CF3000A70196016091FD117091FE118091FF1182
:10CF4000909100120F94A4A16B017C01C701B6015E
:10CF5000CF91FF90EF90DF90CF90089515980F94A8
:10CF6000142281E00F944C2CC82F65E575E585E50A
:10CF700091E40F9411850F94142282E00F94002203
:10CF8000A70196010F94A4A16B017C018C2F0F9433
:10CF90004C2CDCCF8F929F92AF92BF92CF92DF92B8
:10CFA000EF92FF924B015C01C090FD11D090FE11F9
:10CFB000E090FF11F0900012AC019B01C701B60197
:10CFC0000F942EA487FF11C0A5019401C701B601DB
:10CFD0000F94A4A19F77FF90EF90DF90CF90BF9028
:10CFE000AF909F908F900C946867FF90EF90DF90C8
:10CFF000CF90BF90AF909F908F9008952F923F92C7
:10D000004F925F926F927F928F929F92AF92BF9258
:10D01000CF92DF92EF92FF920F931F93CF93DF9304
:10D0200000D01F921F92CDB7DEB7D82E2A013B0148
:10D03000322EE982FA820B831C830F94142281E042
:10D0400080930512FC2CE32CD31010C0ED2CDC10C7
:10D050000DC060E070E080EA90E40E94CA67FF249F
:10D06000F394EE24E3942224239401C02D2C0F94F6
:10D07000FD8F80919C128D8310929C1282E00F9400
:10D0800000226093FD117093FE118093FF11909325
:10D090000012F1100F94AC8B81E00E9479608C013A
:10D0A0000E94C16110927A0210927B0210927C025F
:10D0B00010927D02222019F080E00F945D54EE2042
:10D0C00019F081E00F945D54DD20E9F04114510422
:10D0D00061047104C1F0C301B2010F940B9B9B0169
:10D0E000AC0160918A0470918B0480918C049091C2
:10D0F0008D040F94A5A16093F5117093F6118093A0
:10D10000F7119093F811332001F189819A81AB8155
:10D11000BC810097A105B105C1F0BC01CD010F9400
:10D120000B9B9B01AC0160918E0470918F048091E8
:10D130009004909191040F94A5A16093F9117093BC
:10D14000FA118093FB119093FC11FF2009F499C010
:10D1500060E070E080EA90E40E94CA678091A306D4
:10D16000811102C00F945D548091A406811103C007
:10D1700081E00F945D540F946290E3E5F9E88591A6
:10D180009591A591B491EFE4F9E845915591659198
:10D190007491409393065093940660939506709310
:10D1A00096068093970690939806A0939906B0935D
:10D1B0009A0667E976E083E996E00E9489630F9416
:10D1C000C48F20E030E040E850EC60919706709109
:10D1D00098068091990690919A060F949AA287FFDB
:10D1E0000CC080E090E0A0E8B0EC809397069093AC
:10D1F0009806A0939906B0939A0680E090E0A6E185
:10D20000B3E480937A0290937B02A0937C02B09364
:10D210007D02109277020F94D18360917A0270910F
:10D220007B0280917C0290917D020F94DE840F94AA
:10D2300014228091930690919406A0919506B09146
:10D2400096068093F5119093F611A093F711B09381
:10D25000F8118091970690919806A0919906B09147
:10D260009A068093F9119093FA11A093FB11B09351
:10D27000FC1181E0809377020F94682C82E00F9478
:10D280005D54CC20E9F081149104A104B104C1F0F3
:10D29000C501B4010F940B9B9B01AC0160919204FA
:10D2A0007091930480919404909195040F94A5A19A
:10D2B0006093FD117093FE118093FF119093001203
:10D2C0000F94D183C8010E945F600F94682C0F9463
:10D2D00062900F94008ED11007C0311005C08B8D65
:10D2E000811102C0CC2039F1F11025C09D81992314
:10D2F00011F181E080939C120F9400226B017C015C
:10D3000080E00F940022A70196010F94A9609B0171
:10D31000AC016091FD117091FE118091FF1190910F
:10D3200000120F94A4A16093FD117093FE118093DD
:10D33000FF119093001284E10F94A0980F9414228F
:10D34000109205120F900F900F900F900F90DF9199
:10D35000CF911F910F91FF90EF90DF90CF90BF90F2
:10D36000AF909F908F907F906F905F904F903F9085
:10D370002F900895E3E3F3E09FE781918F3731F039
:10D38000DF01119787FF07C08F778C9383E0EB3322
:10D39000F80799F708959C93F9CF90915B0298173D
:10D3A00010F480935B0280915C02882339F0E09155
:10D3B000D203F091D303309709F019940895CF93D5
:10D3C000DF93CDB7DEB7AE014A5F5F4FFA016191DF
:10D3D0007191AF0180EC93E00F94C49FDF91CF91E6
:10D3E000089560EC73E00D94159F60EC73E0082ED7
:10D3F000000C990B0D94E59ECF93C82FC15020F0DF
:10D4000080E20E94F569FACFCF910895CF93C82F9B
:10D41000862F643008F083E0809332030E944155E8
:10D420008C0F8093310344E650E060E08068CF9138
:10D430000C948D5DCF93DF93EA010E94066A60EC45
:10D4400073E0CE01DF91CF910D94159FCF93C42F40
:10D450000E94066A60EC73E08C2FCC0F990BCF9181
:10D460000D94E59E60E080E00E94066A1092310310
:10D47000089540E456E060E081E00E948D5D1092E6
:10D4800032031092310348E050E06FE770E083E32D
:10D4900093E00D94AFA690915C02981709F18093E8
:10D4A0005C028823E9F0109207051092060510929D
:10D4B000110681EB93E00F9473110F94460F6150A6
:10D4C0007109810991096093930370939403809388
:10D4D0009503909396030E94396A82E00C94CD697B
:10D4E0000895CF93C82F109232031092310348E071
:10D4F00050E06FE770E083E393E00F94AFA644E958
:10D5000051E162E080E30E948D5D46E950E062E017
:10D5100080E30E948D5D46E950E062E080E30E9476
:10D520008D5D46E950E062E080E20E948D5D809171
:10D53000CE0344E650E060E080620E948D5D84E0AE
:10D540008093300344E650E060E08CE00E948D5D03
:10D55000C1110E94396A44E650E060E086E0CF9154
:10D560000C948D5D81E00C94716ACF92DF92FF92F2
:10D570000F931F93CF93DF9300D000D01F921F9281
:10D58000CDB7DEB78A30D9F480913203843018F0F9
:10D590008FEF80933203609132036F5F80E00E94CF
:10D5A000066A28960FB6F894DEBF0FBECDBFDF9196
:10D5B000CF911F910F91FF90DF90CF90089590E849
:10D5C000980F44E650E061E09A3408F5482F40583F
:10D5D000550B9A0196E0929FA001939F500D112444
:10D5E000FA01E45FFA48F490E3E3F3E030E020E08E
:10D5F0009FEF6191782F76277F7789F4F901ED5CB1
:10D60000FC4F8083F22E44E650E061E08F2D0E94B3
:10D610008D5D809131038F5F80933103C2CF6F376F
:10D6200009F03CC0F901ED5CFC4F8083922FF92E8C
:10D63000FA01E95FFA488E010F5F1F4FD8019591FB
:10D6400088E0182E10FE05900294802D9795881F73
:10D650008D931A94B9F7BF2DE8E0BE02C0011124E2
:10D6600044E650E060E080640E948D5D6E01F9E068
:10D67000CF0ED11C44E650E061E0D8018D918D01C0
:10D680000E948D5DC016D106A9F78091310344E652
:10D6900050E060E080680E948D5DB5CF67FF922FFB
:10D6A0002F5F3F4F2830310509F0A3CF9F3F09F08E
:10D6B000BECFA9CF8F929F92AF92BF92EF92FF926F
:10D6C0000F931F93CF93DF93CDB7DEB7A0970FB61D
:10D6D000F894DEBF0FBECDBF6115710581059105C0
:10D6E00099F480E3A0960FB6F894DEBF0FBECDBFCD
:10D6F000DF91CF911F910F91FF90EF90BF90AF906E
:10D700009F908F900C94B56A00E0842E912CB12CE0
:10D71000A12C9E012F5F3F4F7901A50194010F9429
:10D72000F0A0F701E00FF11D6083B901CA010F5F9E
:10D73000611571058105910581F70E0D1F2D111DD4
:10D74000E016F10659F0F80182918F018A3020F439
:10D75000805D0E94B56AF4CF895CFBCFA0960FB6BE
:10D76000F894DEBF0FBECDBFDF91CF911F910F9117
:10D77000FF90EF90BF90AF909F908F900895CF92C1
:10D78000DF92EF92FF926B017C01F7FE0BC08DE2FE
:10D790000E94B56AF094E094D094C094C11CD11C4E
:10D7A000E11CF11C4AE0C701B601FF90EF90DF9049
:10D7B000CF900C945A6B0F931F93CF938C01C62F6D
:10D7C000CC2359F0F8012491222339F00F5F1F4F29
:10D7D00084910E94B56AC150F3CF8C2F0E94FC69DE
:10D7E0008C2FCF911F910F9108950F931F93CF937B
:10D7F0008C01C62FCC2349F0F80181918F01882339
:10D8000021F00E94B56AC150F5CF8C2F0E94FC69AF
:10D810008C2FCF911F910F910895CF93DF93EC013F
:10D820008991882319F00E94B56AFACFDF91CF91D0
:10D8300008950E94B56A90E080E008951092630315
:10D84000109214060895CF9380916303C1E0811173
:10D8500004C0C0E08C2FCF9108950E941E6CFACFB7
:10D860008EEF9FE00F947DA08E3F39F091E02091E4
:10D870002F03281390E0892F089580E008951092D7
:10D880002F036EEF8EEF9FE00D94A1A0853728E661
:10D89000920709F459C0F8F48E3625E6920709F488
:10D8A00059C050F4833723E69207B1F18536944688
:10D8B000B1F184E594E60895823726E6920791F166
:10D8C000823728E6920709F442C08337954689F7E4
:10D8D0008BEA94E608958C3620E7920731F170F4D4
:10D8E0008C362EE6920721F18F362EE6920731F123
:10D8F00084379946F1F689E994E608958B3623E753
:10D900009207F9F0863723E79207A9F08F369247FE
:10D9100081F687E594E608958BEB94E6089583EB12
:10D9200094E6089582EA94E6089582E994E60895DB
:10D9300087E894E608958FE794E6089589E794E6EA
:10D9400008958EE694E6089587E694E608958EE5B8
:10D9500094E6089583EC94E60895E3E0F5E7859175
:10D960009591A591B4918F3F9F4FAF4FBF4FB1F0AD
:10D9700020E031E081E0F901459155916591749184
:10D98000453A5A45644B7B4409F00895F9013496B1
:10D9900045915491240F351F8F5FEDCF81E008959D
:10D9A0000F931F93811113C010922E0310922D0319
:10D9B00010922F0390912F0398135CC0682F8EEF65
:10D9C0009FE00F94A1A081E01F910F9108958130F5
:10D9D00089F7E0E0F1E04591559165917491453A00
:10D9E0005A45644B7B4431F7E4E0F1E0A591B491F2
:10D9F000E8E0F1E06591749150E040E030E020E033
:10DA0000A417B50729F5261B370B32272327322702
:10DA10006217730709F0CECFECE0F1E005911591A4
:10DA200025913491E3E0F5E7459155916591749125
:10DA3000041715072607370709F0BCCF20E031E0AF
:10DA400030932E0320932D0391E090932F03B2CFB8
:10DA5000FA01E050FF4FE491F0E098E040FD90E0E3
:10DA600002C0EE0FFF1F9A95E2F72E0F3F1F4F5F88
:10DA70005F4FC6CF80E0A8CF20912F03211104C0B3
:10DA8000FC013296CF01089540912D0350912E0351
:10DA900041155105A9F3FC01259134912F3F32071F
:10DAA00079F3F9013896EE0FFF1FE40FF51F25916A
:10DAB0003491FA01E20FF31F2491222309F3E2CFFC
:10DAC000CF93DF93EC0120E030E04CE852E460912A
:10DAD00001127091021280910312909104120F941E
:10DAE000A5A1609301127093021280930312909388
:10DAF000041260E070E080EA91E40F9411850E94C6
:10DB0000005F0E94396A84EC9AE50E943C6DAC018A
:10DB100060E080E00E941A6A8881882339F061E021
:10DB200080E00E94066ACE010E940D6C86EB99E3AC
:10DB30000E943C6DAC0162E080E00E941A6A83E4BE
:10DB40009BE20F94DD0BDF91CF910D9414220F9483
:10DB500030418F3F11F180E00E944B6A0E94396A88
:10DB600080E297E50E943C6DAC0161E080E00E949C
:10DB70001A6A80E20E94B56A0F943041682F70E003
:10DB80006F5F7F4F072E000C880B990B0E94BF6BB5
:10DB90000F94346B81E00C944B6A08951F920F929E
:10DBA0000FB60F9211240BB60F922F938F939F9362
:10DBB000EF93FF93E0912803E830E8F4F0E0882742
:10DBC000EB51F2498F4F0D948DA1ED6D076E126EE2
:10DBD000206E366E3F6E626E746E80919206811179
:10DBE0000AC080915B06880F80932703882319F071
:10DBF00081E080932803FF91EF919F918F912F9166
:10DC00000F900BBE0F900FBE0F901F901895809134
:10DC100026038F5F8093260390912703981758F36C
:10DC200082E0E7CF83E0809328038FE08093250391
:10DC30008FEF86BD81E085BD84B58F7E84BDDBCF4F
:10DC4000809125038295807F819588BD80912503F1
:10DC5000882321F0815080932503CDCF84E08093E9
:10DC600028038FEF88BD8EEF86BDC5CF85E08093FA
:10DC700028038FEF88BD86BD82E085BDBCCF2FEF26
:10DC800028BD809192068111B6CF809126038F5FC7
:10DC90008093260390912703891708F4ACCF8091D5
:10DCA0005B0690E08F3791050CF0A5CF86E080935E
:10DCB00028038FE08093250326BD81E085BD84B5D0
:10DCC0008061BCCF809125038295807F819588BD3E
:10DCD000809125038111BECF87E08093280380E8DF
:10DCE00086BD8FEF88BD87CF1092280380E886BD60
:10DCF0008FEF88BDC1CFCF93DF93EC0187E69FE024
:10DD00000F947DA091E0811101C090E081E0288115
:10DD1000211101C080E08913988387E09FE00F9470
:10DD20007DA091E0811101C090E0998385ED9EE096
:10DD30000F947DA091E0811101C090E09A8387E467
:10DD40009DE00F947DA08F3F21F08887DF91CF91D8
:10DD500008951886FBCFCF93C82F682F87E69FE0E2
:10DD60000F94A1A0CC2319F0CF910D94DC525198BF
:10DD7000599810928416CF910895109284030F94AD
:10DD8000460F60938D1670938E1680938F16909326
:10DD9000901608958093240380FD1CC010924003C8
:10DDA000209140038FEF820F8E3FE8F08091A0001A
:10DDB000877F8093A0001092AD001092AC009FB7B7
:10DDC000222361F0F8948091020180628093020125
:10DDD0009FBF08958FEF80934003E2CFF894809126
:10DDE00002018F7DF3CFEFB7F8948091A000886097
:10DDF0008093A00030E0809172004FEF50E081FFEF
:10DE000004C04091A8005091A900249FC001259F03
:10DE1000900D349F900D11246FEF70E00F9446A188
:10DE20007093AD006093AC00EFBF08951F93CF9344
:10DE3000DF93D0912403D1FD1DC010919A03C1E05E
:10DE400020E030E048E452E46091C40D7091C50DCB
:10DE50008091C60D9091C70D0F942EA418160CF04A
:10DE6000C0E0DE7FCD2B81E0111101C080E0C82B26
:10DE7000C093240380912403DF91CF911F910C94D0
:10DE8000CA6EEF92FF920F931F93CF93DF93EC0133
:10DE90008B017A010E949B5581110BC0A801BE0124
:10DEA000C701DF91CF911F910F91FF90EF900D94DB
:10DEB00091A0DF91CF911F910F91FF90EF90089566
:10DEC0000F931F93CF93DF938C01D62FC72F0F94FF
:10DED0008BA08F3F980739F46D2F7C2FC8010F94CA
:10DEE000DBA08D2F9C2FDF91CF911F910F91089573
:10DEF0000F931F93CF938C01C62F0F947DA08F3F5C
:10DF000029F46C2FC8010F94C5A08C2FCF911F91BD
:10DF10000F910895CF93DF93EC010F948BA0BC0178
:10DF20006F5F7F4FCE01DF91CF910D94DBA0CF9338
:10DF3000DF93EC010F947DA061E0680FCE01DF91CB
:10DF4000CF910D94C5A02BE0829FC0011124805B6E
:10DF5000924F0F948BA021E0019609F420E0822FCC
:10DF60000895CF93DF93C82FD8E0CF5FC8300CF06F
:10DF7000C0E08C2F0E94A36F811103C0D150A9F77C
:10DF8000CFEF8C2FDF91CF91089581EA9DE00F9420
:10DF90007DA00E94B16F87FD05C0682F81EA9DE0DA
:10DFA0000D94A1A008950F931F93CF93C82F8B01B9
:10DFB00066EB74E7823070F06FEA74E7843050F0FB
:10DFC00067EA74E7843031F06FE974E7853011F067
:10DFD00068E974E7C8010F94349E8CEF8C0F82308F
:10DFE00028F0C170CF5CF801C6831782CF911F91D2
:10DFF0000F91089561E080EC9FE00F94A1A060E094
:10E000008FEB9FE00F94A1A060E08EEB9FE00F9458
:10E01000A1A060E08DEB9FE00F94A1A060E08CEBED
:10E020009FE00D94A1A0CF93C82F82958F700E947E
:10E03000515D8C2F8F70CF910C94515D4091CF1119
:10E040005091D01190E080E041155105B1F120913F
:10E05000CB113091CC1190E080E0F901E252F04F09
:10E06000A081A23021F461817281860F971F4150F7
:10E07000510919F1F901EF51F04FA1919F012E5D66
:10E080003F40A111FACFF901E252F04F2D3EA1E03D
:10E090003A0730F4A191A111E0CF2F5F3F4FF6CFA7
:10E0A0002D3EE1E03E07C9F6EEEDFFE09F012E5D5B
:10E0B0003F40A191AA23D1F3D0CF08958091CF11F1
:10E0C0009091D011181619060CF043C00197909347
:10E0D000D0118093CF11892BA1F48091DA0F909108
:10E0E000DB0F892B21F41092DD0F1092DC0F809151
:10E0F000DC0F9091DD0F9093CC118093CB1181E0D8
:10E1000008958091CB119091CC110396FC01E252BD
:10E11000F04F208101962111F9CFFC01E252F04F1E
:10E120008D3E21E0920740F441919C012F5F3F4FCB
:10E130004111E1CFC901F4CFEEEDFFE08D3E21E0CA
:10E140009207C9F6CF018E5D9F4021912223D1F322
:10E15000D2CF80E00895FC0120E03EE2DB014D914A
:10E16000BD01403249F0283011F430833196DB0193
:10E1700011974C91408331962F5F2B3079F71082A5
:10E18000089540E050E0BA010D94DB38FC01238192
:10E1900021110D94336F089590910405911107C0DA
:10E1A0009091C00095FFFCCF8093C60008959130F8
:10E1B00031F49091C80095FFFCCF8093CE00089574
:10E1C0000E94CC7090E080E00895CF93DF93EC0143
:10E1D000FE018491882321F00E94CC702196F8CF13
:10E1E000DF91CF910895CF92DF92EF92FF92C0908E
:10E1F000C40DD090C50DE090C60DF090C70D89E01C
:10E2000099E70E94E57042E0C701B6010F94EA97D2
:10E2100081E099E70E94E57060918A0370918B0319
:10E2200080918C0390918D0341E00F94EA97FF90C9
:10E23000EF90DF90CF900D949D984F925F926F92E8
:10E240007F928F929F92AF92BF92CF92DF92EF9286
:10E25000FF920F931F93CF93DF93CC24CA94DC2CAF
:10E2600076010EEA1FE093E2892E912CA12CB12CAD
:10E27000412C512C3201D0E0C0E08FEFC81609F4D8
:10E280005DC0C8010F948BA0EC01BC01990F880BF5
:10E29000990B0F940B9B20913E0430913F044091C9
:10E2A0004004509141040F94A4A22B013C01C701EA
:10E2B000B6010F9443978DE598E70E94E570C5017C
:10E2C000B4010F9443978DE598E70E94E570BE0175
:10E2D0000D2E000C880B990B0F9443978DE598E752
:10E2E0000E94E57020E030E04AE754E4C301B20147
:10E2F0000F944A9B0F942B4185E0880E911CA11C22
:10E30000B11C0E5F1F4F8FEFC81AD80AE80AF80A2F
:10E310000A3B8FE0180709F0B0CFDF91CF911F9132
:10E320000F91FF90EF90DF90CF90BF90AF909F90B4
:10E330008F907F906F905F904F9008958DED9DE34B
:10E340000E94E570B8CF882371F181E598E70E94BB
:10E35000E5706091231270E090E080E00F944397A5
:10E36000809123128430D8F0109223128CE498E725
:10E370000E94E5708091231290E00F9448418091B3
:10E3800023122091EF113091F0113093F21120936C
:10E39000F1110E94CBF60E94005F0D9414228F5F52
:10E3A00080932312E3CF86E89EE30E943C6D70E0E9
:10E3B00060E00E94E5BCE5CFCF93DF9389E498E766
:10E3C0000E94E570C5EFD1E1688179818A819B81E6
:10E3D00042E00F94EA9785E498E70E94E5706C812B
:10E3E0007D818E819F8142E00F94EA9781E498E7D6
:10E3F0000E94E570688579858A859B8542E00F9447
:10E40000EA978DE398E70E94E5706C857D858E859F
:10E410009F8542E00F94EA978BEC94E60E94E570AA
:10E4200080E00F94F2210F940B9BC2E3D4E02C8187
:10E430003D814E815F810F94A4A242E00F94EA9740
:10E4400089E398E70E94E57081E00F94F2210F9430
:10E450000B9B288539854A855B850F94A4A242E0F1
:10E460000F94EA9785E398E70E94E57082E00F94A5
:10E47000F2210F940B9B2C853D854E855F850F9473
:10E48000A4A242E00F94EA9781E398E70E94E57026
:10E4900083E00F94F2210F940B9B288939894A89D4
:10E4A0005B890F94A4A2DF91CF910D942B4180E45E
:10E4B00097E70E94E5706091C40D7091C50D809141
:10E4C000C60D9091C70D41E00F94EA978DE397E751
:10E4D0000E94E5706091F1117091F211072E000C0D
:10E4E000880B990B0F940B9B41E00F94EA9789E3FB
:10E4F00097E70E94E57060918A0370918B03809189
:10E500008C0390918D0341E00F94EA9786E397E79F
:10E510000E94E5706091ED117091EE11072E000CD4
:10E52000880B990B0F940B9B41E00F94EA9781E3C2
:10E5300097E70E94E5706091C40D7091C50D8091C0
:10E54000C60D9091C70D41E00F94EA978EE297E7D0
:10E550000E94E5706091F1117091F211072E000C8C
:10E56000880B990B0F940B9B41E00F94EA978AE27A
:10E5700097E70E94E5706091620670E090E080E0AD
:10E580000F94439785E297E70E94E57060915B06E0
:10E5900070E090E080E00F94439781E297E70E945B
:10E5A000E57060918E0670918F0680919006909133
:10E5B000910641E00F94EA970D949D980E94E570B2
:10E5C0000D949D988F929F92AF92BF92CF92DF92BF
:10E5D000EF92FF920F94460F6B017C012091320263
:10E5E000222309F1409178024130E9F08091140230
:10E5F00090911502A0911602B091170246015701A1
:10E60000881A990AAA0ABB0A30E0A8EEB3E00F9470
:10E610001DA186169706A806B9066CF0443031F1A4
:10E620009CF44230D4F4C0921402D0921502E092CD
:10E630001602F0921702FF90EF90DF90CF90BF90FC
:10E64000AF909F908F900895453069F787E79EE9D6
:10E650000E94E5708CE099E706C087E79EE90E947A
:10E66000E57089E399E70E94DE72DDCF87E79EE9D6
:10E670000E94E57083E299E7F6CFCF9381EA9DE0AF
:10E680000F947DA0CBE08C9FC0011124805B924F42
:10E690000F948BA08156904F803A9F40C8F088ED30
:10E6A00098E70E94DE7281EA9DE00F947DA08C9F26
:10E6B000C001112470E060E0805B924F0F94DBA0FA
:10E6C0008BE998E70F94190B81E0CF910C944B6A7A
:10E6D000CF910895EC01F8940F943112179A10928B
:10E6E000A306169A1092A406149A8AE59EE90E943F
:10E6F000E5708CE798E70E94DE72209779F0CE01F2
:10E700000E94DE72BE0185E99CE00F94DBA062E40A
:10E7100084E99CE00F94C5A00E943261C4E7D8E769
:10E72000F1CF8AE493E00F9473118091CF1190910F
:10E73000D011892B79F0E091CB11F091CC11E252FC
:10E74000F04F8081813011F0863021F485ED99E61B
:10E750000C94DE7208958091CF119091D011892B85
:10E7600029F00E9491730E945E70F5CF1092CC1137
:10E770001092CB111092DD0F1092DC0F81E080938C
:10E78000E6110895EF92FF920F931F93CF93DF93BB
:10E7900080919C12882389F186E098E70E94DE72BE
:10E7A00080EF97E70E94DE728FED97E70E94DE729E
:10E7B000C7E0DCE1C15058F1CD9F7001112401E0A8
:10E7C00010E08CED97E70E94E570F801EE0FFF1F57
:10E7D000EE0FFF1FEE0DFF1DE756FD4E60817181AC
:10E7E0008281938145E00F94EA970F5F1F4F0830B5
:10E7F000110539F70F949D98DDCF83E198E7DF91FC
:10E80000CF911F910F91FF90EF900C94DE72DF91EA
:10E81000CF911F910F91FF90EF900895CF92DF92CB
:10E82000EF92FF926B017C01C0922903D0922A03E0
:10E83000E0922B03F0922C03809145038230B1F4D7
:10E8400020E030E040E950E4C7010F949AA287FF2E
:10E8500014C08091620490916304A0916404B0910B
:10E860006504803D9740A105B10520F5C701B601BB
:10E87000FF90EF90DF90CF9008952AE939E949E9B8
:10E880005EE3C701B6010F949AA287FF0AC020E099
:10E8900030E048E351E4C701B6010F944A9B6B0195
:10E8A0007C018AEE94E70E94E570C701B6010F94DF
:10E8B0002B41DCCF2AE939E949E95EE3C701B6011A
:10E8C0000F949AA287FDE3CF20E030E040E85EE3BA
:10E8D000C701B6010F944A9B20E030E048E550E4C0
:10E8E0000F94A5A1DCCFCF92DF92EF92FF92CF934E
:10E8F000909145039817B9F1C82FC0902903D09083
:10E900002A03E0902B03F0902C0320E030E0A901D3
:10E91000C701B6010F949AA2882341F0C0928604E1
:10E92000D0928704E0928804F09289048DEC94E7F9
:10E930000E94E570C13011F1E0F0C23011F1C093D6
:10E9400045036091860470918704809188049091BA
:10E9500089040E940E7460938604709387048093E8
:10E96000880490938904CF91FF90EF90DF90CF902F
:10E97000089585EC94E70E94DE72E1CF81EC94E784
:10E98000FACF8DEB94E7F7CF0F941422179AE3EAAE
:10E99000F6E01082169A1182149A80E00E94737435
:10E9A0008FEF9FEF90937502809374022FEF209367
:10E9B000710290933E0280933D0220933F02909318
:10E9C00073028093720290933C0280933B020895FD
:10E9D000182FF894CDB7DEB700D0CF90DF90EF902E
:10E9E00088E199E20FB6F894A895809360000FBE75
:10E9F000909360009FB7F894E2E0F1E08081886036
:10EA000080839FBF0F9431128CE794E70E94DE72DF
:10EA100084E794E70E94E570612F70E090E080E069
:10EA20004AE00F94CD9680E794E70E94E5708E2D22
:10EA3000B60190E040E10F94CD968CE694E70E94F9
:10EA4000E570BE0190E080E040E10F94CD960F9418
:10EA50009D9840E060E072E290E080E00F94835285
:10EA600085ED99E60E94DE720E943261C82F729A8B
:10EA7000682F83E09DE00F94A1A080917C068823FD
:10EA800019F08C2F0E94E8740E9432611F920F923D
:10EA90000FB60F92112483E00E9436751F920F92D9
:10EAA0000FB60F92112482E00E94367541ED50E0BE
:10EAB0006BE973E782E394E00F94179E0F94367529
:10EAC0000F9468180E945D5F87E79EE90E94E570D9
:10EAD00089E793E70C94DE7244E050E064E170E073
:10EAE00082E394E00F946DA043E050E06BE973E79C
:10EAF00082E394E00F945C9E892B09F05DC0EFE502
:10EB0000F4E7459155916591749188ED90E00E94EC
:10EB1000AD5DE3E6F4E745915591659174918CED17
:10EB200090E00E94AD5DE7E6F4E7649180EE90E04E
:10EB30000E94786FE8E6F4E76591749181EE90E0C9
:10EB40000E94606FEAE6F4E76591749183EE90E0CD
:10EB50000E94606FEBE5F4E74591559165917491E2
:10EB600084ED90E00E94AD5D47E354E760E170E022
:10EB700080EB90E00E94416F47E454E760E170E071
:10EB800080EC90E00E94416F41ED50E064E170E064
:10EB900082E394E00F946DA00E945D5F0F94367540
:10EBA0000F94681887E79EE90E94E5708FE593E768
:10EBB0000E94DE7281E008950E94567564E070E064
:10EBC00084E190E00E949B5591E0892708956BE9CC
:10EBD00073E782E394E00F94349E41ED50E064E1EA
:10EBE00070E082E394E00F9491A087E79EE90E9491
:10EBF000E5708FE493E70C94DE722F923F924F9270
:10EC00005F926F927F928F929F92AF92BF92CF92BC
:10EC1000DF92EF92FF920F931F93CF93DF93CDB7C5
:10EC2000DEB7A0970FB6F894DEBF0FBECDBF8FE55D
:10EC300090E00E944756882309F4A1C00E944B55DA
:10EC40008F37910561F48091B1059091B205909351
:10EC5000B0058093AF0580E493E70E94DE726E01F9
:10EC60004FE1C40ED11C992493940E944B55181661
:10EC700019060CF078C08091E711882329F00E94D2
:10EC80004861882309F46FC08091610381116BC0D2
:10EC90002091B1053091B2058091AF059091B005FA
:10ECA0008217930711F3F901E15DFA4F80812F5F1D
:10ECB0003F4F2F7733273093B2052093B1058F3F15
:10ECC00009F079C080911B03882309F471C09092E8
:10ECD0001A0310921B031F8E18A280901E03882017
:10ECE00021F280911C038F8FF1E0F81518F48091C8
:10ECF0001D0388A310921E031601822D8C198815FE
:10ED000008F0B3CFF10111911F0181E293E00F945C
:10ED1000A80F17FDF2CF8091DA0F9091DB0F1A3018
:10ED200009F44BC11D3009F448C18F3591050CF031
:10ED300049C11B3311F4909220032091200321112B
:10ED4000DCCF9C012F5F3F4F3093DB0F2093DA0F16
:10ED50002091DC0F3091DD0F2252304F820F931F34
:10ED6000FC011383CACF8091DA0F9091DB0F181644
:10ED700019060CF451C280916A13811167C2A096E2
:10ED80000FB6F894DEBF0FBECDBFDF91CF911F91BC
:10ED90000F91FF90EF90DF90CF90BF90AF909F903A
:10EDA0008F907F906F905F904F903F902F9008953D
:10EDB00090921B0390CF90911A03992309F458C0A5
:10EDC000893FE9F170F5863F09F44AC0873F09F4AD
:10EDD00043C08BE093E70E94E57086E093E70E94D2
:10EDE000E5701091190382E093E710FD02C08DEFEA
:10EDF00092E70E94E570012F027088EF92E711FD03
:10EE000002C083EF92E70E94E57082EF92E70E94D2
:10EE1000DE72002349F185E480930B0210921A03FD
:10EE20005ACF8A3F41F08B3FA1F680911903816050
:10EE300080931903CECF809119038E7FF9CF109262
:10EE40001E0310921A0310921903109218031092C5
:10EE50001B0310921703BDCF809119038260E8CF86
:10EE6000809119038D7FE4CF90E290930B02D6CF6F
:10EE700090911B0330911903992331F1E0911E0306
:10EE800030FF49C020911703222309F440C091E0CC
:10EE90009E0F90931E03AE2FB0E0A45EBC4FFFEF19
:10EEA000FC9340911803442351F0EE5FE0931E035E
:10EEB000E92FF0E0E45EFC4F4083109218032150EC
:10EEC0002093170310921B03E0911E0330FF6CC0C8
:10EED00090911703992349F121E02E0F20931E03EF
:10EEE000AE2FB0E0A45EBC4F8C93809118038823B2
:10EEF00051F0EE5FE0931E03E22FF0E0E45EFC4F82
:10EF0000808310921803915090931703E4CE42E04F
:10EF100040931703D7CF91E09E0F90931E03F0E02C
:10EF2000E45EFC4F9FEF9083CDCFA82FAF7030E011
:10EF300021E0AF3029F0B0E0A050BE4F3C9120E07E
:10EF4000482F407F403F59F4226020FF13C0909229
:10EF5000170321FF0CC0E2E0E0931703BCCE8295BB
:10EF60008F70A82FB0E0A050BE4F9C91EECF909331
:10EF70001803B1CE81E08E0F80931E03AE2FB0E058
:10EF8000A45EBC4F3C933A3009F4A5CE21FF03C0E8
:10EF900090921703A0CEEE5FE0931E03E82FF0E0FF
:10EFA000E45EFC4F908397CE91E09E0F90931E03FA
:10EFB000F0E0E45EFC4F80838ECE009719F410924F
:10EFC0002003DDCE0091DC0F1091DD0F0F51104FAB
:10EFD000800F911FFC0110821A8309838091200306
:10EFE0008111FDC0F80180818E3409F084C04AE0AF
:10EFF00050E0BE016F5F7F4FC80101960F94089CDF
:10F000002B013C01E980FA80F7018081803231F4E4
:10F01000FFEFEF1AFF0AFA82E982F4CF8091D11153
:10F020009091D211A091D311B091D4110196A11D4C
:10F03000B11D84159505A605B70549F044E050E0DB
:10F040006BE373E7C7010F945C9E892BA1F46AE21E
:10F0500070E0C7010F94D4A69093F6168093F5162E
:10F06000009709F441C0F801F12C8E179F07F1F0C9
:10F070002191F226FACF8AE59EE90E94E57082EEA0
:10F0800093E60E94E5706091D1117091D211809148
:10F09000D3119091D4110F9443970F949D980E948F
:10F0A0006D551092DB0F1092DA0F69CE0E94D85581
:10F0B000F816190639F08AE59EE90E94E57083EC9E
:10F0C00093E6DFCFE091F516F091F6161082E98015
:10F0D000FA8066E373E7C7010F942B9E892B39F5FD
:10F0E00089E296E60E946A738AE59EE90E94E570CD
:10F0F00089E993E6C6CF89819A81FC01208120327B
:10F1000021F401969A838983F6CF6AE270E00F9426
:10F11000D4A6892B39F08AE59EE90E94E5708FE636
:10F1200093E6AFCF44244A94542C3201D0CF44E02C
:10F1300050E061E373E7C7010F945C9E5C01F70147
:10F140008081873481F48091CB0D853061F085ED2D
:10F1500091E10F94A80FF6E0F093CB0D60E085EA03
:10F160009FE00F94A1A0AB2821F08091CE118111D6
:10F1700098CF26E077FC21E08091DC0F9091DD0FA5
:10F18000FC01E252F04F208349815A81F801DA01F3
:10F1900040175107A1F501900020E9F79F01201BBE
:10F1A000310B0396280F391F2D3EF1E03F0779F10F
:10F1B0003093DD0F2093DC0F8091CF119091D0110F
:10F1C00001969093D0118093CF1177FC08C04092A4
:10F1D000D1115092D2116092D3117092D411109229
:10F1E000DB0F1092DA0F0E944B55892B09F4C7CD23
:10F1F0008FE590E00E94475681117FCDC0CD6D9183
:10F2000061939D01241B350B6111F9CFCACF109278
:10F21000DD0F1092DC0FD0CF8091CA0D60E273E059
:10F22000811102C060ED77E081E293E00F94790FE5
:10F23000882309F4A0CD109220031092DB0F1092C6
:10F24000DA0F86E293E70E94DE7299CD8091FD1578
:10F25000882309F494CD8091DA0F9091DB0F892BEC
:10F2600009F08DCD8091CF119091D011892B11F49F
:10F2700010921F0312E001E040917E1650917F161C
:10F280006091801670918116809177169091781612
:10F29000A0917916B0917A16481759076A077B072B
:10F2A00008F0C1C080911F038111BDC00F946C484C
:10F2B0004091021650910316609104167091051644
:10F2C00040937E1650937F1660938016709381163C
:10F2D0002091DA0F3091DB0F8A3061F08D3051F0E0
:10F2E000833209F487C02F35310524F48F3F980706
:10F2F00009F087C02115310509F441CD8091FD1534
:10F30000811103C040E050E0BA018091DC1190917E
:10F31000DD11481B590BA091DC0FB091DD0FFD01F1
:10F32000E252F04F10834183528313962252304FA2
:10F33000F901EA0FFB1F1082A252B04FFD010190AC
:10F340000020E9F73197EA1BFB0BF8948091CF116D
:10F350009091D01101969093D0118093CF11EC5FD2
:10F360008091DC0F9091DD0FE80FF92FF11DF093E4
:10F37000DD0FE093DC0F8091FD15882309F43DC07B
:10F3800080917E1690917F16A0918016B091811683
:10F390008093DC119093DD11A093DE11B093DF1107
:10F3A000ED3EF14021F41092DD0F1092DC0F7894C5
:10F3B000109220031092DB0F1092DA0F40917E160C
:10F3C00050917F166091801670918116809177160A
:10F3D00090917816A0917916B0917A16481759072E
:10F3E0006A077B0700F58FE590E00E944756811180
:10F3F00043CFC5CC00931F037DCF80E090E0DC01BC
:10F40000C7CFA9014F5F5F4F5093DB0F4093DA0FD7
:10F410004091DC0F5091DD0F4252504F240F351FA9
:10F42000F901838329CF40917E1650917F16609118
:10F430008016709181168091771690917816A09120
:10F440007916B0917A16481759076A077B0708F4AE
:10F4500096CC0E941E70892B09F091CC0F948241AA
:10F460008CE593E60E94DE720F94381C6B017C01E0
:10F470000E94C35F8CE3882E912CA12CB12CC70174
:10F48000B601A50194010F94F0A0CA01B901A5012C
:10F4900094010F94F0A07F936F93C701B60120E110
:10F4A0003EE040E050E00F94F0A03F932F9382E1C4
:10F4B00093E79F938F938E010F5F1F4F1F930F93BF
:10F4C0000F94949F87E79EE90E94E570C8010F940E
:10F4D0009E99C8010E9453EF0F94DC4C1092560283
:10F4E0000FB6F894DEBF0FBECDBF80916B1388239B
:10F4F00059F00F94AF438091CA0D882309F43FCC93
:10F5000086E00F94A0983BCC81E00F941B4D809136
:10F510006B138111EECFEFCF0F931F93CF93DF9338
:10F52000D82F80918416813009F449C0823009F4C3
:10F530004DC00E94A4618111ECC08091F1119091A5
:10F54000F211009739F42091ED113091EE11232B37
:10F5500009F4DFC0409133025091340260913502CA
:10F5600070913602411551056105710509F4D1C04C
:10F57000892B31F48091ED119091EE11892B29F0B6
:10F5800080911A06882309F42CC18091CA0D882322
:10F5900021F040EE52E369E270E08AE196E00F94D8
:10F5A000B40F882309F4B7C00F94311280E696E3B4
:10F5B0000E943C6D0F94190B0E94E9FDACC082E0E3
:10F5C000809384160E94F7C3809387161092881642
:10F5D00080918416823009F0ACCF80918916811118
:10F5E0003DC00E94F7C3C82F80918716C81709F441
:10F5F000A0CFC093871689E896E10F94A80FCC237B
:10F60000B1F180918516882311F1809162038111F7
:10F610001EC0809194128130D1F08091A80D9091FC
:10F62000A90D891B8F7099F40E94536181110FC03D
:10F630008091C80D843059F08FE59FE00F947DA034
:10F64000811105C061E081E498E30F94CA9481E0E0
:10F650008093881681E080935B026BCF64E670E054
:10F6600089E896E10F94790F8111BBCF62CF809129
:10F670008616882379F3809162038111EBCF809104
:10F68000A80D9091A90D891B8F7021F40E945361E0
:10F69000882301F38091E7118111DCCF80919412CE
:10F6A0008130C1F28091C80D8430A1F28FE59FE0D6
:10F6B0000F947DA08111CECF8AE295E69F938F9320
:10F6C00080E195E69F938F930F943F9F109286164B
:10F6D000109285160F900F900F900F908091E71168
:10F6E000811105C060E070E0CB010F948F4160E0B4
:10F6F00070E0CB010E94CB6185E69FE00E94976F8E
:10F7000081E09FE00E948A6F8FE19CE60F94F542B2
:10F71000A1CF10921A068091CF119091D01103972A
:10F7200014F40E94FD759091A80D8091A90D981771
:10F7300081F08091CB0D863061F468E873E185ED4E
:10F7400091E10F94790F882321F085ED91E10F94D9
:10F75000A80F409146035091470360914803709170
:10F760004903411551056105710509F03FC04091FC
:10F770003702509138026091390270913A02411576
:10F78000510561057105A9F08AE493E00F94B40F67
:10F79000882379F09091A80D8091A90D981309C044
:10F7A000D11107C0179A1092A306169A1092A406B8
:10F7B000149AC091E9119091A90D8091A80D981704
:10F7C00001F18091A90D9EE6899FF0011124E25F6D
:10F7D000F84FC0819091A80D981799F08F5F8F70A6
:10F7E000F9CF8AE196E00F94731195CF8AE493E004
:10F7F0000F94B40F882309F4BACF80E698E70E94EB
:10F800006A73CC2309F4BEC08091410390914203F6
:10F81000A0914303B0914403892B8A2B8B2B81F455
:10F820000F94460F605E7C4F8F4F9F4F6093410354
:10F83000709342038093430390934403CFEF0FC030
:10F840000F94460F0091410310914203209143030E
:10F8500030914403601771078207930778F3809112
:10F860008403882309F497C0C093670280912D0414
:10F87000811107C081E080932D040F94F3641092EE
:10F880002D04809113068823C9F1109213064FB7F7
:10F89000F89480911106282F082E000C330B37FFA7
:10F8A00003C0319521953109243031050CF476C01F
:10F8B000982F87FF02C093E0980F9595959520911A
:10F8C000060530910705290F311D97FD3A953093B4
:10F8D000070520930605837887FF03C081508C6F4E
:10F8E0008F5F809311064FBF86E00F94712C80913B
:10F8F0005B02811103C081E080935B02809114065A
:10F90000882361F00E941E6CE091D403F091D5032E
:10F91000309721F080915C0281111995209162133A
:10F9200030E0A8EEB3E00F941DA1AB01BC0183E66B
:10F9300093E10F94B40F882399F08091611380FDB7
:10F940000E9457728091611382FD0E94DC71809148
:10F95000611381FD0E94286083E693E10F94731187
:10F960008091CA0D811102C00E94E27240E355E706
:10F9700060E070E08AE593E0DF91CF911F910F91F5
:10F980000D94B40F1092410310924203109243035E
:10F990001092440364CFC093050568CF10921106FE
:10F9A0004FBF80E0A2CFCF93DF93EC010F94F731EC
:10F9B00081E00E948C7A80E00E94CD69209799F0C6
:10F9C000C233D10540F062E370E080E090E00F9434
:10F9D0004D0DE297EBCFBE0190E080E00F944D0D0E
:10F9E000D0E0C0E0E3CFDF91CF910895CF93DF93D4
:10F9F000C82FDFEF0F94F73181E00E948C7A80915D
:10FA000092128F3FD9F480912712843021F4809193
:10FA10002A128111EFCF80916512909166120197A1
:10FA200049F780918C1290918D128932904811F390
:10FA300060E089E290E80F94484FDCCFD0939212B7
:10FA4000853039F4CF3FF9F261E08C2F0F948F6B42
:10FA5000D1CF8430C1F6DF91CF910895CF93DF935A
:10FA6000EC018991882319F00E94CC70FACFDF91C4
:10FA7000CF910895FF920F931F93CF93DF93EC01E3
:10FA8000F62E662309F44BC00F943B9E8C01C801EF
:10FA90000E944756882309F453C08091DC0F90914F
:10FAA000DD0FFC01E252F04F23E020838F51904F95
:10FAB000BE01FF20E9F10F94349E87E79EE90E9482
:10FAC000E57081E593E60E94E5708091DC0F9091EE
:10FAD000DD0F8F51904F0E942E7D80EF92E70E94A4
:10FAE000DE728091DC0F9091DD0F0496080F191FD4
:10FAF0000D3E81E01807F9F01093DD0F0093DC0F45
:10FB00008091CF119091D01101969093D011809354
:10FB1000CF11DF91CF911F910F91FF900895FC01BC
:10FB200001900020E9F731978F01081B190BAFCF27
:10FB30000F94E8A6C2CF1092DD0F1092DC0FE0CF39
:10FB40008AE59EE90E94E57081E593E60E94E570F2
:10FB5000CE01FF2059F00E94E57088E29EE9DF9116
:10FB6000CF911F910F91FF900C94DE720E942E7D19
:10FB7000F4CF0F931F93CF93DF93D62F8C01C0E068
:10FB8000F8018591949161E00E943A7DCF5F0E5F0C
:10FB90001F4FDC13F5CFDF91CF911F910F91089587
:10FBA000CF93DF93CDB7DEB76E970FB6F894DEBF75
:10FBB0000FBECDBF9E012C5D3F4FF9014191519188
:10FBC0009F016EE170E0CE0101960F94D39F60E03B
:10FBD000CE0101960E943A7D6E960FB6F894DEBF74
:10FBE0000FBECDBFDF91CF9108951F920F920FB638
:10FBF0000F9211240BB60F922F933F934F935F9365
:10FC00006F937F938F939F93AF93BF93EF93FF93E4
:10FC10002091780030917900E0911603F0E0EE0F2A
:10FC2000FF1FEA5FFC4F80819181820F931F9183B8
:10FC30008083809105038F5F809305038031E9F510
:10FC4000809116038F5F80931603883071F5809141
:10FC500006039091070390934A068093490680918A
:10FC60000A0390910B0390934C0680934B0680916E
:10FC7000080390910903909348068093470681E01A
:10FC800080936306FF91EF91BF91AF919F918F9108
:10FC90007F916F915F914F913F912F910F900BBE8C
:10FCA0000F900FBE0F901F901895809104034FE5A1
:10FCB00053E08F5F41F41092040380917A008064D6
:10FCC00080937A00DFCF9A01082E02C035952795E0
:10FCD0000A94E2F720FFEDCF809304030E94585569
:10FCE00010920503EACFCF93DF93CAE7D0E0888173
:10FCF0008F7B8883109205031092160310920403E1
:10FD000080E00E945855E6E0F3E080E1DF011D92BB
:10FD10008A95E9F7888180648883DF91CF9108957F
:10FD20002F923F924F925F926F927F928F929F920B
:10FD3000AF92BF92CF92DF92EF92FF920F931F93F9
:10FD4000CF93DF93CDB7DEB7A4970FB6F894DEBF9D
:10FD50000FBECDBF0F9414228091AC0D811117C03E
:10FD600081E0809306128091A306882349F0809158
:10FD7000A406882329F02091A5062F83211120C0F5
:10FD800081E08093E61186EB98E60F94F542A49605
:10FD90000FB6F894DEBF0FBECDBFDF91CF911F919C
:10FDA0000F91FF90EF90DF90CF90BF90AF909F901A
:10FDB0008F907F906F905F904F903F902F9008951D
:10FDC0008BEA9DE00F947DA0182F8EE40E94B6551B
:10FDD000082F0E94CB558E83002329F0873009F429
:10FDE000C9C0833029F0133009F0C3C063E06E83CB
:10FDF00080E090E0A0E8BFE38A839B83AC83BD836F
:10FE00008AEA9DE00F947DA0888F83E40E94B65516
:10FE1000182F0E94CB55112329F0882319F08B301D
:10FE200008F4888F88E50E94B655882309F4ABC092
:10FE30000E948E5A20E030E048E052E40F94A4A1E2
:10FE400020E030E048EB51E40F94A4A16A877B875F
:10FE50008C879D8789E50E94B655882309F49CC04C
:10FE60000E948E5A20E030E048E052E40F94A4A1B2
:10FE700020E030E040EA50E40F94A4A16C8B7D8B2D
:10FE80008E8B9F8B87E50E94B655882309F489C025
:10FE90000E948E5A2A853B854C855D850F94A5A1CD
:10FEA00020E030E048E852E40F94A5A1698F7A8FF2
:10FEB0008B8F9C8F88E40E94B655882309F47AC002
:10FEC0000E948E5A2C893D894E895F890F94A5A185
:10FED00020E030E048E852E40F94A5A16D8F7E8FBA
:10FEE0008F8F98A30F94925680912C0290912D029F
:10FEF000A0912E02B0912F0280939D1290939E129A
:10FF0000A0939F12B093A0120F94AC8B05EC1FE04E
:10FF1000C8010F948BA0019609F051C00E5F1F4FCE
:10FF2000053D8FE01807A1F7212CACE9B2E1BAA397
:10FF3000A9A3B987A887512C412C312C042D842DDD
:10FF400063E00F942CA1988B6884798410E0F88981
:10FF5000F11137C0812F63E00F942CA1911131C0B2
:10FF600021103FC17E81733009F470C08F818E876C
:10FF700037C01E836AE979E989E19FE36A837B835D
:10FF80008C839D833DCF80E090E0A0E8BFEF8A871F
:10FF90009B87AC87BD875ECF60E070E080E89FEF15
:10FFA0006DCF80E090E0A0E8BFE7898F9A8FAB8F9C
:10FFB000BC8F80CF60E070E080E89FE78FCF2F801C
:10FFC000B4CF60E070E080EC9FE7D30111966D93B1
:10FFD0007D938D939C931497BE81B330C1F11E869F
:10FFE000812F0F94068C4B015C01802F0F94068C9F
:10FFF0006B017C01A50194016A857B858C859D85BB
:020000021000EC
:100000000F942EA418160CF41CC1298D3A8D4B8D1B
:100010005C8DC501B4010F942EA418160CF411C107
:10002000A70196016C897D898E899F890F942EA4E2
:1000300018160CF406C12D8D3E8D4F8D58A1C701A9
:10004000B6010F942EA418160CF4FBC033941F5F56
:1000500024E0620E711C173009F079CF6FEF461A59
:10006000560A888599854C969987888797E049161E
:10007000510409F063CF0E94CEF0A091C706AF8370
:10008000B091AC03B88781E08093C7068AE0830D06
:100090008093AC0381E00E94CD6980E090E0A0EA0B
:1000A000B0E48093FD119093FE11A093FF11B093E3
:1000B000001265E575E585E591E40F94118580E012
:1000C0000E9479609CA38BA3312C832D67E00F9451
:1000D0002CA1F82E092F682F70E07F876E8780FF94
:1000E00003C076E0791B072F802F63E00F942CA1CB
:1000F000911105C08F2D0F942CA111E0911110E0EA
:10010000802F0F94068C688B798B8A8B9B8B8F2D1D
:100110000F94068C4B015C018E81833009F099C0ED
:100120001111C8C027E0AE85BF852A9FF0012B9F23
:10013000F00D1124E00FF11DEE0FFF1FEE0FFF1F5A
:10014000E456FD4E60E070E080EC9FE761837283CF
:10015000838394833394E1E33E12B7CF80E090E051
:10016000A0EAB0E48093FD119093FE11A093FF11DB
:10017000B093001265E575E585E591E40F9411856E
:100180000F941422B1E33B1609F43CC280913F0363
:1001900091E0980F90933F03882309F4D3C160E066
:1001A00080E00E9464EF84E396E30E943C6D0F942C
:1001B000190B80E00F944D2F81E0809378028BE043
:1001C0009CE60E945FE62F812093C70668856093B6
:1001D000AC0382E00E94CD690F94142210920612A3
:1001E000D6CD011103C0112309F4BCCE812F63E0E9
:1001F0000F9438A1840D952D911D880F991F8D5353
:10020000904F0F948BA0BC01990F880B990B0F9402
:100210000B9B2AE037ED43E25CE30F944A9B9B0182
:10022000AC0160919D1270919E1280919F129091ED
:10023000A0120F94A5A1F301618372838383948339
:1002400091CEFE85FF2309F402CF222009F4FECED1
:10025000FECE288939894A895B896A857B858C85A8
:100260009D850F942EA4181604F1288939894A898E
:100270005B89698D7A8D8B8D9C8D0F949AA287FDF9
:1002800014C0A50194016C897D898E899F890F9482
:100290002EA4181654F0A50194016D8D7E8D8F8DBE
:1002A00098A10F949AA287FF05C0112309F452CF99
:1002B000211050CF10E0A7E08E859F85A89FF00108
:1002C000A99FF00D1124E00FF11FEE0FFF1FEE0F9D
:1002D000FF1FE456FD4E4180528063807480C12C24
:1002E000D12CE0EAEE2EE0E4FE2E222051F023E3B2
:1002F00033E343EB5EE3C301B2010F94A5A16B01AD
:100300007C01A70196016091FD117091FE11809111
:10031000FF11909100120F949AA287FF10C0C09213
:10032000FD11D092FE11E092FF11F092001265E5EE
:1003300075E585E591E40F9411850F941422688981
:1003400079898A899B896093F5117093F61180935E
:10035000F7119093F8118092F9119092FA11A092EE
:10036000FB11B092FC1169EF71E185EF91E10E9400
:10037000316460E070E086E193E40F9411850F949E
:1003800014228091AC0D882339F07F817093C706C9
:1003900088858093AC03FBCC812C912C70E2A72E36
:1003A00071ECB72E222051F02A813B814C815D8176
:1003B000C301B2010F94A4A14B015C01488DC5019A
:1003C000B4010F949C5681110BC089EE92E60E94F5
:1003D0003C6D9F938F930F943F9F0F900F90BECED5
:1003E0002091FD113091FE114091FF1150910012AA
:1003F000C701B6010F94A4A120E030E0A9010F9439
:100400009AA287FF36C060E070E080EA90E46093D3
:10041000FD117093FE118093FF119093001265E51A
:1004200075E585E591E40F9411850F941422488DAC
:10043000C501B4010F949C56882339F22091FD1117
:100440003091FE114091FF115091001260E070E078
:1004500080EA90E40F94A4A12DEC3CEC4CEC5DE31D
:100460000F949AA287FF05C08DEA97E70F94669FC5
:1004700075CEC090FD11D090FE11E090FF11F0906C
:1004800000122220A1F0A7019601C301B2010F942E
:10049000A4A19B01AC015F776A817B818C819D81E6
:1004A0000F949AA287FF03C084E797E7DFCF8FEA14
:1004B0009FE00F947DA0882309F440C086EA9FE066
:1004C0000F947DA08823D1F160918E0670918F06E4
:1004D00080919006909191060E948F5620913E0443
:1004E00030913F0440914004509141040F94A4A2E4
:1004F0009B01AC01E7E0AE85BF85EA9FC001EB9FA1
:10050000900D1124080F191F000F111F000F111F4C
:1005100004561D4EC701B6010F94A4A1D80111962F
:100520006D937D938D939C9314978091AC03815030
:100530008093AC0381E00E94CD690CCE20E030E0D6
:10054000A901D8CF85E00F94712CC12CD12C90EA51
:10055000E92E90E4F92E80E096E30E943C6D0F9422
:10056000920A90E080E00F943D3481E00F9499343A
:1005700080E00F944C2C182F60E070E080E89FEB37
:100580000E94686781E00F944C2CC092FD11D092BC
:10059000FE11E092FF11F092001265E575E585E528
:1005A00091E40F9411850F941422812F0F944C2CF9
:1005B00082E00F94002220E030E040EA50E40F9403
:1005C0002EA4181644F2EF81E093C706F885F09345
:1005D000AC0381E00E944B6ADD24D394DF92812C2E
:1005E000912C5401CC24C394E12CF12C870121E0FF
:1005F00040E050E0BA0181E00E94FE67D092E6112F
:100600000F90C5CB10923F038BA19CA10E945F600D
:1006100010922A051092290580E10E944FD8882364
:1006200091F00E943D7381EA9DE00F947DA02BE044
:10063000829FC0011124805B924F0F948BA09093F6
:100640002A05809329056091290570912A05072EB6
:10065000000C880B990B0F940B9B905820913E0433
:1006600030913F0440914004509141040F94A4A262
:100670000F94728B80EC9FE00F947DA091E081300D
:1006800009F090E099834FEB5FE06CE4CE010196B6
:100690000E94E555F82E4EEB5FE062E5CE01019633
:1006A0000E94E555082F4DEB5FE066E4CE01019610
:1006B0000E94E555182F4CEB5FE062E4CE010196F5
:1006C0000E94E555212F110F330B082E000C990BBA
:1006D0005C01A21AB30A8F2DFF0C990B280F391F4A
:1006E00046E0429F6001439FD00C1124F12CE12C85
:1006F000002E000C110B081B190BB70163567D4E21
:100700003B01460177E07A83D3012D903D904D90D7
:100710005D903D01FD013497FB87EA87B401092C08
:10072000000C880B990B0F940B9B2FE333EC4EE2DC
:1007300059E30F944A9BA20191010F94A5A1AA85A8
:10074000BB856D937D938D939C931397BA81B15024
:10075000BA83800E911EB111D7CFCA0CDB1CECE11D
:10076000EE0EF11CF4ECEF16F10439F60E94CEF017
:100770008DE40E94B655882309F484C00E94CB55AD
:100780002E81273009F094C0882309F491C0BB243E
:10079000B394AA24AA94AB0C09A11AA1612C8EEFE0
:1007A000882E8B0C6A2D862D0F943D8B9924939463
:1007B000960C81116EC06B2D862D0F943D8BC12C34
:1007C000D12C7601712C882381F020E030E0A90142
:1007D000D8015D966D917D918D919C9190970F942C
:1007E000A5A16B017C0177247394682D862D0F944D
:1007F0003D8B882369F0F8017B972081318142810C
:100800005381C701B6010F94A5A16B017C017394BC
:100810006A2D892D0F943D8B882361F0F801258185
:10082000368147815085C701B6010F94A5A16B01A0
:100830007C0173946A2D8FEF860D0F943D8B882376
:1008400031F1F80133972081318142815381C70111
:10085000B6010F94A5A16B017C017394672D70E024
:1008600090E080E00F940B9B9B01AC01C701B601A7
:100870000F94A4A2D80111966D937D938D939C93B0
:10088000149707C08CEA9DE00F947DA079CF71107A
:10089000E5CF692C0C5F1F4FB7E09B1283CFB39459
:1008A000E9A1FAA17C96FAA3E9A3F8E0BF1271CFFF
:1008B00081E080939C128FE40E94B655811103C0A1
:1008C0000F94C78B79CC0E94CB558111F9CF0E9430
:1008D000546072CC2F923F924F925F926F927F92B0
:1008E0008F929F92AF92BF92CF92DF92EF92FF9240
:1008F0000F931F93CF93DF93CDB7DEB7C356D109C4
:100900000FB6F894DEBF0FBECDBF82E080937802B1
:100910000091CB111091CC110F51104F45E050E0D8
:1009200061EC71E8C8010F945C9E892B09F09BC1B2
:100930008091CA0D882309F44DC08DEB9EE70F947A
:10094000F274882379F08091F7161F928F9384EBCD
:1009500095E69F938F930F943F9F0F900F900F906A
:100960000F9008C089EB9EE70F94F274882341F042
:100970001092D60381E0809378020E9491733AC26C
:1009800086EB9EE70F94F274882321F18091F5168F
:100990009091F61661E003960F94A44B0F946C4867
:1009A0008C018091021690910316A0910416B091CB
:1009B000051680937E1690937F16A0938016B093B1
:1009C0008116802F0E94CC700A30110539F70F94E0
:1009D0008241D0CF87EB91E80F94F2748111CACF96
:1009E00083EB91E80F94F274882321F140918703FF
:1009F000509188032CE3249FC001259F900D112462
:100A00009F938F934091850350918603249FC0014B
:100A1000259F900D11249F938F9382ED97E69F93CE
:100A20008F930F943F9F0F900F900F900F900F9008
:100A30000F90A0CF8EEA91E80F94F274882311F101
:100A40008CE89FE00F947DA0811110C061E089E8DF
:100A50009CE60E943A7D60E085EA9FE00F94A1A0A9
:100A600060E08FE79CE00F94A1A084CF813009F073
:100A700081CF0F94282085ED91E10F94A80F0F945A
:100A8000520F78CF87EA91E80F94F274882321F00F
:100A900080E00F94FE626ECF81EA91E80F94F274C9
:100AA00081110E9432618EE991E80F94F2748823DB
:100AB000A9F044E150E065E17DE0CE0101960F949C
:100AC0006DA08C89882329F083E991E80F94669FB3
:100AD00051CFCE0101960F940CA74CCF8FE891E82F
:100AE0000F94F274882329F083E891E80E94DE7263
:100AF00041CF8FE791E80F94F274882319F08FE5C6
:100B000091E8F4CF8AE591E80F94F274882319F004
:100B10000E943F6C2FCF87E591E80F94F2748823F1
:100B200079F081EA9DE00F947DA02BE0829FC001C7
:100B3000112470E060E0805B924F0F94BFA01ACF49
:100B400084E591E80F94F274882351F00E94396A89
:100B500040E070E060E084E690E00F946131D8CF2F
:100B600080E591E80F94F2748823E1F086E50E9415
:100B7000B655882309F4FECE0E94D85511E0892B82
:100B800009F410E00F94142280919C1290E0181741
:100B9000190609F4EFCE10939C128DEF91E10F949A
:100BA0009C75E8CE89E491E80F94F274882309F4E7
:100BB000E1CE84E40E94B6558823A1F00E948E5AAB
:100BC00020E030E04AE754E40F944A9B20E030E014
:100BD00040E05FE30F94A5A10F941DA3CB010E94F9
:100BE000F0EFC8CE85E491E80F94F274882349F1C0
:100BF0008091CA0D882329F18091F5169091F616FF
:100C000002969093F6168093F5160E948E5A6B0109
:100C10007C016FEF87EA9DE00F94A1A020E030E017
:100C20004AE754E4C701B6010F944A9B20E030E044
:100C300040E05FE30F94A5A10F941DA385EA9DE01A
:100C40007CCF85EA9DE00F948BA0BC0190E080E012
:100C50000F94099B20E030E04AE754E40F94A4A2EB
:100C60000F942B4187CED8018C91873411F00C94CE
:100C70005E911093F6160093F5160E94D855909346
:100C80005803809357038B34910509F445C60CF043
:100C90004BC18430910509F4AAC50CF0C5C097FD7D
:100CA000CFC002970CF0A2C10E9400558C010E9497
:100CB000B55B60918406709185068091860690915F
:100CC00087060F94099B6B017C01409001125090A4
:100CD0000212609003127090041280909F06909010
:100CE000A006A090A106B090A206A5019401C301A0
:100CF000B2010F94A4A120E030E048EC52E40F943C
:100D00004A9B9B01AC01C701B6010F942EA4181693
:100D1000D4F4A3019201C501B4010F94A4A120E071
:100D200030E048EC52E40F944A9BA70196010F94DF
:100D3000A5A10F941DA360938406709385068093EC
:100D40008606909387068091B404882309F446C1EF
:100D500088E50E94B655811141C189E50E94B655CA
:100D600081113CC18AE50E94B655811137C185E4E5
:100D70000E94B655882309F431C1209101123091A7
:100D80000212409103125091041260919F067091DB
:100D9000A0068091A1069091A2060F94A4A16B01D8
:100DA0007C012DEC3CEC4CEC5DEB0F949AA287FFA0
:100DB00007C18091030581110C9419B00F9414227E
:100DC00080919F069091A006A091A106B091A206E5
:100DD0008093011290930212A0930312B093041215
:100DE00081E092E10F9469759091030581E0892774
:100DF0000E944EBECD59DF4F0FB6F894DEBF0FBE36
:100E0000CDBFDF91CF911F910F91FF90EF90DF90B9
:100E1000CF90BF90AF909F908F907F906F905F909A
:100E20004F903F902F9008958531910509F4D9C0D6
:100E3000FCF48A30910509F423C50B9709F424C505
:100E40008091CB119091CC118F51904F9F938F93A4
:100E50001F9287E48F9384EF96E69F938F930F946E
:100E60003F9F0F900F900F900F900F900F90B9C071
:100E70008C31910509F40AC54E9711F70F9414228D
:100E800081E0809305120E9479608C0180E090E0FF
:100E9000A8E4B4E480937A0290937B02A0937C024E
:100EA000B0937D0243E060E070E080E291EC0F944B
:100EB0009C567090FD116090FE115090FF11409073
:100EC0000012B090F911A090FA119090FB1180904F
:100ED000FC11F090F511E090F611D090F711C09050
:100EE000F8118FE296E50E943C6D4F925F926F92EF
:100EF0007F928F929F92AF92BF92CF92DF92EF92AA
:100F0000FF929F938F938DEA97E69F938F930F9411
:100F10003F9FC8010E945F60109205120FB6F894BF
:100F2000DEBF0FBECDBF5DC08835910509F459C045
:100F3000F4F48135910511F40C94A4905CF48C3494
:100F4000910509F40CC58035910509F079CF0E940F
:100F5000907E47C08635910511F40C94A890873592
:100F6000910509F06DCF80E10E9480C63AC08C35B2
:100F7000910511F40C94B49074F48A35910511F430
:100F80000C94AD908B35910509F05ACF8091EB11FF
:100F900087600C94B0908236910511F40C944B91BB
:100FA0008336910509F04CCF1092CA0D60E084ECB5
:100FB0009FE00F94A1A082E00E94CD690C945A9109
:100FC0002DEC3CEC4CEC5DE3C701B6010F942EA474
:100FD000181624F4809103058111F0CEC8010E94F7
:100FE0008F651092580310925703C4CC0E9400558D
:100FF0002E969FAF8EAF2E970E94B55B89E40E941C
:10100000B655882309F4A0C30E948E5A60934F03FB
:101010007093500380935103909352038AE40E948B
:10102000B655C12CD12C7601882321F00E948E5A0E
:101030006B017C01C0925303D0925403E09255039C
:10104000F0925603E0915703F0915803A496FFAF36
:10105000EEAFA49780904F0390905003A09051035F
:10106000B0905203A7019601C501B4010F9441A4A9
:1010700024966CAF7DAF8EAF9FAF249760918E02A8
:1010800070918F02072E000C880B990B0F940B9B0D
:1010900020917A0230917B0240917C0250917D0236
:1010A0000F944A9B2EE333EC4EE259E30F944A9B94
:1010B00068AF79AF8AAF9BAF80E1E5EFF1E1DE0188
:1010C000119601900D928A95E1F7A501940150586F
:1010D00028A739A74AA75BA7D701C601B0588CA794
:1010E0009DA7AEA7BFA729813A814B815C81289635
:1010F0002CAF3DAF4EAF5FAF2897C501B4010F9441
:10110000A5A162966CAF7DAF8EAF9FAF62978D81C8
:101110009E81AF81B8852C968CAF9DAFAEAFBFAF2F
:101120002C979C01AD01C701B6010F94A5A166964D
:101130006CAF7DAF8EAF9FAF669729853A854B85A3
:101140005C8560919B0670919C0680919D069091B4
:101150009E060F94A4A16A966CAF7DAF8EAF9FAF31
:101160006A9720919306309194064091950650918C
:1011700096066E962CAF3DAF4EAF5FAF6E97629600
:101180002CAD3DAD4EAD5FAD62976E966CAD7DAD55
:101190008EAD9FAD6E970F94A4A16B017C018091E1
:1011A000970690919806A0919906B0919A06A296FA
:1011B0008CAF9DAFAEAFBFAFA29766962CAD3DADE5
:1011C0004EAD5FAD6697BC01CD010F94A4A14B015C
:1011D0005C013090F6042090F7049091F8049CABE9
:1011E000A091F904ACAFB091FE04B8ABA701960191
:1011F00068A579A58AA59BA50F944A9B2B013C0164
:10120000A50194016CA57DA58EA59FA50F944A9B71
:101210009B01AC01C301B2010F94A5A12B013C01BC
:10122000A501940168A579A58AA59BA50F944A9B61
:101230004B015C01A70196016CA57DA58EA59FA51C
:101240000F944A9B9B01AC01C501B4010F94A4A16A
:10125000A30192010F9424A26B017C0120E030E0F5
:10126000A9010F949AA287FF0AC02BED3FE049EC39
:1012700050E4C701B6010F94A5A16B017C016091F8
:10128000FF04709100056115710509F461C290E0D9
:1012900080E00F94099B9B01AC016BED7FE089EC32
:1012A00090E40F94A4A224962CAD3DAD4EAD5FAD5D
:1012B00024970F944A9B5B018C016091010570910A
:1012C000020561157105E1F090E080E00F94099B43
:1012D00020E030E040E752E40F944A9B9B01AC01D0
:1012E00068AD79AD8AAD9BAD0F94A4A23B014C01D2
:1012F0009501A8010F949AA287FF02C053018401AF
:101300004090FA045090FB046090FC047090FD043F
:101310009501A801B201C3010F942EA4181684F000
:101320009501A801632D722D8CA99CAD0F949AA2F2
:101330002501380187FF04C0432C522C6CA87CACDB
:10134000A496EEADFFADA497329751F42BED3FE09C
:1013500049EC50E4C701B6010F94A4A16B017C01D4
:101360006E962CAD3DAD4EAD5FAD6E9728966CADD3
:101370007DAD8EAD9FAD28970F949AA2811123C0A9
:10138000A2962CAD3DAD4EAD5FADA2972C966CAD47
:101390007DAD8EAD9FAD2C970F949AA2811113C095
:1013A00020E030E0A901C701B6010F949AA2811193
:1013B0000AC02BED3FE049EC50E4C701B6010F94A1
:1013C000A5A16B017C01A701960124966CAD7DADB2
:1013D0008EAD9FAD24970F944A9B6A962CAD3DAD80
:1013E0004EAD5FAD6A970F9441A44B015C012FE6AF
:1013F00032E143E85AE30F949AA287FD9EC192011D
:10140000A301C501B4010F94A4A20F9483A20F9469
:101410001DA37DAB6CAB6230710508F45EC12E96E6
:101420004EAD5FAD2E97452B09F457C190E080E09B
:101430000F94099B4B015C01AC019B01C701B601F4
:101440000F94A4A22B013C01A50194016A966CADF6
:101450007DAD8EAD9FAD6A970F94A4A228966CAF18
:101460007DAF8EAF9FAF28972D853E854F855889DC
:1014700060919F067091A0068091A1069091A206AE
:101480000F94A4A1A50194010F94A4A22C966CAF73
:101490007DAF8EAF9FAF2C97A3019201C301B20124
:1014A0000F944A9B6B017C01AC019B01C301B2010B
:1014B0000F944A9B20E030E040EC50E40F94A4A24B
:1014C0009B01AC01C301B2010F94A4A16CAF7DAF2D
:1014D0008EAF9FAF20E030E040E05FE3C701B60190
:1014E0000F944A9B9B01AC0160E070E080E89FE3B1
:1014F0000F94A4A124966CAF7DAF8EAF9FAF2497BD
:1015000022242394312CD8A8DA9458A9511125C14A
:10151000B10190E080E00F94099BA30192010F9428
:101520004A9B6B017C010F949FA26CA77DA78EA79D
:101530009FA7C701B6010F9465A54B015C01C09040
:101540004F03D0905003E0905103F0905203F7FA0C
:10155000F094F7F8F0948091530390915403A09184
:101560005503B091560388AB99ABAAABBBABA701AF
:1015700096016CA57DA58EA59FA50F944A9B68A793
:1015800079A78AA79BA728A939A94AA95BA9C50158
:10159000B4010F944A9B9B01AC0168A579A58AA56B
:1015A0009BA50F94A5A168A779A78AA79BA7A701C8
:1015B0009601C501B4010F944A9B6B017C0128A9D7
:1015C00039A94AA95BA96CA57DA58EA59FA50F94F5
:1015D0004A9B9B01AC01C701B6010F94A4A16CA763
:1015E0007DA78EA79FA79091FE0498AB28A539A54B
:1015F0004AA55BA562966CAD7DAD8EAD9FAD629741
:101600000F94A5A169837A838B839C832CA53DA528
:101610004EA55FA566966CAD7DAD8EAD9FAD669710
:101620000F94A5A16D837E838F83988728962CAD18
:101630003DAD4EAD5FAD289769857A858B859C85DC
:101640000F94A5A169877A878B879C872C962CADF0
:101650003DAD4EAD5FAD2C976D857E858F859889AC
:101660000F94A5A16D877E878F87988BCE010196F9
:101670000E9450652E96AEADBFAD2E972A163B0642
:10168000F8F0E984FA840B851C852D813E814F8119
:10169000588569817A818B819C813F922F92E5EFF9
:1016A000F1E1FF93EF9388AC99ACAAACBBACFE011F
:1016B0003D966F010F94C3750F900F900F900F9090
:1016C0008091AC0D811139C0FFEF2F1A3F0A2CA970
:1016D0003DA92215330509F016CF83E996E00E9453
:1016E0005065E0909B06F0909C0600919D0610913D
:1016F0009E06209197063091980640919906509148
:101700009A06609193067091940680919506909147
:1017100096061F921F92E5EFF1E1FF93EF9388ACDD
:1017200099ACAAACBBACEFE9CE2EE6E0DE2E0F946E
:10173000C3750F900F900F900F900E9437558AE459
:1017400093E00F9473114DCC60E070E0CB015ECC60
:10175000A32CB22C0CA91CADB0CD28A539A54AA547
:101760005BA56CAD7DAD8EAD9FAD0F944A9B4B01DB
:101770005C012CA53DA54EA55FA524966CAD7DAD65
:101780008EAD9FAD24970F944A9B9B01AC01C50180
:10179000B4010F94A5A17B018C0128A539A54AA508
:1017A0005BA524966CAD7DAD8EAD9FAD24970F9457
:1017B0004A9B4B015C012CA53DA54EA55FA56CADD8
:1017C0007DAD8EAD9FAD0F944A9B9B01AC01C501D1
:1017D000B4010F94A4A168A779A78AA79BA7D8AA48
:1017E000C701D8018CA79DA7AEA7BFA7FFCE80E5F4
:1017F0000E94B655C12CD12C7601882331F00E946D
:101800008E5A0F941DA36B017C0183E50E94B6558F
:10181000882361F00E948E5A20E030E04AE754E4C9
:101820000F944A9B0F941DA36B017C01C114D1043A
:10183000E104F10441F08091C706873021F089EC82
:1018400097E60E945FE60F9414220F94460FC60E8F
:10185000D71EE81EF91E8AE493E00F9473110F94CB
:10186000460F6C157D058E059F0508F0BACB0F94C9
:10187000F73180E00E948C7A80E00E94CD69EFCF42
:1018800081E00E944EBEADCB80E0FBCF88E50E9498
:10189000B655382E412C512C3201882321F00E945C
:1018A0001E562B013C0189E50E94B655282E88233F
:1018B00071F10E941E566CA77DA78EA79FA78AE58F
:1018C0000E94B655D82E812C912C5401882321F0EA
:1018D0000E941E564B015C0187E50E94B65588A701
:1018E0008F93CD2CECA4FDA40EA51FA5222DB30132
:1018F000A201832D0E94FE670F90311072CB211040
:1019000070CB38A531116DCBD1106BCB20CB1CA681
:101910001DA61EA61FA6D3CF08E210E094EAE92E6A
:1019200097E6F92E602F70E090E080E00F94099B1D
:101930000E948F569F938F937F936F931F930F9364
:10194000FF92EF920F943F9F0F5F1F4F0FB6F894D7
:10195000DEBF0FBECDBF0F36110521F742CB0F946E
:101960008414811105C081E391E80E94DE7239CBB5
:1019700082E00E944FD8811107C08BE29AE30E9457
:101980003C6D0F94190B2DCB8091A306882341F059
:101990008091A406882321F0D090A506D11008C01C
:1019A00081E08093E61186EB98E60F94F54219CB1F
:1019B00082EE99E30E943C6D0F94190B8BE991E53F
:1019C0000E943C6D41E060E00F94892D81116EC052
:1019D00080E090E0A0EAB0E48093FD119093FE11C6
:1019E000A093FF11B093001260E070E088E492E4ED
:1019F0000F94118580E090E0A8E4B2E48093FD119B
:101A00009093FE11A093FF11B093001280E090E03C
:101A1000A4E3B3E48093F9119093FA11A093FB111E
:101A2000B093FC1160E070E088E492E40F941185BB
:101A30000F94142281E791E50E943C6D0F94190BDD
:101A4000E3E5F9E885919591A591B4918093F91119
:101A50009093FA11A093FB11B093FC11EFE4F9E815
:101A600085919591A591B4918093F5119093F6117C
:101A7000A093F711B093F81160E070E088E492E46D
:101A80000F9411850F94142281E08F93812C912C57
:101A90005401CC24C394E12CF12C870120E040E0D8
:101AA00050E0BA0180E00E94FE670F9020E030E035
:101AB0004CE052E460918E0670918F068091900602
:101AC000909191060F942EA418160CF076C0809178
:101AD000CA0D811172C080E090E0A8ECB2E480935E
:101AE000FD119093FE11A093FF11B093001260E0DE
:101AF00070E088E492E40F9411850F9431121982FA
:101B00001A821B821C821D82CE0101960F947311D2
:101B100083E2F82E0EEA1EE720E030E04CE052E4CB
:101B200060918E0670918F0680919006909191063B
:101B30000F942EA41816C4F584E999E30E943C6D15
:101B40000F94920A42E864E080E00E94266A1F92A5
:101B5000FF9260918E0670918F0680919006909111
:101B600091060F9416A37F936F931F930F930E9478
:101B7000DF6981E80E94F56988EE93E00E94D37CDA
:101B80000E94F37040E053E567E070E0CE010196FB
:101B90000F94B40F0F900F900F900F900F900F9025
:101BA000882309F4B9CFD12C81E00E944B6AD1106F
:101BB00004C080E00F94AA0B14CA0F94142281E091
:101BC000809305120E944B6A83E191E80E94DE72C5
:101BD00080908E0690908F06A0909006B09091060F
:101BE00020E030E040EA50E4C501B4010F94A4A223
:101BF0000F9416A325E0269FA001279F500D1124C6
:101C0000BA01550F880B990B0F940B9B1B017C019C
:101C100020E030E04CE052E40F949AA287FF06C027
:101C2000212C312C1CE0E12E02E4F02E222D332D4C
:101C30004E2D5F2DC501B4010F942EA4181664F427
:101C400020E030E040EA50E4622D732D8E2D9F2D70
:101C50000F94A5A11B017C01FF92EF923F922F925E
:101C60008BE897E69F938F930F943F9F20E030E09F
:101C700040EF51E4622D732D8E2D9F2D0F94A4A162
:101C800020E030E04CE852E40F94A5A10F9416A395
:101C90007093EE116093ED1184E08093C70681E0AC
:101CA0008093AC0386E39BE30E943C6D0E945FE659
:101CB00080E090E0A0EAB0E48093FD119093FE11E3
:101CC000A093FF11B093001260E070E088E492E40A
:101CD0000F94118580E090E0A0EAB1E48093F511C3
:101CE0009093F611A093F711B093F81180E090E073
:101CF000A0E7B2E48093F9119093FA11A093FB113D
:101D0000B093FC1160E070E088E492E40F941185D8
:101D10008AE999E9A9E1BEE38093FD119093FE1150
:101D2000A093FF11B093001260E070E088E492E4A9
:101D30000F9411850F9414220F900F900F900F9015
:101D40000F900F9020918E0630918F064091900653
:101D500050919106622D732D8E2D9F2D0F942EA4E0
:101D600018163CF488EE93E00E94D37C0E94F37036
:101D7000E9CF60E086EA9FE00F94A1A080E090E0C8
:101D8000A0EAB0E48093FD119093FE11A093FF119F
:101D9000B093001260E070E088E492E40F94118543
:101DA000EFE4F9E885919591A591B4918093F511AF
:101DB0009093F611A093F711B093F811E3E5F9E8C9
:101DC00085919591A591B4918093F9119093FA1111
:101DD000A093FB11B093FC1160E070E088E492E402
:101DE0000F9411850F94142243E060E070E080E8C6
:101DF0009FEB0F949C56811105C00F94AA0B109273
:101E00000512EFC89091FD1198A7A091FE11ACA703
:101E1000B091FF11B8ABE0910012E8AFEF93BF9320
:101E2000AF939F938EE797E69F938F930F943F9F77
:101E30000F900F900F900F900F900F90AEEA8A2E98
:101E4000AFE09A2EB3E2CB2ED12C0FEF1FEFB601ED
:101E50000D2C000C880B990B0F940B9B2B013C0154
:101E6000DF92CF92C80102969F938F9322E437E6C8
:101E70003F932F930F943F9F58015FEFA51AB50A28
:101E80000F900F900F900F900F900F9011F40C94F3
:101E900027B070E060E0C4010F94BFA0A3019201DD
:101EA000622D732D8E2D9F2D0F949AA2181644F437
:101EB00085E0A816B10411F00C9433B005E010E0F1
:101EC000580197E2A91A98EFB90AAA0CBB1C85E041
:101ED000809F1001819F300C11240D5F1F4FEAE994
:101EE0004E2EE9E95E2EE9E16E2EEEE37E2EF9E05C
:101EF0008F2EF7E69F2EC801029705970CF0D4C0ED
:101F0000B101635D7F4F072E000C880B990B0F9476
:101F10000B9B6B017C011F930F93A5E3B7E6BF9367
:101F2000AF930F943F9F0093AC0320E030E040EF6D
:101F300051E4C701B6010F94A4A120E030E040E2D3
:101F400051E40F944A9B20E030E040EA50E40F94C3
:101F5000A4A220E030E048E452E40F94A5A10F943D
:101F600016A37093EE116093ED1180E090E0A0EA6B
:101F7000B0E48093FD119093FE11A093FF11B093F4
:101F8000001260E070E088E492E40F94118520E094
:101F900030E040EA51E42093F5113093F61140937C
:101FA000F7115093F81180E090E0A0E7B2E480933D
:101FB000F9119093FA11A093FB11B093FC1160E01A
:101FC00070E088E492E40F9411854092FD115092E4
:101FD000FE116092FF117092001260E070E088E4E0
:101FE00092E40F9411850F9414220F900F900F908C
:101FF0000F9020918E0630918F064091900650915F
:102000009106C701B6010F942EA418163CF488EE71
:1020100093E00E94D37C0E94F370EBCF80E090E0CD
:10202000A0EAB0E48093FD119093FE11A093FF11FC
:10203000B093001260E070E088E492E40F941185A0
:10204000EFE4F9E885919591A591B4918093F5110C
:102050009093F611A093F711B093F811E3E5F9E826
:1020600085919591A591B4918093F9119093FA116E
:10207000A093FB11B093FC1160E070E088E492E45F
:102080000F9411850F94142243E060E070E080E823
:102090009FEB0F949C5695E0290E311C0F5F1F4F4C
:1020A000811104C00F94AA0B81E0A7CE78A56CA57E
:1020B00098A988AD272F362F492F582F6091FD11F1
:1020C0007091FE118091FF11909100120F94A4A1C4
:1020D000F62EE72ED82EC92E20913E0430913F04D3
:1020E0004091400450914104D701F6016B2F7A2FA3
:1020F0008F2F9E2F0F944A9B0F9416A36CAB7DAB32
:102100008EAB9FABCF92DF92EF92FF9280919106C0
:102110008F93809190068F9380918F068F938091FB
:102120008E068F939F928F920F943F9F6CA97DA9EB
:10213000C5010F94BFA0A2E0AA0EB11C0FB6F8947F
:10214000DEBF0FBECDBFD7CE0E94C2730C94F18705
:1021500080E10E942BC60C94F1878091EB11887F5F
:102160008093EB110C94F18754ECC52E52E0D52EE0
:102170008E010C5D1F4F5801EE24E394F12CD60123
:102180008D916D010E94B655F50181935F01882301
:1021900091F00E948E5AF701EE0FFF1FEE0FFF1F06
:1021A000349721E030E02C0F3D1FE20FF31F6083D6
:1021B0007183828393833FEFE31AF30A45E0E416C9
:1021C000F104E9F69FA0FCA0992001F120E030E0A5
:1021D000A9016D857E858F8598890F949AA28111BA
:1021E00015C0F11013C08DA1811110C08EA18111F5
:1021F0000DC010920112109202121092031210924E
:10220000041281E08093EF030C94F1870F94142261
:10221000CE0101965C012AE8C22E24E0D22E35EFD1
:10222000E32E31E1F32E380193E0690E711CD801E1
:102230008D918D01882389F0F601208131814281C1
:102240005381D5016D917D918D919C910F94A5A1A4
:10225000F7016083718382839383F4E0AF0EB11C36
:1022600024E0C20ED11C34E0E30EF11C60167106AE
:10227000F1F6992061F08D859E85AF85B8898093B0
:10228000011290930212A0930312B09304120F94C0
:10229000D1830C94F18781E08093CA0D61E084ECD6
:1022A0009FE00F94A1A01092890360E08FEF9FE060
:1022B0000F94A1A00E945CD80C94F1878D3411F08A
:1022C0000C9429AF1093F6160093F516F801319689
:1022D00081918032E9F38930D9F380538A3030F02C
:1022E0001F930F938FEF90E80C94A9840E94D85508
:1022F0009093AB0D8093AA0D8E3B910511F40C9435
:10230000369C0CF007C38C34910511F40C944F9B50
:102310000CF0DEC18C31910511F40C9486990CF00F
:10232000F4C08531910509F40AC70CF05AC0813117
:10233000910509F4F9C6DCF4029708F45DC68091B2
:10234000CB119091CC118F51904F9F938F931F92EF
:102350008DE48F9384EF96E69F938F930F943F9F26
:102360000F900F900F900F900F900F90A8C6823192
:10237000910511F40C94E19C449709F781E0809356
:10238000780284EE96E60E94DE7284E50E94B655DD
:10239000182F8CE40E94B65500E080FB00F910FB7A
:1023A00001F980EF93E10E94C17083E2E0EFF3E175
:1023B000DE01119601900D928A95E1F720E050E040
:1023C00040E0BE016F5F7F4F8AED92E00F940745BA
:1023D000CE0101960E94C67086ED96E60E94DE72DE
:1023E0006EC68831910509F4BBC684F48631910527
:1023F00009F4A9C6479709F0A2CF8091F5169091EC
:10240000F61661E004960F94A44B59C68A319105E3
:1024100009F4ECC60CF00CC704EC12E0F2E4AF2EA9
:10242000F2E0BF2EA4E2CA2EA2E0DA2EB8E1EB2E33
:10243000B2E0FB2E87EC882E82E0982EF801819185
:102440008F010E94B655882321F10E948E5AD60131
:102450004D905D906D907C90A30192010F949AA293
:1024600087FD11C00E948E5AF70140805180628022
:102470007380A30192010F942EA4181624F00E94D9
:102480008E5A2B013C01D5014D925D926D927C924A
:102490001397B4E0AB0EB11CE4E0CE0ED11CF4E017
:1024A000EF0EF11C8016910649F683E50E94B655A1
:1024B000882311F40C94FFA80E94CB558111FFC50D
:1024C00080E090E0A8E4B2E480934202909343025B
:1024D000A0934402B093450280E090E0AEE3B3E401
:1024E0008093460290934702A0934802B09349021A
:1024F00080E090E0A0EAB1E480934A0290934B021E
:10250000A0934C02B0934D02DAC58C32910509F4C8
:10251000CEC70CF08FC08F31910509F49EC70CF027
:1025200052C08D31910509F4CAC54E9709F007CF05
:1025300080916B13882309F4C2C50F9482410091E6
:10254000F5161091F6160C5F1F4F80916B138823C0
:1025500009F4B5C58AEF95E10F94336F10926A13B1
:102560001DA30CA3CE0184960F941F4B882309F45E
:10257000A6C54CA15DA16091131470911414198229
:102580001C8222E0CE0101960F942A9A8111C6C6C0
:1025900010E0CE0101960E94C670112309F4D5C641
:1025A00084E79EE70E94E5708CA19DA10F949E99FF
:1025B00010927E1610927F1610928016109281163D
:1025C0000F94E3487CC58032910509F4CCC68A9704
:1025D00009F0B5CE83E50E94B655882309F46FC58E
:1025E0000E94CB55082F80E50E94B6551DE0882338
:1025F00019F00E94CB55182FE4EDF0E88491811773
:1026000009F45DC5319630E8E03FF307B9F71630BD
:1026100009F04AC70093E91161E0812F0E943BC095
:10262000602F812F0E940DC0602F70E0812F0E94CB
:102630006CC045C58F32910509F462C75CF58D32D7
:10264000910509F44DC78E9709F079CE8091DB157D
:10265000882309F450C7CE0101960F94285288238D
:1026600009F444C789810E94CC708EE20E94CC702C
:102670008A810E94CC708EE20E94CC708B810E9475
:10268000CC708EE20E94CC708C810E94CC700F9432
:102690009D9815C58934910509F45BC78B34910564
:1026A00011F40C94499B8834910509F048CE83E5D8
:1026B0000E94B655882309F43DC70E94CB55882354
:1026C00009F435C7813009F0FAC48093CB0DF7C403
:1026D0008B36910511F40C94D89C0CF083C0843592
:1026E000910511F40C94E19CBCF58F34910509F42B
:1026F000EEC71CF58D34910509F4E4C78E349105BD
:1027000009F01DCE89EA90E80E94E5708DEE9FE009
:102710000F9485A04AE00F94CD9683EA90E80E943A
:10272000E57081EF9FE00F9485A04AE00F94CD966D
:102730008EE990E80E94DE72C2C48235910511F4E0
:102740000C94DB9C8335910509F0F9CD8091EB1158
:1027500088608093EB11B3C48C35910511F40C940F
:102760004A9D34F58535910511F40C94319D8635DB
:10277000910509F0E4CD83E50E94B655882309F45C
:102780009EC40E948E5A20E030E04AE754E40F9441
:102790004A9B0F941DA3609333027093340280937D
:1027A0003502909336028AE196E00F94731187C444
:1027B0008936910509F4DEC714F00C94CA9C88365A
:1027C000910509F0BCCD83E50E94B655882309F434
:1027D00076C40E948E5A0F9416A37093F2116093E0
:1027E000F1116DC48537910511F40C94C89EB4F5B0
:1027F0008037910509F4ABC7CCF48D36910509F407
:10280000E5C78E36910509F09ACD8EE40E94B65543
:10281000882309F454C40E941E566093D11170930A
:10282000D2118093D3119093D41149C4823791056A
:1028300011F40C94C59E14F40C94D29D8337910529
:1028400009F07DCD86E50E94B655882311F40C94DD
:10285000F19D89ED9FE90E94DE7231C48B379105AD
:1028600011F40C94209F0CF048C08637910511F4A8
:102870000C94D89E8737910509F061CD80E196E6EA
:102880000E94E5700F949D9888E096E60E94E5709E
:102890001E9B02C00C94109F83E096E60E94E57098
:1028A0000F949D9881EF95E60E94E5701D9B02C0F4
:1028B0000C94149F83E096E60E94E5700F949D9817
:1028C00089EE95E60E94E5701C9B02C00C94189F4F
:1028D00083E096E60E94E5700F949D9881EE95E660
:1028E0000E94E570019902C00C941C9F83E096E65B
:1028F0000E94E5700F949D98E2C38C38910509F40D
:102900002AC78B39910509F441C78D37910509F024
:1029100016CD82CD843A41E0940711F40C943FA285
:102920000CF038C2823E910511F40C94C9A00CF051
:102930006BC18E3C910511F40C94DC9F0CF0B1C07E
:102940008B3C910511F40C94669F5CF5883C9105D5
:1029500011F40C94239F04EC12E0A2E3EA2EA4E00D
:10296000FA2EB8ECCB2EB2E0DB2E893C910509F0B3
:10297000E6CCD8018D918D010E94B655882349F08F
:102980000E948E5A0F941DA3F70164A375A386A31A
:1029900097A3F4E0EF0EF11CC016D10651F70C948A
:1029A000C79D8C3C910511F40C94859F8D3C91053D
:1029B00009F0C5CC83E50E94B655882351F00E94EA
:1029C0008E5A60936E0470936F048093700490939A
:1029D000710484E50E94B655882351F00E948E5AF6
:1029E00060937204709373048093740490937504DD
:1029F00082E40E94B655882361F00E948E5A0F949B
:102A00001DA3609376047093770480937804909369
:102A1000790488E50E94B655882391F00E948E5A69
:102A200060937E0470937F0480938004909381046C
:102A300060937A0470937B0480937C0490937D046C
:102A400089E50E94B655882351F00E948E5A609302
:102A50007E0470937F0480938004909381048AE5C0
:102A60000E94B655882351F00E948E5A60938204CA
:102A700070938304809384049093850485E40E947A
:102A8000B655882309F41BC30E948E5A0E940E7407
:102A900060938604709387048093880490938904DC
:102AA0000EC3813D910511F40C9429A05CF58F3C77
:102AB000910511F40C94F89F803D910509F03FCCED
:102AC00083E50E94B655882351F00E948E5A609388
:102AD000C1047093C2048093C3049093C40486E439
:102AE0000E94B655882309F4EAC20E948E5A0E94B9
:102AF00058606093C5047093C6048093C704909394
:102B0000C804DDC28C3D910511F40C9469A08D3D83
:102B1000910511F40C94A8A0863D910509F00FCC05
:102B200080E50E94B655882311F40C9455A00E94AC
:102B30008E5A2B013C0183E50E94B655882311F47F
:102B40000C945FA00E948E5A4B015C018EE40E949F
:102B5000B655D090FE04882329F00E948E5A0F9417
:102B60001DA3D62E82E50E94B655E090FF04F0909A
:102B70000005882329F00E948E5A0F941DA37B0123
:102B800086E40E94B6550091010510910205882344
:102B900029F00E948E5A0F941DA38B0120E030E093
:102BA000A901C301B2010F949AA218160CF087C2B2
:102BB00020E030E0A901C501B4010F949AA287FD7D
:102BC0007EC2A5019401C301B2010F949AA287FDB0
:102BD00076C24092F6045092F7046092F804709224
:102BE000F9048092FA049092FB04A092FC04B09243
:102BF000FD04D092FE04F0920005E092FF041093D1
:102C00000205009301055BC28033A1E09A0711F42D
:102C10000C94A4A10CF06CC08D32E1E09E0711F47D
:102C20000C942BA154F5803F910509F448C28C32D5
:102C3000914009F084CB80E50E94B65508EE13E080
:102C4000882329F00E948E5A0F941DA38B0183E5DF
:102C50000E94B655882311F40C9423A10E948E5A29
:102C60000F941DA36115710511F00C9425A1B801F5
:102C700090E080E00F944D0D22C28E3231E0930738
:102C800011F40C941DA28F32914009F058CB85E4C9
:102C90000E94B65510E000E0882359F00E94D855F4
:102CA0008C01C12CD12C5CE8E52E52E4F52E97FD69
:102CB00006C0C12CD12C66E1E62E63E4F62E83E536
:102CC0000E94B655882321F00E948E5A6B017C0128
:102CD00083E40E94B655882311F40C942DA20E941F
:102CE000D8559C01A801C701B6010F949518E7C1FA
:102CF000803951E0950711F40C9431A204F58E351A
:102D0000B1E09B0711F40C9455AD8F35914009F05B
:102D100016CB83E50E94B655882371F00E948E5A27
:102D20000F9416A36130710511F40C948BAD6230D1
:102D3000710511F40C94ADAD0F947020C0C18539AC
:102D4000F1E09F0711F40C9435A2863921E0920737
:102D500011F40C943AA28339914009F0F0CA8091A1
:102D60009412813009F0ABC185E40E94B6558111FF
:102D70000E94CB5586E40E94B65581110E94CB5526
:102D80000F945554882309F49AC160E080E00F94B1
:102D9000696A95C1803C42E0940711F40C949CAEA2
:102DA0000CF057C08832A2E09A0711F40C94E0A40A
:102DB0004CF5863FE1E09E0711F40C9447A26CF4B9
:102DC000843F21E0920711F40C9443A2853F914087
:102DD00009F0B5CA0E946C7572C1873F41E0940743
:102DE00011F40C944BA28D3F914009F0A8CA0E94A7
:102DF0003F6C87E79EE90E94E57086EA9FE70E94A4
:102E0000E5705DC18A35A2E09A0711F40C940EA911
:102E10005CF48835E2E09E0711F40C9415A5893521
:102E2000924009F4F9CA8BCA8D3B22E0920711F453
:102E30000C94C6AD8E3B32E0930711F40C9468AE4F
:102E40008B35924009F07BCA60E080E00E9464EF1D
:102E500036C18C3553E0950711F40C9430AA0CF070
:102E600042C0833CB2E09B0711F40C94A8AE7CF402
:102E7000813CF2E09F0711F40C94A2AE823C924098
:102E800009F05DCA82EC92E00E94545A18C1853C58
:102E900032E0930711F40C94F1AE14F40C94C5AE27
:102EA0008235934009F04BCA188683E50E94B655D7
:102EB000882311F40C9416A90E94CB55182F883042
:102EC00010F40C941BA982E89FE70E94E5704AE089
:102ED00067E070E080E090E00F94CD968AED92E09C
:102EE0000F949E99ECC08438A3E09A0711F40C94D7
:102EF000A6AC0CF04DC08D35E3E09E0711F40C94A8
:102F0000BAAA8E35934009F01ACA0E948E5A20E060
:102F100030E040E251E40F944A9B0F941DA36C5A99
:102F2000633011F40C94C0AB10F00C9452AB6130D0
:102F300011F40C947BAB623009F0C1C08091941203
:102F4000E7EBF9E7813011F0E9EBF9E7059114912E
:102F500080E50E94B655882311F40C94AFAB0E9413
:102F60001E56F090B803FF2009F4A9C0601771073E
:102F700009F4A5C089EC97E30E943C6D8C0181E9BE
:102F800097E30E943C6D4F2DB8010E94B1EF97C0AE
:102F90008C3823E0920709F492C0803A33E093071B
:102FA00009F450C28B38934009F0C9C988E50E94E2
:102FB000B655882339F00E948E5A0F9416A380E0EC
:102FC0000F9461218AE50E94B655882339F00E944A
:102FD0008E5A0F9416A381E00F94612185E40E941C
:102FE000B655882309F46BC00E948E5A0F9416A31D
:102FF000CB010F94612063C00091F5161091F61675
:103000000E5F1F4F80E50E94B655C12CD12C760172
:10301000882321F00E941E566B017C0183E50E94EB
:10302000B655882351F00E941E569B01AC01A8EEB4
:10303000B3E00F9412A16B017C01C8010F5F1F4F19
:10304000DC014C914032C9F326E02093C706C1143D
:10305000D104E104F104C9F52C912223B1F10E94BD
:1030600053EF0F9414228091CD1184608093CD1181
:103070008AE493E00F947311C114D104E104F104C4
:10308000D9F10F94460FC60ED71EE81EF91E84E034
:10309000809378020F94460F6C157D058E059F0571
:1030A00010F182E0809378028091CD118B7F809324
:1030B000CD1180916A13882391F11092C706109266
:1030C000AB0D1092AA0D0C94BA848091CA0D811197
:1030D00007C08FEC99E30E943C6D0E945FE6C1CF70
:1030E0001092C706BECF0E94236C8111DACF90E008
:1030F00080E00E94D37CCECF1091780284E0809350
:1031000078020E941E6C0E94236C811105C090E021
:1031100080E00E94D37CF7CF10937802C5CF8BE07C
:103120009CE60E945FE6CBCF84EC99E30E943C6D65
:103130000E945FE61798169815981498C0CF81E002
:103140000F941B4DBCCF10926A1310926B1387E73C
:103150009EE90E94E5708DE898E60E94DE72AFCF8E
:103160000E944861882319F00E9424EFA8CF0E9492
:10317000C2EF882309F4A3CF8091FD15882361F065
:1031800080917E1690917F16A0918016B091811645
:10319000892B8A2B8B2B69F40E9429561092DC1103
:1031A0001092DD111092DE111092DF1180E00E946A
:1031B000737480916B13882331F081E080936A13DC
:1031C00085E08093CB0D0F9428208091941281305C
:1031D00009F075CF80916A12882309F470CF0E949C
:1031E000F7C381116CCF0F94346B69CF80916B134F
:1031F000882309F464CF83E50E94B655882309F437
:103200005ECF0E941E566B017C01C0927E16D0924A
:103210007F16E0928016F09281160F949443C0922C
:10322000DC11D092DD11E092DE11F092DF1147CF78
:1032300080E50E94B655182F0E944861882391F0BE
:103240008091E711882349F080917902811105C0AE
:103250008EE99EE70E94DE7232CF82E99EE70E94ED
:10326000DE722DCF80916A13882309F44AC011239E
:10327000E1F10F9419480F949D9882EA95E60E9417
:10328000E57060917E1670917F1680918016909106
:1032900081164AE00F94CD968FE20E94CC70609127
:1032A0007716709178168091791690917A164AE087
:1032B0000F94CD960F949D980F94381C2CE330E01A
:1032C00040E050E00F94F0A0C9016CE370E00F946F
:1032D00046A18C0190E080E00F9443978AE30E941E
:1032E000CC70C8010F944841EACE809181138823A5
:1032F00029F081E893E10F949E99BFCF8CE693E18A
:10330000FACF82E89EE70E94DE72D9CE8091F51650
:103310009091F61604960F94C051D1CECE0101962D
:103320000F947544882309F433C961E0CE010196F6
:103330000F943C6F009709F42BC925EEFC01208304
:103340001C820F94CA35182F24C98CE59EE70E9471
:10335000E5708CA19DA10E942E7D8EE20E94CC7012
:103360000F949D98ACCE80916A1381110F94142212
:103370000091F5161091F6160C5F1F4F61E270E098
:10338000C8010F94D4A6009719F08C010F5F1F4F4E
:1033900080E50E94B655F82E8091F5169091F616AC
:1033A0000817190708F4F12C80916B13882309F48E
:1033B00086CE61E06F25C8010F94A44B83E50E947F
:1033C000B655882399F08091F5169091F6168017DE
:1033D000910760F40E941E5660937E1670937F16CC
:1033E00080938016909381160F94944380916B1371
:1033F000882331F081E080936A1385E08093CB0DC0
:10340000F1105DCE8091FD15882361F080917E16CC
:1034100090917F16A0918016B0918116892B8A2BEE
:103420008B2B69F40E9429561092DC111092DD1149
:103430001092DE111092DF1180E00E9473740F94DD
:1034400028203DCE8091F5169091F61621E020932C
:10345000691305960F94C05132CE0F94381C2CE39B
:1034600030E040E050E00F94F0A07F936F933F93E3
:103470002F9380EF90E89F938F938E010F5F1F4FE4
:103480001F930F930F94949F87E79EE90E94E57026
:10349000C8010F949E99C8010E9453EF0FB6F8948B
:1034A000DEBF0FBECDBF0BCE17FD09CEB5C880E184
:1034B0000E942BC681EA9DE00F947DA04BE0849F83
:1034C000C001112470E060E0805B924F0F94BFA0B8
:1034D00082E00E942BC60F941C900F94FD8FEFCDBD
:1034E0008AE50E94B6550E948DC6E9CD84EB90E82E
:1034F0000E94E570E4CD80EB90E80E94DE72DFCDA3
:1035000084E0809378020E94396A0E941E6C0F94B6
:10351000F73181E00E948C7A0F94160A0E94236C86
:103520008823A9F30E94396A0E94E9FDC8CD109250
:10353000CB0DC5CD8091CB0D1F928F9384EC96E679
:103540009F938F930F943F9F0F900F900F900F902A
:10355000B6CD80E50E94B655882321F00E94CB5558
:103560008093710282E50E94B655882341F00E9443
:103570008E5A0F941DA3709375026093740281E5B7
:103580000E94B655882321F00E94CB5580933F02BC
:1035900083E50E94B655882341F00E948E5A0F940D
:1035A0001DA370933E0260933D0283E40E94B655D2
:1035B0008823A9F00E948E5A6B017C0120E030E044
:1035C000A9010F949AA26FEF7FEF181624F4C70198
:1035D000B6010F941DA3709373026093720284E48A
:1035E0000E94B6558823A9F00E948E5A6B017C0177
:1035F00020E030E0A9010F949AA26FEF7FEF181638
:1036000024F4C701B6010F941DA370933C0260938C
:103610003B02809173028F93809172028F9380910D
:1036200075028F93809174028F9380917102282F7D
:10363000082E000C330B3F938F938AE696E69F93F8
:103640008F9301E716E61F930F930F943F9F80918E
:103650003C028F9380913B028F9380913E028F9327
:1036600080913D028F9380913F02282F082E000CFD
:10367000330B3F938F9383E696E69F938F931F932D
:103680000F930F943F9F0FB6F894DEBF0FBECDBFD0
:1036900016CD0E94C2EF882309F411CDD0CE8091BF
:1036A0005903813009F00BCD82E0809359030F94C8
:1036B000460F609378067093790680937A0690930C
:1036C0007B06FDCC0F944C200E94C35FF8CC8AE5AA
:1036D00093E00F94731183E50E94B655882309F196
:1036E00062E270E08091F5169091F6160F94D4A6E0
:1036F0008C01892BB1F00F5F1F4F62E270E0C801AF
:103700000F94D4A6892B69F0E2E7F6E083E0DF01AD
:103710001D928A95E9F742E050E0B801CF010F947D
:10372000FDA68CE89FE00F947DA0813009F0C7CC06
:103730000E943E61882309F4C2CC0E94486188231C
:1037400009F4BDCC86E496E60E94DE72B8CC89E22C
:1037500096E60E946A7383E50E94B655882309F4B1
:10376000AECC0E948E5A0F9416A37093EE11609304
:10377000ED11A5CC8AE990E80E94E5700E9457728D
:103780000E945E7081E08093E61199CC83E50E94EF
:10379000B655882351F00E94CB558093621388233D
:1037A00071F083E693E10F94731183E40E94B655A0
:1037B000882341F00E94CB558093611380CC1092F6
:1037C0006313F3CF81E08093611379CC80E799E4B0
:1037D0000E943C6D0E945FE681E0809399030F9404
:1037E000A09883E50E94B655882349F00E948E5A1E
:1037F0000F9416A37093F2116093F11105C082E546
:103800000E94B6558111F2CF0F94460F6B017C01D7
:103810006091F1117091F211072E000C880B990B39
:103820000F940B9B11E02091C40D3091C50D409178
:10383000C60D5091C70D0F942EA418160CF010E071
:103840001093C30DC701B6010F94364E80E699E47C
:103850000E943C6D0E945FE682E0809399030F9482
:10386000A0988AE493E00F94731129CC82E599E43F
:103870000E943C6D0E945FE683E08093990381E0A3
:103880000F94A09883E50E94B655182F882349F01D
:103890000E948E5A0F9416A37093EE116093ED114F
:1038A00005C082E50E94B6558111F2CF0F94460FF4
:1038B0006B017C011092C90D6091ED117091EE11B8
:1038C000072E000C880B990B0F940B9B01E02091A5
:1038D0008A0330918B0340918C0350918D030F9498
:1038E0002EA418160CF000E00093C30D8091C90DB2
:1038F00081111AC06091ED117091EE11072E000C2C
:10390000880B990B0F940B9B20918A0330918B03AA
:1039100040918C0350918D03E091C30DEE2391F003
:103920000F942EA41816A4F087E499E40E943C6D2D
:103930000E945FE684E0809399038AE493E00F9409
:103940007311BDCB0F949AA287FFEECF1111ECCF6C
:103950008091C80D823041F30F94460F6C197D0998
:103960008E099F09693E73408105910550F0809151
:10397000CA0D811102C00E94F3700F94460F6B01B3
:103980007C010F94F73180E00E948C7A80E00E94E5
:10399000CD69ACCF83E50E94B655882329F00E94FB
:1039A000CB558093E9118BCB8FEF8093E91187CBB7
:1039B0001092E91184CB8091EB11877F8093EB11FA
:1039C0007ECB83E50E94B655882399F00E948E5ADB
:1039D00020E030E04AE754E40F944A9B0F941DA383
:1039E00060933702709338028093390290933A02C1
:1039F00066CB88E50E94B6558823D1F00F94142237
:103A000088E50E94B655811128C089E50E94B65507
:103A1000882319F0169A1092A4068AE50E94B655DA
:103A200085E40E94B655882309F449CB149A47CB04
:103A300089E50E94B6558111E1CF8AE50E94B6550D
:103A40008111DCCF85E40E94B6558111D7CF0F9448
:103A50001422149A0E94C47432CB179A1092A306AF
:103A6000D4CF83E50E94B655882309F428CB0E9461
:103A70008E5A20E030E04AE754E40F944A9B0F94BA
:103A80001DA360934603709347038093480390936C
:103A9000490315CB84EC882E82E0982E92E3A92E60
:103AA00094E0B92E10E0F40181914F010E94B655C7
:103AB000882309F465C00E948E5A6B017C01133083
:103AC00009F068C020E030E040EA51E40F949AA287
:103AD00087FF4EC0A7019601609142047091430494
:103AE00080914404909145040F94A4A22B013C01C1
:103AF000AC019B01609186047091870480918804D9
:103B0000909189040F944A9B609386047093870474
:103B10008093880490938904A301920160915204D8
:103B20007091530480915404909155040F944A9BD2
:103B300060935204709353048093540490935504FB
:103B40006091F1167091F2168091F3169091F4162F
:103B50000F94099BA30192010F944A9B0F941DA3FC
:103B60006093F1167093F2168093F3169093F41607
:103B7000C0924204D0924304E0924404F09245047F
:103B8000B4E0AB0EB11C1F5F143009F08CCF0F9462
:103B9000367595CAD5011496CD92DD92ED92FC92C0
:103BA0001797EECF83E50E94B655882329F00E942F
:103BB000CB558093320283CA87E79EE90E94E57065
:103BC000C0903202D12CF12CE12C83E990E80E94C4
:103BD000E5704AE0C701B6010F94CD960F949D9809
:103BE0006ECA85E50E94B655882309F45AC0009133
:103BF000F5161091F6160F5F1F4F1093F6160093EF
:103C0000F5168091B703882309F459CABE016F5F86
:103C10007F4FC8010E9411E1882309F450CA82E550
:103C200097E8DE011196BE01675F7F4FFC01459169
:103C300054912D913D914217530710F40C943CB0D0
:103C40002417350708F43BCA0296A617B70771F781
:103C500036CA80E699E30E943C6DAC0163E080E0E7
:103C60000E941A6A40E068EE73E082E390E00F94ED
:103C7000613184EF91E00E94D37C40E068EE73E014
:103C800082E390E00F9461318EE190E00F943D3437
:103C900081E00E944B6A0E94396A80E00E94CD69EF
:103CA0000ECA41E150E060E87CE0CE0101960F943D
:103CB0006DA085E790E80E94E57089ED9FE90E947C
:103CC000E57083E790E80E94E5708EE690E80E9438
:103CD000E5708CE690E80E94E57082E690E80E942C
:103CE000E57088E090E80E94E57084E090E80E942A
:103CF000E57085EF9FE70E94E570CE0101960E9476
:103D00002E7D83EE9FE70E94E57082EE9FE70E9482
:103D1000DE721F9201E3F02EFF928BE49EE79F93E9
:103D20008F9304E01EE71F930F930F943F9F1F9202
:103D3000FF928BE39EE79F938F931F930F930F94B4
:103D40003F9F1F92FF9287E29EE79F938F931F935F
:103D50000F930F943F9F1F92FF928AE19EE79F93DC
:103D60008F931F930F930F943F9F1F92FF928FE0AB
:103D70009EE79F938F931F930F930F943F9F0FB6D0
:103D8000F894DEBF0FBECDBF9AC90E94DC7197C9FF
:103D9000E091F516F091F616CF01049624812032B9
:103DA00009F401960E9453EF87E08093C70687C904
:103DB0000091F5161091F6160B5F1F4F83E0F12C62
:103DC00040E08150E9F0D8019C91292F2B7F2134CC
:103DD000B9F411962C91213399F4913471F0953402
:103DE00009F441E098012E5F3F4F89012F5F3F4F5B
:103DF000F80190819032C9F3E4CFFF24F394F2CF1D
:103E0000442321F087E79EE90E94E570FF2021F01E
:103E10008FED9FE70E94E570C8010F949E994FC9EE
:103E200089EF95E60C944E9489EF95E60C945C949A
:103E300089EF95E60C946A9489EF95E60C94789452
:103E40000E9428603CC984E50E94B655882369F029
:103E50000E94CB55882349F087E79EE90E94E570D0
:103E60008AEC95E60E942E7D2AC984E40E94B6550C
:103E7000882309F424C90E948E5A20E030E0A90169
:103E80000F949AA2811105C01092C9040E945D5F2F
:103E900016C90E948E5A6B017C0120E030E0A90116
:103EA0000F949AA2811106C0C12CD12C10EEE12EE4
:103EB0001FE3F12EC092CA04D092CB04E092CC044E
:103EC000F092CD0481E08093C904E0CF04EC12E0CD
:103ED000E2E3EE2EE4E0FE2EF8ECCF2EF2E0DF2E51
:103EE000D8018D918D010E94B655882339F00E942A
:103EF0008E5AF701648B758B868B978BF4E0EF0EEF
:103F0000F11CC016D10661F7DAC883E50E94B655E8
:103F1000882319F10E948E5A6093F2047093F3047F
:103F20008093F4049093F50460936604709367049F
:103F3000809368049093690484E50E94B6558823B1
:103F400009F4BDC80E948E5A60936A0470936B0492
:103F500080936C0490936D04B2C880E50E94B655BE
:103F6000882351F00E948E5A609366047093670410
:103F7000809368049093690482E50E94B655882373
:103F800051F00E948E5A60936A0470936B04809380
:103F90006C0490936D0484E50E94B655882309F45F
:103FA0008EC80E948E5A6093F2047093F30480933B
:103FB000F4049093F50483C804EC12E07AE8E72E49
:103FC00074E0F72ED8018D918D010E94B65588239B
:103FD00039F00E948E5AF701608371838283938344
:103FE000F4E0EF0EF11C22E0073C120759F767C816
:103FF00083E50E94B655882351F00E948E5A609343
:10400000B5047093B6048093B7049093B80486E423
:104010000E94B655882361F00E948E5A0E94586013
:104020006093B9047093BA048093BB049093BC046A
:104030008AE50E94B655882309F441C80E948E5A29
:104040006093BD047093BE048093BF049093C0043A
:1040500036C883E50E94B655882309F430C80E940B
:10406000CB558823B9F08130D1F087E79EE90E94D3
:10407000E57087EB95E60E94E5708091CB119091F9
:10408000CC118F51904F0E942E7D8AED9FE70E94A8
:10409000DE7215C81092B4041092030510C8809304
:1040A000B404109203050C945F984090F60450906D
:1040B000F7046090F8047090F9040C949B9580903C
:1040C000FA049090FB04A090FC04B090FD040C94C2
:1040D000A69582E40E94B655182F882341F080915E
:1040E0008E0290918F02909331028093300283E58B
:1040F0000E94B655082F882339F00E94D855909316
:104100008F0280938E02102F82E50E94B65588237D
:1041100051F0809130029091310290938F02809300
:104120008E020C945F9811110C945F9880918F020D
:104130008F9380918E028F9384ED9FE79F938F934F
:104140000F943F9F0F900F900F900F900C945F98DB
:1041500083E50E94B655882351F00E94D85590936C
:104160005A02809359020E945D5F0C945F9880917F
:104170005A028F93809159028F938EEC9FE79F9301
:104180008F930F943F9F0F900F900F900F900C9470
:104190005F9880E50E94B655882311F40C945F98CF
:1041A0000E94D8557C0183E50E94B6550FEF1FEFA2
:1041B000882319F00E94D8558C01C80101960397F5
:1041C00010F00C945F98E4EDF0E820EF30E8849173
:1041D000082E000C990BE816F90611F40C945F9860
:1041E00031962E173F0799F7F7FE02C00C945F989F
:1041F0000F941422DE2C60E08E2D0E943BC00F3FF6
:104200001007B1F00130110511F010E000E08D2D24
:104210000E94E4BF8017910711F40C945F980F94EB
:10422000F73180E00E948C7A80E00E94CD69EFCF68
:104230008E2D0E94E4BF31E020E0892B09F030E0B0
:10424000032F122FE4CF70E060E040E0C8010F942C
:1042500061310C945F9880E50E94B655882351F037
:104260000E948E5A60939A0470939B0480939C04DE
:1042700090939D0489E40E94B655882381F00E94A2
:104280008E5A2CEA35EC47E25EE30F944A9B60932A
:104290009E0470939F048093A0049093A10484E4EF
:1042A0000E94B655882381F00E948E5A2CEA35EC84
:1042B00047E25EE30F94A4A26093A2047093A30468
:1042C0008093A4049093A5040F94681885ED99E653
:1042D0000E94E5708AEC9FE70E94E57060919A0465
:1042E00070919B0480919C0490919D0442E00F94F6
:1042F000EA9786EC9FE70E94E5702CEA35EC47E2EE
:104300005EE360919E0470919F048091A00490915F
:10431000A1040F94A4A242E00F94EA9782EC9FE7D5
:104320000E94E5702CEA35EC47E25EE36091A2045E
:104330007091A3048091A4049091A5040F944A9BCA
:104340000F942B410C945F9880E50E94B65588230A
:1043500051F00E948E5A6093A6047093A704809334
:10436000A8049093A90489E40E94B655882381F09B
:104370000E948E5A2CEA35EC47E25EE30F944A9B8A
:104380006093AA047093AB048093AC049093AD0443
:1043900084E40E94B655882381F00E948E5A2CEA4C
:1043A00035EC47E25EE30F94A4A26093AE047093F1
:1043B000AF048093B0049093B1040F94681885ED16
:1043C00099E60E94E5708EEB9FE70E94E570609190
:1043D000A6047091A7048091A8049091A90442E0DA
:1043E0000F94EA978AEB9FE70E94E5702CEA35EC80
:1043F00047E25EE36091AA047091AB048091AC0443
:104400009091AD040F94A4A242E00F94EA9786EB3A
:104410009FE70E94E5702CEA35EC47E25EE360918D
:10442000AE047091AF048091B0049091B1040F94E8
:104430004A9B0F942B410C945F9883E50E94B655DC
:10444000882341F00E94D8559093580280935702D8
:104450000C945F9890E080E0F7CF85E090E00C94BA
:1044600071960F9414220C945F9881E00E94AB6EB9
:104470000C945F9880E00E94AB6E0C945F980E9451
:10448000C2730C945F980E94E7750C945F980E9429
:1044900056750C945F98809195048F938091940445
:1044A0008F93809193048F93809192048F93809146
:1044B00091048F93809190048F9380918F048F93B8
:1044C00080918E048F9380918D048F9380918C04C2
:1044D0008F9380918B048F9380918A048F9307E749
:1044E0001EE91F930F931F930F93809189048F935D
:1044F000809188048F93809187048F9380918604A4
:104500008F93809185048F93809184048F93809101
:1045100083048F93809182048F93809181048F9381
:10452000809180048F9380917F048F9380917E048B
:104530008F9380917D048F9380917C048F938091E1
:104540007B048F9380917A048F93809179048F9369
:10455000809178048F93809177048F938091760473
:104560008F93809175048F93809174048F938091C1
:1045700073048F93809172048F93809171048F9351
:10458000809170048F9380916F048F9380916E045B
:104590008F931F930F931F930F938091F5048F9325
:1045A0008091F4048F938091F3048F938091F204AF
:1045B0008F9380916D048F9380916C048F93809181
:1045C0006B048F9380916A048F93809169048F9319
:1045D000809168048F93809167048F938091660423
:1045E0008F931F930F931F930F93809165048F9365
:1045F000809164048F93809163048F93809162040F
:104600008F93809161048F93809160048F93809148
:104610005F048F9380915E048F9380915D048F93EC
:1046200080915C048F9380915B048F9380915A04F6
:104630008F93809159048F93809158048F93809128
:1046400057048F93809156048F931F930F931F935A
:104650000F93809155048F93809154048F93809190
:1046600053048F93809152048F93809151048F93C0
:10467000809150048F9380914F048F9380914E04CA
:104680008F9380914D048F9380914C048F938091F0
:104690004B048F9380914A048F93809149048F93A8
:1046A000809148048F93809147048F9380914604B2
:1046B0008F931F930F931F930F93809145048F93B4
:1046C000809144048F93809143048F93809142049E
:1046D0008F93809141048F93809140048F938091B8
:1046E0003F048F9380913E048F9380913D048F937C
:1046F00080913C048F9380913B048F9380913A0486
:104700008F93809139048F93809138048F93809197
:1047100037048F93809136048F931F930F931F93C9
:104720000F9389EF9BE79F938F930F943F9F0FB653
:10473000F894DEBF0FBECDBF2CEA35EC47E25EE356
:104740006091A2047091A3048091A4049091A504A7
:104750000F944A9B9F938F937F936F932CEA35EC32
:1047600047E25EE360919E0470919F048091A004F3
:104770009091A1040F94A4A29F938F937F936F9322
:1047800080919D048F9380919C048F9380919B04D2
:104790008F9380919A048F931F930F931F930F937E
:1047A0008CEC9BE79F938F930F943F9F2CEA35EC03
:1047B00047E25EE36091AE047091AF048091B00473
:1047C0009091B1040F944A9B9F938F937F936F9323
:1047D0002CEA35EC47E25EE36091AA047091AB04E9
:1047E0008091AC049091AD040F94A4A29F938F93F9
:1047F0007F936F938091A9048F938091A8048F93E6
:104800008091A7048F938091A6048F931F930F9399
:104810001F930F9387E99BE79F938F930F943F9F7D
:104820000FB6F894DEBF0FBECDBF8091B4041F92C7
:104830008F931F930F931F930F9320E030E040E777
:1048400052E46091C5047091C6048091C7049091B0
:10485000C8040F944A9B9F938F937F936F9380918B
:10486000C4048F938091C3048F938091C2048F936B
:104870008091C1048F931F930F931F930F93809187
:10488000C0048F938091BF048F938091BE048F9357
:104890008091BD048F9320E030E040E752E46091C6
:1048A000B9047091BA048091BB049091BC040F9438
:1048B0004A9B9F938F937F936F938091B8048F93BC
:1048C0008091B7048F938091B6048F938091B50443
:1048D0008F931F930F931F930F9386E99AE79F93EC
:1048E0008F930F943F9F0FB6F894DEBF0FBECDBFDE
:1048F0008091C904882309F456C08091CD048F9318
:104900008091CC048F938091CB048F938091CA04C3
:104910008F931F930F931F930F9380E79AE79F93B3
:104920008F930F943F9F0FB6F894DEBF0FBECDBF9D
:10493000809102058F93809101058F9380910005EE
:104940008F938091FF048F938091FE041F928F9329
:104950008091FD048F938091FC048F938091FB04E0
:104960008F938091FA048F938091F9048F938091B3
:10497000F8048F938091F7048F938091F6048F93BE
:1049800087E79EE99F938F939F938F938FEC99E78F
:104990009F938F930F943F9F0FB6F894DEBF0FBE87
:1049A000CDBF0C945F981F930F9381E59AE79F9377
:1049B0008F930F943F9F0F900F900F900F90B8CF51
:1049C00080E50E94B655882311F40C945F981092EC
:1049D0007D0610927E0610927F06109280060DE7EB
:1049E00016E031E8E32E36E0F32E4AE2D42EE091D1
:1049F000F516F091F616D0820E94D855D8018D9305
:104A00008D01EA16FB0611F40C945F988EE20E9469
:104A1000B6558111ECCF10927D0610927E06109251
:104A20007F06109280060C945F980F941422809158
:104A3000E711811102C00E94B95E85E40E94B6555B
:104A4000812C912CA12C20ECB22E882321F00E94E5
:104A50008E5A4B015C018CE40E94B655C12CD12CBE
:104A60007601882321F00E948E5A6B017C018AE531
:104A70000E94B655412C512C98ED692E91E4792E67
:104A8000882331F00E948E5A2B013C01E89477F87C
:104A900088E50E94B655882309F4B5C10E948E5A54
:104AA00068A779A78AA79BA789E50E94B65588239E
:104AB00009F4B2C10E948E5A6CA77DA78EA79FA74A
:104AC0001A821982FE01339683E1DF011D928A95D5
:104AD000E9F783E40E94B6558823F9F062E270E0BA
:104AE0008091F5169091F6160F94D4A68C01892B1F
:104AF000A1F00F5F1F4F62E270E0C8010F94D4A6CF
:104B0000009759F0801B843108F084E1482F50E071
:104B1000B801CE0101960F94A6A68091941210E0E0
:104B2000813029F481EA9FE70F94F274182F0F94D3
:104B3000142286E10F94A0981092E9110E94486116
:104B400081116FC1A501940160910112709102124F
:104B500080910312909104120F94A5A16093011209
:104B600070930212809303129093041260E070E03D
:104B700088EE92E40F9411850F9414228AED9AE640
:104B80000E94DE72C301B2010E94686728A539A5A0
:104B90004AA55BA52093F5113093F6114093F711C8
:104BA0005093F8118CA59DA5AEA5BFA58093F911D2
:104BB0009093FA11A093FB11B093FC1160E070E0A8
:104BC00088E492E40F9411850F941422B12CA12C47
:104BD0000BEB202E09E7302E83EC882E89E7982EE8
:104BE00080919412813009F01FC10F943041A82E9A
:104BF0000E94A76D0F9414221092861610928516AB
:104C000080919412813009F4D9C184E080937802B4
:104C10008EE399E30E943C6D40E060E00F94892DA3
:104C2000082F80E00E944B6A013029F50E94396A02
:104C300086EB99E30E943C6DAC0162E080E00E944B
:104C40001A6A80E090E0A8ECB2E48093F5119093AA
:104C5000F611A093F711B093F81160E070E088E4CA
:104C600092E40F9411850F9414228CE099E30E9432
:104C70003C6D0F94190B0E94396A8AE998E30E94EF
:104C80003C6DAC0160E080E00E941A6A61E080E067
:104C90000E94066A8981882341F0CE0101960E9414
:104CA0000D6C62E080E00E94066A80918516811199
:104CB00006C085E898E30E943C6D0E94F16984E09B
:104CC000809378020E94236C811110C00F94F731F9
:104CD00081E00E948C7A80918816882399F340E0C5
:104CE00068EE73E082E390E00F94613132E030933C
:104CF0007802CE0101960E94606D40E068EE73E09C
:104D000082E390E00F94613111119EC1B4E0BB2E9B
:104D1000B09278020E94396A86ED98E30E943C6D59
:104D2000AC0160E081E00E941A6A80EC98E30E9486
:104D30003C6DAC0161E081E00E941A6A8CEA98E364
:104D40000E943C6DAC0162E081E00E941A6A8CEB2B
:104D50009CE30E943C6DAC0163E081E00E941A6A12
:104D60004EE360E080E00E94266A0E941E6C00E034
:104D70000F94F73181E00E948C7A80910605909122
:104D800007050097D9F097FF22C1002309F423C13A
:104D9000015047EC59E760E080E00E941A6A4EE358
:104DA000602F80E00E94266A109207051092060587
:104DB00064E670E080E090E00F944D0D0E94236C5B
:104DC0008823B1F20E94396A0E94E9FD42E04093D3
:104DD0007802023009F408C1033009F4EDC1013052
:104DE00009F021C180919412813009F0F8C00F942C
:104DF0003041082F0E94A76D802F0E94F67C80E032
:104E00000E94A37185CF20E030E043E553E428A75A
:104E100039A74AA75BA748CE1CA61DA61EA61FA69B
:104E20004FCE0E94365FAECE84E0809378020F941E
:104E3000460F2B013C018AE598E30E943C6D0F94DC
:104E4000920A0E94236C082F811134C0A3019201A1
:104E50002054384D464F5F4F28A739A74AA75BA774
:104E60000F94F73181E00E948C7A023009F465C01A
:104E70000F94673584E090E0013029F10E94D37CE3
:104E80000F94460F28A539A54AA55BA52617370715
:104E900048075907B0F689E298E30E943C6D0F94E9
:104EA000920A1092F2111092F1110F941422149A96
:104EB00001E0D6CF10922B0510922E05C701B60146
:104EC0000E941EF097CE0E94D37C0E94236C882300
:104ED00039F28091EF119091F0119093F21180933B
:104EE000F11187E09FE40E943C6D0F94920A42E822
:104EF00064E080E00E94266A8091F2118F93809195
:104F0000F1118F936091C40D7091C50D8091C60D04
:104F10009091C70D0F9416A37F936F933F922F929A
:104F20000E94DF6981E80E94F5690F900F900F9051
:104F30000F900F900F9002E093CF6091F11170915C
:104F4000F211072E000C880B990B0F940B9B2091EC
:104F5000C40D3091C50D4091C60D5091C70D0F94F1
:104F6000A4A19F7720E030E040EA50E40F949AA299
:104F700087FF0BC08AE598E30E943C6D0F94920A6C
:104F80000F94460F2B013C015CCF64E081E00E944E
:104F9000066A6091C40D7091C50D8091C60D909107
:104FA000C70D0F9416A37F936F939F928F920E94C9
:104FB000DF690F900F900F900F9052CF111103C027
:104FC0008A2D0E94F67C812F0E94A3719DCE033012
:104FD00010F40F5FDECE87E00F94712CDACECE0195
:104FE00001960E94606D94CE0F9414220E94005F7F
:104FF0000E94396A8AEE98E30E943C6DAC0160E041
:1050000080E00E941A6A86EB99E30E943C6DAC0135
:1050100062E080E00E941A6A87E99DE10F94DD0B4F
:105020000F94142275CE0E94396A8AEF98E30E9489
:105030003C6DAC0162E080E00E941A6A002319F026
:10504000033009F065CEB12C84E896E10E947B6EB6
:10505000B110C6CD81E00E944B6A8091E811809327
:10506000E911111127C00E944861C0900112D0902F
:105070000212E0900312F0900412882309F49FC0FA
:1050800020E030E040E85FE3C701B6010F94A4A13F
:105090006093011270930212809303129093041292
:1050A00060E070E088EE92E40F9411851092F211A6
:1050B0001092F111E090FD11F090FE110091FF119E
